S01C00005354345F537065637472756D5F576F726B696E672E737265633B
S3150800800000000220AD710308FD710308FD71030825
S31508008010FD710308FD710308FD71030800000000E7
S31508008020000000000000000000000000FD710308C9
S31508008030FD71030800000000FD710308F9670308D5
S31508008040FD710308FD710308FD710308FD7103083E
S31508008050FD710308FD710308FD710308FD7103082E
S31508008060FD710308FD710308FD710308FD7103081E
S31508008070FD670308FD71030809680308FD71030815
S315080080801568030821680308FD710308FD710308D4
S31508008090FD710308FD710308FD710308FD710308EE
S315080080A0FD710308FD710308FD710308FD710308DE
S315080080B02D68030839680308FD710308FD71030874
S315080080C0FD710308FD710308FD710308FD710308BE
S315080080D0FD71030845680308516803085D680308CD
S315080080E0FD710308FD710308FD710308FD7103089E
S315080080F0FD710308FD710308FD710308696803082B
S31508008100FD71030875680308FD7103088168030893
S31508008110FD710308FD710308FD710308FD7103086D
S31508008120FD710308FD7103088D6803089968030843
S31508008130FD7103080000000000000000FD7103083F
S31508008140FD710308FD710308FD710308A56803089E
S31508008150FD710308B1680308BD680308FD710308CB
S31508008160FD710308FD710308FD710308FD7103081D
S31508008170FD710308FD710308FD7103080000000086
S3150800818000000000FD710308000000000000000068
S31508008190FD7103080000000000000000FD710308DF
S315080081A0000000000000000000000000FD71030848
S315080081B0FD710308FD710308FD710308FD710308CD
S30D080081C0FD7103084433221186
S315080081D010B5054C237833B9044B13B10448AFF3F3
S315080081E000800123237010BD380F00200000000016
S315080081F0E494040808B5034B1BB103490348AFF3DD
S31508008200008008BD000000003C0F0020E49404082C
S3150800821010F8012B11F8013B012A28BF9A42F7D022
S31508008220D01A7047034613F8012B002AFBD1181AF7
S315080082300138704700000000000000000000000040
S3150800824001F0FF01102A2BDB10F0070F08D010F8F9
S31508008250013B013A8B422DD010F0070F42B3F6D1FD
S31508008260F0B441EA012141EA014122F007047FF016
S3150800827000070023F0E80256083C85EA010586EA6D
S31508008280010685FA47F5A3FA87F586FA47F6A5FAA9
S3150800829087F68EB9EED1F0BC01F0FF0102F00702B5
S315080082A032B110F8013B013A83EA010313B1F8D160
S315080082B00020704701387047002D06BF3546033841
S315080082C0073815F0010F07D1013015F4807F02BF7A
S315080082D0013015F4C03F0130F0BC0138704700BFCB
S315080082E081F0004102E000BF83F0004330B54FEA59
S315080082F041044FEA430594EA050F08BF90EA020FC6
S315080083001FBF54EA000C55EA020C7FEA645C7FEA58
S31508008310655C00F0E2804FEA5454D4EB5555B8BF7B
S315080083206D420CDD2C4480EA020281EA030382EAEC
S31508008330000083EA010180EA020281EA0303362D7E
S3150800834088BF30BD11F0004F4FEA01314FF4801C51
S315080083504CEA113102D0404261EB410113F0004F63
S315080083604FEA03334CEA133302D0524263EB43031A
S3150800837094EA050F00F0A780A4F10104D5F1200EB8
S315080083800DDB02FA0EFC22FA05F2801841F1000113
S3150800839003FA0EF2801843FA05F359410EE0A5F1E7
S315080083A020050EF1200E012A03FA0EFC28BF4CF018
S315080083B0020C43FA05F3C01851EBE37101F00045CE
S315080083C007D54FF0000EDCF1000C7EEB00006EEBDB
S315080083D00101B1F5801F1BD3B1F5001F0CD3490865
S315080083E05FEA30004FEA3C0C04F101044FEA4452BC
S315080083F012F5800F80F09A80BCF1004F08BF5FEA43
S31508008400500C50F1000041EB045141EA050130BD22
S315080084105FEA4C0C404141EB0101013C28BFB1F534
S31508008420801FE9D291F0000F04BF01460020B1FA7F
S3150800843081F308BF2033A3F10B03B3F120020CDA52
S315080084400C3208DD02F1140CC2F10C0201FA0CF030
S3150800845021FA02F10CE002F11402D8BFC2F1200C95
S3150800846001FA02F120FA0CFCDCBF41EA0C0190404B
S31508008470E41AA2BF01EB0451294330BD6FEA040494
S315080084801F3C1CDA0C340EDC04F11404C4F120027F
S3150800849020FA04F001FA02F340EA030021FA04F391
S315080084A045EA030130BDC4F10C04C4F1200220FAE8
S315080084B002F001FA04F340EA0300294630BD21FA26
S315080084C004F0294630BD94F0000F83F4801306BFEC
S315080084D081F480110134013D4EE77FEA645C18BFE0
S315080084E07FEA655C29D094EA050F08BF90EA020F77
S315080084F005D054EA000C04BF1946104630BD91EA6F
S31508008500030F1EBF0021002030BD5FEA545C05D171
S315080085104000494128BF41F0004130BD14F58004B0
S315080085203CBF01F5801130BD01F0004545F0FE4124
S3150800853041F470014FF0000030BD7FEA645C1ABF59
S31508008540194610467FEA655C1CBF0B46024650EA90
S31508008550013406BF52EA033591EA030F41F40021BC
S3150800856030BD00BF90F0000F04BF0021704730B542
S315080085704FF4806404F132044FF000054FF0000117
S3150800858050E700BF90F0000F04BF0021704730B5D8
S315080085904FF4806404F1320410F0004548BF4042AD
S315080085A04FF000013EE700BF42004FEAE2014FEA02
S315080085B031014FEA02701FBF12F07F4393F07F4FDD
S315080085C081F06051704732F07F4208BF704793F0E0
S315080085D07F4F04BF41F40021704730B54FF46074F3
S315080085E001F0004521F000411CE700BF50EA0102F6
S315080085F008BF704730B54FF000050AE050EA01029F
S3150800860008BF704730B511F0004502D5404261EB0E
S3150800861041014FF4806404F132045FEA915C3FF44F
S31508008620D8AE4FF003025FEADC0C18BF03325FEAEC
S31508008630DC0C18BF033202EBDC02C2F1200300FA9D
S3150800864003FC20FA02F001FA03FE40EA0E0021FAC2
S3150800865002F11444BDE600BF70B54FF0FF0C4CF4B0
S31508008660E06C1CEA11541DBF1CEA135594EA0C0F62
S3150800867095EA0C0F00F0DEF82C4481EA030621EA9D
S315080086804C5123EA4C5350EA013518BF52EA0335D8
S3150800869041F4801143F4801338D0A0FB02CE4FF08A
S315080086A00005E1FB02E506F00042E0FB03E54FF0BA
S315080086B00006E1FB03569CF0000F18BF4EF0010EB2
S315080086C0A4F1FF04B6F5007F64F5407404D25FEAAE
S315080086D04E0E6D4146EB060642EAC62141EA555161
S315080086E04FEAC52040EA5E504FEACE2EB4F1FD0CA3
S315080086F088BFBCF5E06F1ED8BEF1004F08BF5FEA21
S31508008700500E50F1000041EB045170BD06F00046D2
S3150800871046EA010140EA020081EA0301B4EB5C047F
S31508008720C2BFD4EB0C0541EA045170BD41F4801177
S315080087304FF0000E013C00F3AB8014F1360FDEBF9C
S31508008740002001F0004170BDC4F10004203C35DA78
S315080087500C341BDC04F11404C4F1200500FA05F3FB
S3150800876020FA04F001FA05F240EA020001F000429C
S3150800877021F0004110EBD37021FA04F642EB060112
S315080087805EEA430E08BF20EAD37070BDC4F10C043C
S31508008790C4F1200500FA04F320FA05F001FA04F200
S315080087A040EA020001F0004110EBD37041F10001EC
S315080087B05EEA430E08BF20EAD37070BDC4F12005F7
S315080087C000FA05F24EEA020E20FA04F301FA05F25F
S315080087D043EA020321FA04F001F0004121FA04F207
S315080087E020EA020000EBD3705EEA430E08BF20EAD7
S315080087F0D37070BD94F0000F0FD101F00046400011
S3150800880041EB010111F4801F08BF013CF7D041EA92
S31508008810060195F0000F18BF704703F00046520096
S3150800882043EB030313F4801F08BF013DF7D043EA67
S315080088300603704794EA0C0F0CEA135518BF95EA1D
S315080088400C0F0CD050EA410618BF52EA4306D1D1A4
S3150800885081EA030101F000414FF0000070BD50EAC3
S31508008860410606BF1046194652EA430619D094EA4D
S315080088700C0F02D150EA013613D195EA0C0F05D137
S3150800888052EA03361CBF104619460AD181EA03018B
S3150800889001F0004141F0FE4141F470014FF0000043
S315080088A070BD41F0FE4141F4780170BD70B54FF0DE
S315080088B0FF0C4CF4E06C1CEA11541DBF1CEA13555E
S315080088C094EA0C0F95EA0C0F00F0A7F8A4EB050440
S315080088D081EA030E52EA03354FEA013100F0888037
S315080088E04FEA03334FF0805545EA131343EA126300
S315080088F04FEA022245EA111545EA10654FEA0026B5
S315080089000EF000419D4208BF964244F1FD0404F56D
S31508008910407402D25B084FEA3202B61A65EB0305C9
S315080089205B084FEA32024FF480104FF4002CB6EB86
S31508008930020E75EB030E22BFB61A754640EA0C0006
S315080089405B084FEA3202B6EB020E75EB030E22BF46
S31508008950B61A754640EA5C005B084FEA3202B6EB87
S31508008960020E75EB030E22BFB61A754640EA9C0046
S315080089705B084FEA3202B6EB020E75EB030E22BF16
S31508008980B61A754640EADC0055EA060E18D04FEAD4
S31508008990051545EA16754FEA06164FEAC30343EA74
S315080089A052734FEAC2025FEA1C1CC0D111F4801F41
S315080089B00BD141EA00014FF000004FF0004CB6E73A
S315080089C011F4801F04BF01430020B4F1FD0C88BFD9
S315080089D0BCF5E06F3FF6AFAEB5EB030C04BFB6EBE4
S315080089E0020C5FEA500C50F1000041EB045170BDD7
S315080089F00EF0004E4EEA113114EB5C04C2BFD4EB04
S31508008A000C0541EA045170BD41F480114FF0000E87
S31508008A10013C90E645EA060E8DE60CEA135594EA03
S31508008A200C0F08BF95EA0C0F3FF43BAF94EA0C0F06
S31508008A300AD150EA01347FF434AF95EA0C0F7FF47B
S31508008A4025AF104619462CE795EA0C0F06D152EACF
S31508008A5003353FF4FDAE1046194622E750EA4106B3
S31508008A6018BF52EA43067FF4C5AE50EA41047FF4C4
S31508008A700DAF52EA43057FF4EBAE12E74FF0FF3C29
S31508008A8006E000BF4FF0010C02E000BF4FF0010CFA
S31508008A904DF804CD4FEA410C7FEA6C5C4FEA430C73
S31508008AA018BF7FEA6C5C1BD001B050EA410C0CBFC2
S31508008AB052EA430C91EA030F02BF90EA020F002024
S31508008AC0704710F1000F91EA030F58BF994208BF8B
S31508008AD090422CBFD8176FEAE37040F00100704748
S31508008AE04FEA410C7FEA6C5C02D150EA013C07D19F
S31508008AF04FEA430C7FEA6C5CD6D152EA033CD3D0EA
S31508008B005DF8040B704700BF8446104662468C46E3
S31508008B101946634600E000BF01B5FFF7B7FF002816
S31508008B2048BF10F1000F01BD4DF808EDFFF7F4FF3F
S31508008B300CBF012000205DF808FB00BF4DF808EDCA
S31508008B40FFF7EAFF34BF012000205DF808FB00BFED
S31508008B504DF808EDFFF7E0FF94BF012000205DF80F
S31508008B6008FB00BF4DF808EDFFF7CEFF94BF0120C4
S31508008B7000205DF808FB00BF4DF808EDFFF7C4FFBD
S31508008B8034BF012000205DF808FB00BF4FEA410C06
S31508008B907FEA6C5C02D150EA013C0AD14FEA430CE9
S31508008BA07FEA6C5C02D152EA033C02D14FF0000026
S31508008BB070474FF0010070474FEA410212F5001264
S31508008BC015D211D56FF47873B3EB625212D94FEA06
S31508008BD0C12343F0004343EA505311F0004F23FAF0
S31508008BE002F018BF404270474FF00000704750EA45
S31508008BF0013005D111F0004008BF6FF00040704702
S31508008C004FF00000704700BF4A0011D212F500125B
S31508008C1011D20DD56FF47873B3EB62520ED44FEAC6
S31508008C20C12343F0004343EA505323FA02F0704746
S31508008C304FF00000704750EA013002D14FF0FF3084
S31508008C4070474FF0000070474FEA4102B2F1E04327
S31508008C5024BFB3F5001CDCF1FE5C0DD901F0004C15
S31508008C604FEAC0024CEA5070B2F1004F40EB830065
S31508008C7008BF20F00100704711F0804F21D113F191
S31508008C803872BCBF01F00040704741F480114FEACA
S31508008C905252C2F11802C2F1200C10FA0CF320FA53
S31508008CA002F018BF40F001004FEAC1234FEAD32370
S31508008CB003FA0CFC40EA0C0023FA02F34FEA4303DA
S31508008CC0CCE77FEA625307D150EA01331EBF4FF063
S31508008CD0FE4040F44000704701F0004040F0FE407E
S31508008CE040F40000704700BF53B94AB9002908BFCD
S31508008CF000281CBF4FF0FF314FF0FF3000F0A4B939
S31508008D00ADF1080C6DE904CE00F03CF8DDF804E09E
S31508008D10DDE9022304B0704738B500220023044673
S31508008D200D46FFF70BFF28B920462946BDE838400F
S31508008D3000F00AB8204605F1004100F005F8404267
S31508008D4061EB410138BD00BFD0B50C4B0022064689
S31508008D500F46FFF781FCFFF757FF0446FFF702FCB3
S31508008D60074B0022FFF778FC02460B463046394689
S31508008D70FFF7BAFAFFF748FF2146D0BD0000F03DDD
S31508008D800000F0412DE9F047089D04468C46002B6B
S31508008D9040F083808A42174647D9B2FA82F242B136
S31508008DA0C2F1200024FA00F09140974040EA010CF5
S31508008DB094404FEA1748230CBCFBF8F61FFA87FEC7
S31508008DC008FB16C143EA014306FB0EF1994209D98D
S31508008DD0FB1806F1FF3080F01981994240F216819E
S31508008DE0023E3B445B1AA4B2B3FBF8F008FB10330F
S31508008DF044EA034400FB0EFEA64509D93C1900F1D6
S31508008E00FF3380F00581A64540F2028102383C44D2
S31508008E1040EA0640A4EB0E0400261DB1D440002308
S31508008E20C5E900433146BDE8F08702B9FFDEB2FA6C
S31508008E3082F2002A50D1CB1B4FEA174E1FFA87F849
S31508008E400126B3FBFEFC210C0EFB1C3341EA034151
S31508008E5008FB0CF38B4207D979180CF1FF3002D2C4
S31508008E608B4200F2E9808446C91AA3B2B1FBFEF030
S31508008E700EFB101143EA014408FB00F8A04507D988
S31508008E803C1900F1FF3302D2A04500F2D9801846FA
S31508008E90A4EB080440EA0C40BFE78B4209D9002D31
S31508008EA000F0B1800026C5E9000130463146BDE82C
S31508008EB0F087B3FA83F6002E4AD18B4202D3824258
S31508008EC000F2B880841A61EB030101208C46002D5C
S31508008ED0A8D0C5E9004CA5E7C2F1200320FA03F69D
S31508008EE0974001FA02F04FEA174ED9403043030C77
S31508008EF0B1FBFEF61FFA87F80EFB161143EA01438B
S31508008F0006FB08F1994204FA02F409D9FB1806F19E
S31508008F10FF3C80F08D80994240F28A80023E3B44B5
S31508008F205B1A81B2B3FBFEF00EFB103341EA034134
S31508008F3000FB08F38B4207D9791800F1FF3C73D27E
S31508008F408B4271D902383944CB1A40EA064678E78B
S31508008F50C6F1200C03FA06F422FA0CF31C4320FA95
S31508008F600CF701FA06F34FEA144E21FA0CF11F43E7
S31508008F703B0CB1FBFEF91FFA84F80EFB191143EA04
S31508008F80014109FB08FA8A4502FA06F200FA06F3D5
S31508008F9008D9611809F1FF3048D28A4546D9A9F19E
S31508008FA002092144A1EB0A01BFB2B1FBFEF00EFB98
S31508008FB0101147EA014700FB08F8B84507D9E71931
S31508008FC000F1FF312ED2B8452CD90238274440EAA1
S31508008FD00940A7EB0807A0FB02894F45C646494644
S31508008FE01AD317D05DB1B3EB0E0267EB010707FA88
S31508008FF00CFCF2404CEA0202F740C5E900270026BD
S315080090003146BDE8F0872E4628460BE70646E9E6D0
S315080090101846FDE64345E5D2B8EB020E69EB0401B6
S315080090200138DFE70846D2E760468DE78146B9E7AB
S31508009030664675E730464AE7ACF1020C394413E751
S3150800904002383C4424E700BF704700BFF8B572B148
S3150800905006460C468F180025336814F8011B1B6852
S3150800906030469847A7420544F6D12846F8BD154626
S315080090702846F8BD2DE9F8430668DFF87C9077683E
S3150800908004460D4659B30846FFF7CCF84F458046C7
S3150800909027D160B12F184FF00008336815F8011B67
S315080090A020469847BD4226688044F6D177684F45E2
S315080090B00ED133680D212046984722680346126868
S315080090C020460A211C46904720444044BDE8F883C0
S315080090D0084920460222B8474044BDE8F883884636
S315080090E0E5E7024629462046B84726688046776857
S315080090F0DDE700BFB89604084D9000084FF0FF3032
S31508009100704700BF704700BF10B54FF0FF331446D5
S31508009110006992B233F09AFB204610BD00B583B0C1
S315080091204FF0FF3301220DF10701006933F03CFCD3
S315080091309DF8070003B05DF804FB00BF10B504688E
S315080091400B4A646882B094428DF807100AD14FF032
S31508009150FF3301220DF10701006933F077FB012087
S3150800916002B010BD01220DF10701A04702B010BDE3
S3150800917009910008F8B50026C0E90066044686602D
S3150800918079B108460D46FFF74DF8074601303BF022
S31508009190D5FE30B1C4E900070670A76029463CF041
S315080091A005FD2046F8BD00BFF8B588424FF000051A
S315080091B0C0E90055044685600DD00E685EB18F681B
S315080091C0781C3BF0BBFE30B1C4E900070570A76008
S315080091D031463CF0EBFC2046F8BD00BF30B4D1E97F
S315080091E000258C6802600022C0E90154C1E900220A
S315080091F030BC8A60704700BF10B5044600683BF073
S31508009200A5FE204610BD00BF884270B504461FD093
S315080092100D680068ADB18E6810B163689E4209D9C1
S31508009220711C3CF0F7FB58B1A368C4E900060BB9FA
S3150800923003702068A66029463CF0B8FC204670BD3D
S31508009240206808B13BF082FE0023C4E9013323609D
S31508009250204670BD884238B5044612D000680D46CF
S3150800926028B162688B689A420DD23BF06FFED5E949
S315080092700031AA6823600023C4E90112C5E9003356
S31508009280AB60204638BD09683CF090FCAB68A3602B
S315080092900023AB60204638BD70B50446E1B10846E8
S315080092A00D46FEF7BFFF2368064613B16268904273
S315080092B00BD91846711C3CF0ADFB034660B1A26899
S315080092C0C4E900060AB902702368A660294618464A
S315080092D03CF06CFC204670BD206808B13BF036FEB9
S315080092E00023C4E901332360204670BD30B5836886
S315080092F083B0044600688DF8041000225D1C8DF8C2
S31508009300052010B1626895420AD9991C3CF082FB87
S3150800931060B1A368C4E9000513B903702068A3689F
S31508009320184401A93CF042FCA560012003B030BDF9
S31508009330826808B50B463AB161B10068FEF768FF66
S31508009340B0FA80F0400908BD31B11878B0FA80F05B
S31508009350400908BD0368F8E7012008BD82688A420B
S3150800936003D9006808B1084470470248002303700F
S31508009370704700BF540F00208368934207D910B581
S315080093800468A0183CF005FC20B1001B10BD4FF086
S31508009390FF3070474FF0FF3010BD00BF9A422DE9ED
S315080093A0F0411746984604460D4601D94746904669
S315080093B00026C4E90066A66001203BF0BFFD08B19F
S315080093C020600670AE68BE4202D82046BDE8F0812D
S315080093D046452B6828BF4646002213F806809A554C
S315080093E0296820463944FFF757FF2B6803F806809B
S315080093F02046BDE8F08100BF006808B13BF06FBDAC
S31508009400704700BF30B5851840F2FE34A54285B0D6
S315080094101BDCFF280B4616D9B0F5007F18D3B0F52C
S31508009420407F34BFA421A6210E24CDE90032029440
S31508009430C2B2012307482FF0C5F904202DF030FFEA
S31508009440012005B030BDA021EEE7002005B030BDF3
S31508009450A221E9E7F4AE012030B5851840F2FE34C2
S31508009460A54285B01BDCFF280B4616D9B0F5007F50
S3150800947018D3B0F5407F34BFA421A6210E24CDE928
S3150800948000320294C2B2012307482FF09BF9042048
S315080094902DF006FF012005B030BDA021EEE7002023
S315080094A005B030BDA221E9E7F4AE012010B50B885E
S315080094B086B0841840F2FE315BBA8C42ADF814309F
S315080094C01BDCFF2817D9B0F5007F19D3B0F5407F0C
S315080094D034BFA421A62105AB0E2401920093C2B283
S315080094E00123029407482FF06DF904202DF0D8FEC9
S315080094F0012006B010BDA021EDE7002006B010BD82
S31508009500A221E8E7F4AE012010B50B6886B08418EE
S3150800951040F2FE311BBA8C4205931BDCFF2817D993
S31508009520B0F5007F19D3B0F5407F34BFA421A6213A
S3150800953005AB0E2401920093C2B201230294084897
S315080095402FF040F904202DF0ABFE012006B010BD27
S31508009550A021EDE7002006B010BDA221E8E700BF74
S31508009560F4AE012030B5851840F2FE34A54285B028
S3150800957018DCFF280B4613D9B0F5007F15D3B0F5D4
S31508009580407F34BFA521A7210E24CDE900320294DD
S31508009590C2B2012306482FF009FA012005B030BDF2
S315080095A0A121F1E7002005B030BDA321ECE700BFFB
S315080095B0F4AE012030B540F2FE3384189C4287B0E1
S315080095C020DCFF280D461BD9B0F5007F1DD3B0F56A
S315080095D0407F34BFA521A72105AB0E240192009335
S315080095E0C2B2029401230A482FF0E0F99DF814202C
S315080095F09DF81530012043EA02232B8007B030BDC1
S31508009600A121E9E7002007B030BDA321E4E700BFA8
S31508009610F4AE012030B5851840F2FE34A54285B077
S3150800962018DCFF280B4613D9B0F5007F15D3B0F523
S31508009630407F34BFA521A7210E24CDE9003202942C
S31508009640C2B2012306482FF0B1F9012005B030BD9A
S31508009650A121F1E7002005B030BDA321ECE700BF4A
S31508009660F4AE012030B540F2FE3384189C4287B030
S315080096701CDCFF280D4617D9B0F5007F19D3B0F5C5
S31508009680407F34BFA521A72105AB0E240192009384
S31508009690C2B20294012308482FF088F9059B0120DD
S315080096A01BBA2B6007B030BDA121EDE7002007B03B
S315080096B030BDA321E8E700BFF4AE01202DE9F04153
S315080096C0044682B001464C2200F5FC703BF046FC8D
S315080096D094F86D5294F8653294F86C1294F864E232
S315080096E094F8710294F8696294F8752294F868728D
S315080096F094F8748294F867C29FED657A2D0445EA5A
S3150800970001611B0494F8705243EA0E63000494F84E
S315080097106FE240EA056094F86E5281EA0E0141EA6A
S315080097200521360494F8775294F86AE261641204C3
S3150800973046EA076642EA086294F86B7294F87282FF
S3150800974083EA0C036A4094F866C2D4F85852019525
S315080097507E40D4F8505294F8737243EA0C2346EAD2
S315080097600E2605EB030C94F876E2019DE363784038
S31508009770D4F85472266442EA0E2237440D4440EA6D
S315080097800820C4E900C7C4E90250226194F88D2272
S3150800979094F88C0294F88F7294F878E294F87952D7
S315080097A084F83B70120442EA006245EA0E257A40C4
S315080097B094F87CE294F87D7294F87AC294F87B0265
S315080097C0258347EA0E27A783D4F87E72676240EAA4
S315080097D00C20D4F8827294F88EC294F890E294F829
S315080097E094526083C4F82E7094F89102D4F8867265
S315080097F0C4F83270D4F88A72C4F8367042EA0C2279
S3150800980040EA0E2094F8937294F892E26261803DE1
S3150800981084F83AC02562A08584F848E084F849703F
S3150800982094F89522803A07EE902AF8EEE77A67EEE2
S31508009830877AC4ED0A7A20B3B4F8242282420ED07D
S31508009840D4E97F52A4F8F401D4F8F801AE1B511AF2
S31508009850C31AC4F85462C4F85812C4F8503294F8BB
S31508009860773094F89720A3EB0E0EBA42BEFA8EFE16
S315080098704FEA5E1E0CBF0123002384F84AE084F8F1
S315080098804B30012384F85C3202B0BDE8F08100BF9A
S31508009890CDCCCC3DF0B504460D468FB000F25D2028
S315080098A004F25E213C223BF067FB94F85D3284F8B3
S315080098B09952492B01D00FB0F0BD94F85E32572B60
S315080098C0F9D194F85F32412BF5D194F86032502BD8
S315080098D0F1D194F86132492BEDD194F86232022B1A
S315080098E040F0AA8094F897323B2B40F0AC8094F86D
S315080098F09832212B40F0A7803B2D40F0A48004F23B
S31508009900622501AF04F2922C28686968AA68EB6898
S315080099103E460FC6103565453746F5D1286830608E
S31508009920DDE90132DDE9030103F07F35534002F03A
S315080099307F322A4403F080335340434002F07F329B
S3150800994000F07F30024403F0803353404B4002F06E
S315080099507F3201F07F315018DDE9052503F08033A9
S315080099604340534000F07F3002F07F32024403F058
S31508009970803353406B4002F07F3205F07F352A442E
S31508009980079903F080335340DDE908054B4002F0A0
S315080099907F3201F07F310A4403F08033534043405D
S315080099A002F07F3200F07F30024403F080335340E8
S315080099B06B4002F07F3205F07F352A440A9903F09E
S315080099C0803353404B4002F07F3201F07F318D18CF
S315080099D0DDE90B0203F080336B40434005F07F3529
S315080099E000F07F30284403F080334340534000F0B2
S315080099F07F3002F07F320D99024403F080335340E2
S31508009A004B4002F07F3201F07F310A4403F0803385
S31508009A105340C3F307221A44C3F307410A4402EB2F
S31508009A20136394F89622DBB29A420ED120460FB001
S31508009A30BDE8F040FFF742BE054906480FB0BDE84D
S31508009A40F040FFF717BB0449F7E70449F5E700BFFD
S31508009A50DC960408DC1A0020FC960408EC96040838
S31508009A6030B4C47B029D8583013414F0FF0408BF1B
S31508009A700124C473C0E9041230BC8361704700BF77
S31508009A8090F85C320BB91846704716490A7830B414
S31508009A900025012480F85C5280F818411AB1134653
S31508009AA0184630BC7047104A90F82E405578A542A3
S31508009AB018BF5470957890F82F40A54218BF947037
S31508009AC0D57890F8304090F83100A54218BFD47088
S31508009AD01479844218BF10710122184630BC0A70E6
S31508009AE0704700BF550F0020580F0020044B828D89
S31508009AF0198891421ABF01201A800020704700BFBA
S31508009B00560F002070B50446034694F84912D0F85B
S31508009B10450294F84422C4F8190184F81D1184F802
S31508009B201E21B4F8F45120686168A268A4F81F5190
S31508009B30C4F82921C4F82101C4F8251153F84C1F8B
S31508009B4094F864205868C4F83101C4F82D111B7ABA
S31508009B5084F83531234684F8362153F8551F5A6858
S31508009B609868C4F83F01C4F83711C4F83B219A89AC
S31508009B709B7B84F845312346A4F8432153F8681F94
S31508009B80A66F5A689868C4F84E01C4F84611C4F816
S31508009B904A219A899B7B84F85431A4F8522123469A
S31508009BA0E56FD4F88000B4F8841094F87720C4F8E8
S31508009BB05561C4F85951C4F85D01A4F8611184F8D7
S31508009BC0632153F8881FD4F89C505A689868C4F8DB
S31508009BD06C01C4F86411C4F868219A899B7BD4F88F
S31508009BE0A000A4F8702184F87231D4F89830C4F82B
S31508009BF07331B4F8A41094F89720C4F87751234623
S31508009C00C4F87B01A4F87F1184F8812153F8A81FB2
S31508009C105A689868C4F88A01C4F88211C4F886217B
S31508009C209A899B7B84F890312346A4F88E2153F8B1
S31508009C30B71F5A689868C4F89901C4F89111C4F80E
S31508009C4095219A899B7B84F89F312346A4F89D2108
S31508009C5053F8C60F9A685968C4F8A001C4F8A41145
S31508009C60C4F8A8219A899B7B84F8AE312346A4F8C8
S31508009C70AC2153F8D51F5A689868C4F8B701C4F8D8
S31508009C80AF11C4F8B3219A899B7B84F8BD3123466A
S31508009C90A4F8BB2153F8E41F5A689868C4F8C601AB
S31508009CA0C4F8BE11C4F8C2219A899B7B84F8CC31CA
S31508009CB02346A4F8CA2153F8F31F5A689868C4F8CB
S31508009CC0D501C4F8CD11C4F8D1219A899B7B84F8B3
S31508009CD0DB31B6B0D4F80801D4F80C11D4F8045125
S31508009CE0D4F81431A4F8D921D4F81021C4F8E00125
S31508009CF0C4F8E411C4F8E82104F58F71C4F8DC51FE
S31508009D00C4F8EC3101A8D2223BF028F935AE01A8F7
S31508009D10002150F8043B01F07F3503F07F324B40B9
S31508009D2003F080332A44B04282EA0301F1D19DF858
S31508009D30D4209DF8D530B4F84A02A4F8F1011344AA
S31508009D400B44C1F307221344C1F30742134494F8A2
S31508009D504C2284F8F32103EB116384F8F03136B012
S31508009D6070BD00BF012910D0022905D003291ED0D5
S31508009D70042913D000207047114B90F82F209978AA
S31508009D809142F7D09A70012070470D4B90F82E201B
S31508009D9058789042EED05A7008467047084B90F8AB
S31508009DA0312019799142E5D01A7101207047044B88
S31508009DB090F83020D9789142DCD0DA7001207047CB
S31508009DC0580F00200020704700207047704700BFDA
S31508009DD000207047704700BF002070472DE9F0410A
S31508009DE004460D4600F002FCA36B217CDBB9204635
S31508009DF000F030FC334F344E002D54D1334BA1685C
S31508009E0033481D8808F0A6FD3188A3683A782D1ACC
S31508009E1005EBD57501EB650189B231802C48BDE8A3
S31508009E20F04108F033BD0139C9B2204600F012FCF2
S31508009E30244F254E002D3DD1A268264926483BF0E1
S31508009E4045FE224B244922481D8808F083FD3188A7
S31508009E50214B3A780D442D1AA9B21D48318008F0D5
S31508009E6015FDA36A1B784FF00C08302518FB035321
S31508009E70E358B3B1217C01312046C9B200F0EAFBB0
S31508009E80A36A16491B78144818FB035562593BF018
S31508009E901DFE3A783188104B0D48BDE8F04108F0B0
S31508009EA0F5BCBDE8F0813A7831880D4B084808F0D2
S31508009EB0EDFCA3E73A783188094B054808F0E6FC3B
S31508009EC0BAE700BF740F0020760F0020780F002035
S31508009ED02CAE01200C970408600F002098F804089F
S31508009EE0089704081C303BF061BE00BF2DE9F04717
S31508009EF082B00225074600951E46DDE90A9300F062
S31508009F0047FB3B46154A43F81C2B07F13005002250
S31508009F10DFF84CA0FA612C465A601A8107F16008EE
S31508009F20204651460C34FFF725F94445F8D156B179
S31508009F30314628460C35FFF767F9454506F10C0604
S31508009F40F6D10C9BBB62B9F1000F01D0C7F82C9073
S31508009F5001233846FB7102B0BDE8F0871C97040858
S31508009F6024F1040810B5044600F000FBE06A10BDB1
S31508009F70704700BF2DE9F04F044685B00D4600F046
S31508009F8035FB217CDFF890815B4E204600F062FBB2
S31508009F90002D40F0A880A268584959483BF096FD24
S31508009FA0584B574958481D8808F0D4FC3188544BFB
S31508009FB098F800200D442D1AA9B25348318008F0AC
S31508009FC065FC217C25790231C9B22046002D33D1A2
S31508009FD000F040FB4D494C4808F0BCFC63693288E8
S31508009FE09B681044308023B3474FDFF830913846DA
S31508009FF0032108F013FE94F82830AB42384641D0C6
S3150800A000D4F8D43098F800205B57318804EB8303E2
S3150800A0100135DB6B039308F039FC039B3846194678
S3150800A02008F098FC636932889B681044AB4230801C
S3150800A030DDD805B0BDE8F08F00F00CFBE26A3449C4
S3150800A0402F483BF043FD98F800202D4B31882E48C9
S3150800A05008F01CFCE16A2C4808F07CFC626934882C
S3150800A06012682B4903462344254833803BF02EFDCE
S3150800A07098F800203188224B234805B0BDE8F04FF8
S3150800A08008F004BC94F9393098F80020B6F800B006
S3150800A090039204EB83030135D3F83CA0514608F03C
S3150800A0A059FC99F80010039A009103465946384618
S3150800A0B009F07CF80021384608F0B0FD98F8002031
S3150800A0C031885346384608F0E1FB5146384608F0D1
S3150800A0D041FC636932889B681044AB42308086D85D
S3150800A0E005B0BDE8F08F98F800203188094B06487E
S3150800A0F008F0CCFB4FE700BF760F00200C9704084A
S3150800A100600F0020780F00202CAE01200CE3040815
S3150800A11098F8040808970408740F00207A0F00209E
S3150800A120F8B50B780B3B0446202B34D8DFE803F050
S3150800A13011433334333343333433333333333333E1
S3150800A14033333333333333333333333333333333D1
S3150800A150630090F82830D0F8D42090F93910D154FB
S3150800A160406994F828308268013A93424DD2013307
S3150800A17094F83820DBB284F8283062B10168C95CEB
S3150800A180914208D1D4F8D4202521D15494F8283006
S3150800A190013384F82830F8BD90F8393090F8E0207B
S3150800A1A0013B5BB280F83930F2B9002BF3DA23238E
S3150800A1B084F83930F8BD90F8393090F8E02001334A
S3150800A1C05BB280F839302AB9232BE4DD002384F802
S3150800A1D03930F8BD012A3FD0022ADCD1232BDADD3B
S3150800A1E01A2384F83930F8BD012A2FD0022AD2D191
S3150800A1F0192BDCDDF8BD90F828301BB1013B80F83F
S3150800A2002830F8BD43790371F8BD237E04F11C0696
S3150800A210ABB10025D4F8D4305B5704EB8302252B69
S3150800A220294630460CBFD4F8D070D76BFFF796F89E
S3150800A2303B780370237E0135AB42EBDC606931461F
S3150800A240FEF7E2FF40F20113A380F8BD002BA2DA65
S3150800A250192380F83930F8BD192BB7DCF8BD00BFD3
S3150800A26010B50446D0F8D400074B236008B139F07E
S3150800A270AFFC04F12C00FEF7BFFF04F11C00FEF74B
S3150800A280BBFF204610BD00BFB89704082DE9F84F5C
S3150800A290D0E900960546A6EB09036FF00040834215
S3150800A2A051D08A469346002B48D0B3EB430F4FEA6A
S3150800A2B0430831D98046AAEB0904404639F08AFC9E
S3150800A2C0074680449BF800303B55002C0FDCA6EB74
S3150800A2D00A060134002E3C4426DC3444B9F1000F4A
S3150800A2E011D1C5E90074C5F80880BDE8F88F224683
S3150800A2F049463846A6EB0A063AF03EFE0134002ED9
S3150800A3003C4411DC3444484639F062FCC5E9007423
S3150800A310C5F80880BDE8F88FB8F1000FCADBA1EBD5
S3150800A3200904CAD14746CDE72046514632463AF097
S3150800A33015FE3444B9F1000FD3D0E4E7A1EB0904C4
S3150800A3404FF00108B9E7014839F05AFC9497040818
S3150800A3502DE9F04F85B0022580461E4600950E9BD6
S3150800A3609DF83C709DF84090044600F011F9324B78
S3150800A37048F81C3B314904F12C0A4046FEF7FAFE20
S3150800A3802E495046FEF7F6FE002598222C4904F180
S3150800A3903C003AF0E3FD11996661C4E9355550462B
S3150800A3A0C4F8DC5084F82850FEF72EFF61698B68E4
S3150800A3B00422E2716BB304F1D40B24264FF0250A6C
S3150800A3C00EE099428DF80F602FD00E70D4F8D83071
S3150800A3D00133C4F8D83061698B680135AB4217D9A7
S3150800A3E00B68D4F8D8105B5DBB42D4F8DC30E8D1F2
S3150800A3F099428DF80FA018D081F800A0D4F8D8306B
S3150800A40061690133C4F8D8308B680135AB42E7D8A7
S3150800A410DBB223764046FEF7F7FE204684F8E09046
S3150800A42084F8387005B0BDE8F08F0DF10F02584674
S3150800A430FFF72CFFCFE700BFB897040824F10408FC
S3150800A440009504082DE9F04F87B01E469DF8405048
S3150800A450119B0095814604469DF848809DF84CA0BE
S3150800A46000F096F8314B49F81C3B31494846FEF74F
S3150800A47081FE2F4904F12C00FEF77CFE2D49982217
S3150800A48004F13C003AF06AFDB268666100230421D3
S3150800A490C4E93533E171C4F8DC3084F82830002A81
S3150800A4A041D004F1D40019461D4624274FF0250B48
S3150800A4B010E099428DF817702ED00F70D4F8D83066
S3150800A4C00133C4F8D8306669B3680135AB4215D98B
S3150800A4D0D4E936133268525D4245EAD199428DF87D
S3150800A4E017B019D081F800B0D4F8D83066690133AE
S3150800A4F0C4F8D830B3680135AB42E9D8DBB2237665
S3150800A50031464846FEF780FE204684F8E0A084F8E7
S3150800A510388007B0BDE8F08F0DF117020390FFF7FA
S3150800A520B5FE0398CFE71346E9E700BFB8970408D6
S3150800A53024F104080095040810B5044600F016F83E
S3150800A54094F8E030012B0AD9022B08BF1A234FF0E2
S3150800A550000008BF84F8393084F8280010BD0023AD
S3150800A560002084F8393084F8280010BD08B58379AE
S3150800A570012B0AD00379032B07D08B4218BF4371EE
S3150800A580C36801710BB108469847002008BD00BF93
S3150800A59070B44D1E0E2D094E82604FF0020588BF1D
S3150800A5A00021C3604FF4A0629DF80C300660457127
S3150800A5B0C28070BC01740371704700BFE497040839
S3150800A5C0037901718B4218BF437170474379037150
S3150800A5D0704700BF00797047807970470023837100
S3150800A5E0704700BF81717047C079704770B5144CC9
S3150800A5F014490546204608F0C3F9204608F06AF9CA
S3150800A600204608F0A1F994F8293094F82A600E48F3
S3150800A610AA790E499B1B0370012A23880B8002D056
S3150800A6202B79032B05D1BDE870400548012108F0B8
S3150800A630F5BA20460321BDE8704008F0EFBA00BF1E
S3150800A6402CAE012010A704087A0F00207C0F0020EA
S3150800A65080687047013930B40B2914D8DFE801F057
S3150800A660222F3B06475461707E8C95154D4A4E4BFA
S3150800A67012781B884D4D4E4C4E4952005B080020FF
S3150800A6802A702380088030BC7047464A464B1278A9
S3150800A6901B88464C464847495B089200227003804F
S3150800A6A00B80F0E7404B3F4C40491B884048414AE5
S3150800A6B024780C705B08002103801180E3E7394C8D
S3150800A6C03A4A39483A493B4B2478008814700022A4
S3150800A6D008801A80D7E7344B324C1B883449354AF0
S3150800A6E03248247804705B080B801380CBE72D4B27
S3150800A6F02D4C2F491B782D482E4A24880C805B0048
S3150800A700002103701180BEE7264A274B12781B8862
S3150800A710264C274827495B085200227003800B8085
S3150800A720B1E7204B204A1B781288204D204C21493E
S3150800A73003EB4303520800202B7022800880A2E70F
S3150800A740184B194C1A491B7818481A4A24880C8041
S3150800A75003EB430300210370118094E7114A124B5F
S3150800A76012781B88114C124812495B0802EB420208
S3150800A770227003800B8086E70A4A0B4B12781B88E7
S3150800A7800A4D0B4C0B49920078E7064B064C0849D4
S3150800A7901B780648074A24880C809B000021037012
S3150800A7A0118070E77A0F00207C0F0020740F0020BC
S3150800A7B0780F0020760F0020C3690BB1427E1A700D
S3150800A7C00020704741610276704700BF90F9192052
S3150800A7D0436953F82200704790F82000704700BF7D
S3150800A7E02DE9F04F044681B00D46FFF7FFFE94F8B9
S3150800A7F02030012B48D023B1022B02D001B0BDE88E
S3150800A800F08F217CDFF88481564F2046FFF722FF20
S3150800A810002D40F08D80217C23790231C9B2204673
S3150800A820002B58D0FFF716FF237E002B69D0E2696C
S3150800A8306369127853F822204B494C483BF046F995
S3150800A8404A4B98F800203988494808F01FF8A2684A
S3150800A850484946483BF03AF9217C2046FFF7FAFE7C
S3150800A860454B424942481C8808F074F8398898F8DC
S3150800A87000203E4B0C44241A3D48A1B2398001B051
S3150800A880BDE8F04F08F002B8217CDFF80081354FAB
S3150800A8902046FFF7DFFE35BB257965BBDFF8F0A05C
S3150800A8A0DFF8CC902E46013505EB4501C9B22046A6
S3150800A8B0FFF7D0FE94F91930002B1A46B8BFDA1CF8
S3150800A8C0921006EB8206B3423AD0237EB34225DCC9
S3150800A8D0042DE7D1BBE7FFF7BDFE237E8BB194F9C4
S3150800A8E019206369A6E798F800203988234B204881
S3150800A8F007F0CCFFD0E7A26821491C483BF0E6F8F0
S3150800A900AAE7204D194B07CD186059609A60398817
S3150800A91098F80020164807F0B9FF98E7636998F891
S3150800A920002053F826303988484607F0AFFFCFE7AE
S3150800A93098F800203988114B0D4807F0A7FF6AE7F9
S3150800A940114B51464846B3F800B008F003F8ABEB94
S3150800A950000081B298F800205346484607F096FF53
S3150800A960B3E700BF760F002098F80408600F0020B0
S3150800A9702CAE01200C980408780F002008970408CC
S3150800A98010980408149804087C0F0020740F0020FF
S3150800A990089804080B780E2B10B504461DD00AD863
S3150800A9A00B2B0DD00C2B05D1437E013B5BB2002B44
S3150800A9B043761CDB10BD2B2BFCD14379037110BDEC
S3150800A9C003680E4A5B68934215D1C3690BB1427E90
S3150800A9D01A7040F20113A38010BD437E027E013334
S3150800A9E05BB29A424376E5DC0023437610BD037ECC
S3150800A9F0013B437610BD9847EBE700BFB9A70008AF
S3150800AA002DE9F04182B00226044600961D460B9BAE
S3150800AA109DF828809DF82070099EFFF7B9FD084922
S3150800AA2084F820800022032321606276E3710DB149
S3150800AA30656127762046E66102B0BDE8F08100BF71
S3150800AA40289804082DE9F04182B0044600930A9D2F
S3150800AA509DF830709DF82C80DDE90836FFF798FDE3
S3150800AA60084984F820700022032321606276E37186
S3150800AA7015B1656184F818802046E66102B0BDE824
S3150800AA80F08100BF2898040810B50446FFF76EFD4C
S3150800AA9094F82030022B01D0002010BD637E217E61
S3150800AAA001335AB291426276DBB222680849DCBFAA
S3150800AAB00023637652688A4207D1E26902B11370AD
S3150800AAC040F20113A380002010BD20469047F7E707
S3150800AAD0B9A70008704700BF90F82600704700BF66
S3150800AAE02DE9F04104460D46FFF780FD217C224FF3
S3150800AAF0224E0139C9B22046FFF7ACFD3DBBA2681C
S3150800AB001F4920483AF0E2FF1F4B1E491F481D887F
S3150800AB1007F020FF31881B4B3A780D442D1AA9B24D
S3150800AB201A48318007F0B2FE2379022B16D0012B82
S3150800AB301AD0217C01312046C9B2FFF78BFD3A783D
S3150800AB403188104B1148BDE8F04107F09FBE3A78AE
S3150800AB5031880F4B0D4807F099FED0E762690D4919
S3150800AB6008483AF0B3FFE4E7A3690B49054804F13E
S3150800AB701C023AF0ABFFDCE7740F0020760F0020CA
S3150800AB800C970408600F0020780F00202CAE0120D7
S3150800AB900897040898F804084C9804081C303BF0F9
S3150800ABA005B800BF70B582B00226044600961D4659
S3150800ABB0DDE90663FFF7ECFC22460A4B42F81C3B2C
S3150800ABC00023E3615360138184F826301DB1D5E96B
S3150800ABD00032C4E9053202232046A662E37102B0B8
S3150800ABE070BD00BF5C980408704700BF416170479C
S3150800ABF010B50446FFF7BAFCA06A10BD2DE9F84F58
S3150800AC0005464FF0000805F8048BDFF840909DF8DC
S3150800AC1028A004460F462846494693461E46FEF790
S3150800AC20A9FA494604F11000FEF7A4FA2846A4F842
S3150800AC30228084F824805946FEF72EFB277784F86D
S3150800AC401DA0A6772046BDE8F88F00BF24F10408AA
S3150800AC5010B504461030FEF7CFFA201DFEF7CCFAE1
S3150800AC60204610BD807F70471030FEF7CDBA00BF72
S3150800AC700430FEF7C9BA00BF017070470078704704
S3150800AC80407F7047037F0C2B15D8DFE803F01521AA
S3150800AC902B34414C5664707B8A8F0700C38C90F81E
S3150800ACA025205B08002163F30F0163F31F4193001E
S3150800ACB0016280F824307047C38C00215B080A467D
S3150800ACC063F30F0263F31F4280F824100262704791
S3150800ACD0C38C90F8252080F824205B080022038482
S3150800ACE04284704790F82530C28C80F824300023BF
S3150800ACF0028443847047C38C90F8252080F824206A
S3150800AD005B08002263F30F0263F31F420262704777
S3150800AD1090F82520C38C52005B08002180F8242077
S3150800AD2003844184704790F82530C28C02845B0006
S3150800AD30002280F8243042847047C38C90F825207E
S3150800AD405B08002163F30F0163F31F41530001629F
S3150800AD5080F82430704790F82530C28C03EB430303
S3150800AD605208002180F8243002844184704790F804
S3150800AD702530C28C028403EB4303002280F824307A
S3150800AD8042847047C28C90F825305208002162F33D
S3150800AD900F0162F31F4103EB4303016280F824307D
S3150800ADA0704790F82520C38C9200B5E790F82530B7
S3150800ADB0C28C02849B00002280F8243042847047AB
S3150800ADC00378012B00D1704730B5224D22498FB048
S3150800ADD00446284607F0D4FD284607F07BFD28469A
S3150800ADE007F0B2FD95F82A2095F829302988E184DC
S3150800ADF09B1A84F825300321284607F00FFF2046C2
S3150800AE00FFF740FF23696268144901A83AF05EFE1D
S3150800AE10237F28469BB101A9258C07F09BFD618CF1
S3150800AE20281A00EBD07001EB600189B2618494F8AE
S3150800AE302420084801AB07F029FD0FB030BD01A951
S3150800AE40258C07F087FD618C0D442D1AA9B2618403
S3150800AE50EDE700BF2CAE012010A70408F8F9040896
S3150800AE60704700BF80697047002070472DE9F041A0
S3150800AE7006460C46FFF7BAFB317CDFF85880114FBF
S3150800AE803046FFF7E7FBACB90F4BB1680F481C8893
S3150800AE9007F060FD3988B36898F80020241A04EB97
S3150800AEA0D47401EB640189B239800848BDE8F041E1
S3150800AEB007F0ECBC98F800203988054B034807F0E2
S3150800AEC0E5FCE1E7760F0020780F00202CAE012084
S3150800AED008970408740F002070B582B002261D4634
S3150800AEE00096069B0446FFF753FB044A6561002358
S3150800AEF020462260A361E37102B070BD88980408F9
S3150800AF00704700BF10B50446FFF730FB606910BDF7
S3150800AF1070B49DF814504161836106999DF81C3000
S3150800AF2042620122049E0572C1609DF80C509DF88C
S3150800AF30201002744374B5FBF1F200230132466017
S3150800AF400577C0E90D3370BC827780F8201003704E
S3150800AF50C377C363704700BF704700BF416170473E
S3150800AF600378042B70B5044660D0052B04D0032B58
S3150800AF700BD00023237470BDC16A0B78052BC368F8
S3150800AF8000F0BC800BB198472070A2690123237496
S3150800AF90002A61D0616A0B780B3B212BE9D801A006
S3150800AFA050F823F01FB200083BB1000871B1000841
S3150800AFB0E7B10008A5B1000873AF000873AF000831
S3150800AFC073AF000873AF000873AF000873AF0008CB
S3150800AFD073AF000873AF000873AF000873AF0008BB
S3150800AFE073AF000873AF000873AF000873AF0008AB
S3150800AFF073AF000873AF000873AF000873AF00089B
S3150800B00073AF000873AF000873AF000873AF00088A
S3150800B01073AF000873AF000873AF000873AF00087A
S3150800B02073AF0008A9B2000853B00008836990F905
S3150800B0301D20416A53F822000368DB689847636A53
S3150800B0401B782B2B00F047810B2B1FD00123237471
S3150800B05070BDE36A5BB170BD636A1B780B2B00F0A9
S3150800B06081812B2B85D1E36A002B40F0BC81D4E982
S3150800B0700D12E06B00F03CFCE36800222270002B06
S3150800B0803FF479AF20469847207070BD94F91D208B
S3150800B090A36953F82200FFF79DFA0028D6D0E36883
S3150800B0A0002B00F0B481A36994F91D2053F82200FF
S3150800B0B0036801211B689847E36813B1204698473F
S3150800B0C0207094F91D20A36953F82200FFF78CFA23
S3150800B0D0032820D02378032BB8D0052B7FF455AF4F
S3150800B0E0A56AE06B00232B7000F056FCE36BEB635C
S3150800B0F0E862A16AE06B00F023FC46E702220270D0
S3150800B10013B19847E16A2070E06B00F019FCE06B18
S3150800B11000F026FC9AE794F82050E27F237F15FB7F
S3150800B12002F59D42D6DAA36953F82500FFF756FAC9
S3150800B130237F0135AB42F6DCCCE794F91D00431EAC
S3150800B1405BB2002B6377C0F2408194F8201001337C
S3150800B150B3FBF1F201FB1233002B7FF40CAFE37F54
S3150800B160002B3FF408AF042900F0B280607770BD69
S3150800B17094F82020042A40F2ED8094F91D10042941
S3150800B18000F02E81E37F002B00F01181891A49B265
S3150800B190013BDBB20029E377B6BF12FB03F3617705
S3150800B1A0637770BD94F82000042840F2BA8094F9B9
S3150800B1B01D30022B40F32581227F01335BB29A4270
S3150800B1C0637740F3A78093FBF0F200FB1233002B62
S3150800B1D07FF4D1AEA37FE27F013B9A42BFF6CBAEA6
S3150800B1E00132E27770BD94F91D00227F431C5BB2E1
S3150800B1F09A42637740F38E8094F8201093FBF1F21D
S3150800B20001FB1233002B7FF4B6AEA37FE27F013B2E
S3150800B2109A42BFF6B0AE0429E2D06077A7E7237852
S3150800B220022B00F0AB8094F91D3052F82300FFF78B
S3150800B230D3F994F91D20A369054653F82200FFF7B0
S3150800B240C9F9012D3FF497AE03283FF494AE94F95B
S3150800B2501D20A36953F82200FFF7C6F9A36994F9DC
S3150800B2601D20064653F82200036800211B689847EC
S3150800B2700546002800F00A81E36A1B78052B00D0F2
S3150800B28000232370002E40F0F2800023E06BA562B5
S3150800B2902B7000F081FBE36BEB63E862A16AE06B5D
S3150800B2A0BDE8704000F04CBBE36A002B3FF4DFAE0C
S3150800B2B0206BFFF78BF900232370E16A0B78052BC7
S3150800B2C001D100230B70E06BBDE8704000F038BB7D
S3150800B2D0013BE37770BD94F91D20A36953F822005A
S3150800B2E0FFF778F900283FF4B1AEE3680BB12046C2
S3150800B2F09847237F03222270002B3FF4A7AE002530
S3150800B300A36953F82500FFF769F9237F0135AB4296
S3150800B310F6DC9BE6637C013AD3B1012362770B70B6
S3150800B32070BDA37FE27F013B9A42BFF624AE042894
S3150800B3303FF421AE94F91D30217F03445BB20132FC
S3150800B340D2B29942E27763773FF715AE10FB02F265
S3150800B350627770BDE37F53B3042A3FF40CAE94F9C9
S3150800B3601D1013E7E3680422227013B1204698479C
S3150800B3702070A56A002D60D102232370E3680BB103
S3150800B3802046984700230121206B2370FFF718F900
S3150800B390E16A31B10B78052B95D1A36A002B00F031
S3150800B3A09180E06B0021BDE8704000F0C9BAE56AFB
S3150800B3B0002D51D0206BFFF709F9E16A00232370AD
S3150800B3C00A78052A08BF0B707DE7637C4BB100231A
S3150800B3D06377D4E90D12E06BBDE8704000F088BAD7
S3150800B3E00323637770BDE368227013B1204698473C
S3150800B3F02070206BFFF7EAF8E16AE06B00F0A0FA2C
S3150800B4005BE7A17FE27F01398A4295DB70BDE27F67
S3150800B41094F82050237F15FB02F59D424FF0030256
S3150800B4202270BFF613AEA36953F82500FFF7CEF8CE
S3150800B430237F0135AB42F6DC08E600232B70E06B70
S3150800B44000F0AAFAE36BEB63E862A16AE06B00F02E
S3150800B45077FA0123237470BDD4E90D12E06B00F06E
S3150800B46047FAE3682570002B7FF40CAE70BD012EF9
S3150800B47018D0022E16D0032E2CD0042E7FF47BADC6
S3150800B4802378032B7FF477AD267070BDAEB9E16AD9
S3150800B490E06B0B78052B18BF33462370BDE8704068
S3150800B4A000F04EBA0023A5622B7094F91D20A369FB
S3150800B4B0E06B53F822302B63EBE6012E3CD0022ECC
S3150800B4C0D9D170BDE06B00F03BFAE06BBDE8704087
S3150800B4D000F046BA2378032B7FF44DADA36994F99F
S3150800B4E01D2053F8220003681B6A984702283FF478
S3150800B4F042ADE36813B1204698472070237894F844
S3150800B5002050E27F042B1CBF04232370237F15FBE6
S3150800B51002F59D42BFF62FAD94F91D30AB424FF0B0
S3150800B5200101A3690DD053F82500FFF75BF8237FC7
S3150800B5300135AB42F0DC70BDE368002B7FF4A2ADA9
S3150800B54070BD53F825000021FFF73AF8237F01352F
S3150800B5509D42E1DB70BD00BF416370478163704760
S3150800B560C1637047F0B56F498BB007466E4807F060
S3150800B57007FA6D4807F0E8F96B48032107F04EFB18
S3150800B5806A4B69480522D72107F080F9684B664857
S3150800B5900522F92107F07AF96649634807F0F0F9B8
S3150800B5A0614807F097F9604807F0CEF95E4803212D
S3150800B5B007F034FB796901A8FDF7DCFD5E4904A8AC
S3150800B5C0FDF7D8FD5D4901A8FDF7B2FE002800F099
S3150800B5D092800823002207A801A9FDF7DFFE07A924
S3150800B5E004A8FDF737FE07A8FDF706FE0022114658
S3150800B5F0049B4D4807F04AF904994B4807F0AAF905
S3150800B6000C230822064601A907A8FDF7C7FE07A9C5
S3150800B61004A8FDF71FFE07A8FDF7EEFDFB7FF6B2AF
S3150800B620002B76D04048012107F0F8FA049B3E48E3
S3150800B6300022314607F02AF904993B4807F08AF9AF
S3150800B64003213518384807F0E9FAFB7FEDB2002BDD
S3150800B65064D10F230D2201A907A8FDF79FFE07A9AC
S3150800B66004A8FDF7F7FD07A8FDF7C6FD049B2E48BD
S3150800B6700022294607F00AF904992B4807F06AF9C7
S3150800B6800F2213232C1801A907A8FDF787FE07A97F
S3150800B69004A8FDF7DFFD07A8FDF7AEFDFB7F2248EE
S3150800B6A0012B0CBF03210121E4B207F0B7FA049B72
S3150800B6B01D480022214607F0E9F804991A4807F0C0
S3150800B6C049F903210444184807F0A8FA039B1322F2
S3150800B6D001A907A8FDF762FE07A904A8FDF7BAFDA8
S3150800B6E0E4B207A8FDF788FD049B0F48214600220F
S3150800B6F007F0CCF805E002467B690B48114607F0CF
S3150800B700C5F804A8FDF778FD01A8FDF775FD0BB08F
S3150800B710F0BD0548032107F081FA87E70E230C22BE
S3150800B72099E700BF78AF04082CAE0120F4E20408BC
S3150800B730AC98040810A7040824F10408B098040873
S3150800B7400378052B70B5044632D1524A1378013373
S3150800B750DBB2072B2AD9C3680025012115700174AD
S3150800B7601BB39847E368207005461BB120469847E7
S3150800B77005462070002D7FD0042D16D194F8205050
S3150800B780E27F237F15FB02F59D420EDA94F91D3000
S3150800B790AB424FF00101A36964D053F82500FEF7C8
S3150800B7A021FF237F0135AB42F0DC70BD137070BDFD
S3150800B7B0FFF7D8FE94F82030E57F267F15FB03F5C2
S3150800B7C02B449E42A8BF1E46B5420FDA94F91D3097
S3150800B7D0AB42A36953F8250003684FF000019B6844
S3150800B7E005F1010539D09847AE42EFD1237A0025F5
S3150800B7F023B91DE0237A0135AB4219DD636853F896
S3150800B8002500FFF72FFA237883424FEA8506F1D100
S3150800B810636853F82500FFF733FAE37F8342E9D1DB
S3150800B82063689859FFF7CCFA237A0135AB42E5DC11
S3150800B8302278002AB9D117490B780133DBB2072BD6
S3150800B8400B70B2D9E5680123237023740A70002DA2
S3150800B850ABD02046A847207070BD01219847B54255
S3150800B860B4D1C3E753F825000021FEF7A9FE237FCC
S3150800B87001359D428ADB70BD0121206BFEF7A0FED3
S3150800B880E16A21B1E06BBDE8704000F059B829467D
S3150800B890F8E700BF7E0F0020007870470023037486
S3150800B8A0704700BF007C704790F82030B2FBF3F376
S3150800B8B00133027781618377704700BF90F91D20B5
S3150800B8C0836953F822007047006B7047816270479E
S3150800B8D0806A003818BF0120704700BF0022012384
S3150800B8E002700374704700BF4160704781607047FB
S3150800B8F0F0B50568104F2E684FF0000C0123BE42C4
S3150800B90083B00446C0F80CC0037407D16B68616045
S3150800B9100A498B420AD1A26003B0F0BD0192B04732
S3150800B920256806496B68019A8B42F4D01146204671
S3150800B93003B0BDE8F0401847E9B80008EDB80008BC
S3150800B94009B1C160704701230374C160704700BF25
S3150800B950C36813B11846FFF7F3BE4368184700BF1C
S3150800B960C36813B11846FFF7FBBA8368184700BFC8
S3150800B97010B50446C06818B1FFF794FF207410BDCF
S3150800B980207C10BD10B50446C06808B1FFF786FFD5
S3150800B9900023237410BD00BFC0687047436810B504
S3150800B9A0044603B1984723682046DB69BDE8104082
S3150800B9B0184700BF704700BF10B4012480F8C9407B
S3150800B9C080F8C4105DF8044B80F8C52080F8C630AE
S3150800B9D0704700BF02EBC20202EB8101084490F8EF
S3150800B9E0A43090F8A30003F00F0340EA0320704741
S3150800B9F002EBC20202EB8101084490F8A53090F8E8
S3150800BA00A4001B0143EA1010704700BF02EBC202F4
S3150800BA1002EB8101084490F8A20000F07F0070470D
S3150800BA2002EBC20202EB8101084490F8A20080F002
S3150800BA308000C009704700BF90F89D0000F00F0015
S3150800BA40704700BF00220123A0F8C22080F8C93041
S3150800BA50704700BF20290CBF4FF47F42FF22012305
S3150800BA60A0F8C22080F8C930704700BF012380F8CB
S3150800BA70C21080F8C32080F8C9307047012380F8C7
S3150800BA80C71080F8C82080F8C9307047407E7047D4
S3150800BA90C3683BB1002001210622187283F84810BA
S3150800BAA083F88120704700BF783003F0E7B900BFFC
S3150800BAB0043002F047BB00BFF0B54F2397B00C46E1
S3150800BAC005461A4602A8002139F070FA0022E271EA
S3150800BAD0EA7DA97D0091019267782078A178E678B9
S3150800BAE094F804E094F805C08DF80F708DF81000EE
S3150800BAF0A779A8688DF811108DF81260A9898DF8B4
S3150800BB0013E04F2302AA41F252168025FF248DF82E
S3150800BB1014C08DF81570ADF808608DF80A508DF8C8
S3150800BB200C4002F02BF817B0F0BD00BFF0B54F235C
S3150800BB3097B00C4605461A4602A8002139F036FA8F
S3150800BB400022E27115F8612C15F8621C0091019229
S3150800BB5067782078A178E67894F804E094F805C028
S3150800BB608DF80F708DF81000A77955F8700C8DF8C0
S3150800BB7011108DF8126035F86C1C8DF813E04F2300
S3150800BB8002AA41F252168025FF248DF814C08DF8BA
S3150800BB901570ADF808608DF80A508DF80C4001F064
S3150800BBA0EDFF17B0F0BD00BF30B5044685B078305C
S3150800BBB003F064F9E27DA37DCDE9003240F2432526
S3150800BBC00223A189A068ADF80C5003AA01F0D6FF9C
S3150800BBD063680BB105B030BDFF210122A4F8C0305F
S3150800BBE084F8C21084F8C52005B030BD783003F05B
S3150800BBF0D5B800BF7C3003F0CDB800BF7C3003F069
S3150800BC0095B800BF7C3002F0F7BE00BF7C3002F06A
S3150800BC10B3BF00BF08B5B0F99430012900EE903AD9
S3150800BC200CBFB0F99630B0F9923000EE103AF8EE43
S3150800BC30E00AB8EEC00A38F0C5F89FED047ADFEDE1
S3150800BC40047A30EE070A20EE270A08BDDB0F4940C2
S3150800BC50E12E654210B50D4B82B00446002240F82D
S3150800BC60043B0B4B02F0B4FA0A4BE36704F17C0081
S3150800BC70019003F003F9084B636030330198E367DA
S3150800BC8003F0FCF8204602B010BD00BF3099040846
S3150800BC90D8980408E8980408F498040810B401240D
S3150800BCA080F8C64080F8C3105DF8044B80F8C420BD
S3150800BCB080F8C530704700BF00EB8101D1F8B000AD
S3150800BCC0C0F30B20704700BF00EB8101B1F8B2004A
S3150800BCD0C0F30B10704700BF00EB810191F8B0006C
S3150800BCE000F07F00704700BF00EB810191F8B000BB
S3150800BCF080F08000C00970470F207047002201239A
S3150800BD00A0F8BE2080F8C630704700BF20290CBFB7
S3150800BD104FF47F42FF220123A0F8BE2080F8C630E8
S3150800BD20704700BF012380F8BE1080F8BF2080F856
S3150800BD30C6307047704700BF407E7047C3683BB146
S3150800BD40002001210622187283F8481083F8812002
S3150800BD50704700BF783003F03BBB00BF043002F0E9
S3150800BD60F1B900BFF0B5064697B00F464722002145
S3150800BD7004A839F01BF996F8C6305A1CD2B20F2A15
S3150800BD804FEA03138DF80A3043F2A2110ABF0023C3
S3150800BD9086F8C62086F8C630ADF8081010213A781D
S3150800BDA0BB787C788DF80B1006F184000DF116012E
S3150800BDB04FF2FF758DF80F208DF814308DF80E4070
S3150800BDC0ADF80C5003F02AFB0DF1210106F17C00B9
S3150800BDD003F024FBFB787A68CDF83720002B14BFD4
S3150800BDE001220222032317498DF835208DF83230B7
S3150800BDF002AC4FF0FF320DF1530014F8013BD5B2F7
S3150800BE006B40844251F8233083EA1222F5D100238D
S3150800BE103B72317ED343727E01920091190A1D0C42
S3150800BE201C0E8DF853308DF85410B068B1898DF812
S3150800BE30555002AA4F238DF8564001F09FFE17B0C1
S3150800BE40F0BD00BFC0990408F0B5064697B00F4686
S3150800BE504722002104A839F0A9F896F84E305A1C52
S3150800BE60D2B20F2A4FEA03138DF80A3043F2A21111
S3150800BE700ABF002386F84E2086F84E30ADF8081023
S3150800BE8010213A78BB787C788DF80B1006F10C00F7
S3150800BE900DF116014FF2FF758DF80F208DF814304D
S3150800BEA08DF80E40ADF80C5003F0B8FA0DF12101EB
S3150800BEB0301D03F0B3FAFB787A68CDF83720002BEB
S3150800BEC014BF01220222032318498DF835208DF864
S3150800BED0323002AC4FF0FF320DF1530014F8013B3B
S3150800BEE0D5B26B40844251F8233083EA1222F5D149
S3150800BEF000233B7216F8601CD34316F85F2C019298
S3150800BF000091190A1D0C1C0E8DF853308DF854102B
S3150800BF1056F8700C36F86C1C8DF8555002AA4F234B
S3150800BF208DF8564001F02AFE17B0F0BDC0990408F6
S3150800BF3030B5044685B0783003F04AFAE27DA37D31
S3150800BF40CDE9003240F643150223A189A068ADF871
S3150800BF500C5003AA01F012FE63680BB105B030BDA0
S3150800BF60FF210122A4F8C03084F8BF1084F8C2204B
S3150800BF7005B030BD783003F0AFB900BF7C3003F0B0
S3150800BF80A7B900BF7C3003F06FB900BF7C3002F060
S3150800BF90B1BF00BF7C3003F07BB800BF012908B5EC
S3150800BFA017D0B0F9A730B0F9A5205B4200EE102AE9
S3150800BFB000EE903AF8EEE00AB8EEC00A37F002FF53
S3150800BFC09FED097ADFED097A30EE070A20EE270A97
S3150800BFD008BDB0F9A720B0F9A93052425B4200EE7D
S3150800BFE0902A00EE103AE5E7DB0F4940E12E65425C
S3150800BFF030B5144B044683B0002240F8043B124B7C
S3150800C00002F0E6F800251149E16704F17C00C4E96D
S3150800C0102055C4E9225584F8875084F88F50A4F82F
S3150800C020C850019003F0D4F9094B019884F8CA5016
S3150800C03003F130026360E26703F0CAF9204603B0F1
S3150800C04030BD00BFC89D0408D89804088099040824
S3150800C0508C9904080E4B1A7810B44AB90D4B186817
S3150800C06003681C681146A446FF235DF8044B604725
S3150800C070012A02D05DF8044B7047074B186802681E
S3150800C08014680023A44619465DF8044BFF2260474E
S3150800C090840F0020880F00208C0F0020124B10B54B
S3150800C0A0187020B1012810D00024204610BDCC20DD
S3150800C0B037F090FD0D4B19680446FFF7CBFD0C4A87
S3150800C0C00C4B14602046A36010BDCC2037F082FDCF
S3150800C0D0064B19680446FFF78BFF074A054B1460A1
S3150800C0E02046A36010BD00BF840F0020800F0020EB
S3150800C0F0880F002055C000088C0F002010B4044C8F
S3150800C100044B216000225DF8044B1A70704700BF8B
S3150800C110800F0020840F0020704700BF0020704762
S3150800C120704700BF002070470120704790F8500004
S3150800C130704700BF90F87A00704700BFA1F1E00091
S3150800C140B0FA80F0400970472DE9F04385B00446FF
S3150800C150ADF80A10039200F12205042700260029EB
S3150800C1604AD094F83030042BFDD8DFE803F0030EEC
S3150800C1707A7348000223D4F80910237240F2022287
S3150800C18001232161A28284F830300DF10A0203A945
S3150800C19004F1100005F000FF70B3D4F809201378F5
S3150800C1A084F83130527884F83220C4F80950294688
S3150800C1B0042AA3F10203DBB208BF84F83360042A19
S3150800C1C0237263752375216184F830701BD0052AA4
S3150800C1D05CD0022A4AD0237F002B78D0012BE38B30
S3150800C1E07CD04BB904F12008BDF80A10C4F80980C0
S3150800C1F084F830600029B4D105B0BDE8F08394F81E
S3150800C2003220042AE3D10DF10A0203A904F1100031
S3150800C21005F0C2FE0028EFD094F82530FF2BE1D1B7
S3150800C22094F82630012BDDD194F83830002B69D0EC
S3150800C23094F82730002BD5D094F8222084F835308E
S3150800C240012194F8233084F8331084F8362084F8D2
S3150800C2503730C7E7D4F8091094F8322094F831300B
S3150800C260A6E794F8322094F831309EE70DF10A02D9
S3150800C27003A904F1100005F08FFE0028BCD094F83D
S3150800C280253084F8343004F12008ADE70DF10A02B0
S3150800C29003A904F1100005F07FFE0028ACD094F83D
S3150800C2A03330002B9ED0606800289BD094F8352048
S3150800C2B0036804F12008CDE90028D3F8009094F823
S3150800C2C0362094F8373094F83410C8478CE794F839
S3150800C2D03130023B9BB20122E383227783B1BDF85A
S3150800C2E00A20039903E0E383013182B22BB1013BB3
S3150800C2F09BB2501E002AF6D17EE7ADF80A200391BC
S3150800C30026776FE794F82730012B7FF46BAF93E716
S3150800C31040F65C23994222D040F20D53994215D03B
S3150800C32043690BB9008B00B340F24C53994214D1C0
S3150800C330B2F51A7F17D040F22F439A4213D040F233
S3150800C340D530101AB0FA80F04009704740F25A63A7
S3150800C3509A4208D04369002BE4D00020704742F285
S3150800C360E8139A42F6D1012070477047019A2BBB11
S3150800C37080F85D10D37803F00303032B1FD0022B3C
S3150800C3801CD192F902309178002BACBF032302230B
S3150800C39003EB4303034401F00F0183F8511091881E
S3150800C3A083F85210937990F878209A4238BF80F82B
S3150800C3B0783090F85E30013380F85E30704792F935
S3150800C3C00230002BFADA90F85610012363F387013E
S3150800C3D080F856109178DBE72DE9F04385B00446DE
S3150800C3E0ADF80A10039200F1220504270026002959
S3150800C3F04AD094F83030042BFDD8DFE803F0030E5A
S3150800C4007A7348000223D4F80910237240F20222F4
S3150800C41001232161A28284F830300DF10A0203A9B2
S3150800C42004F1100005F0B8FD70B3D4F809201378AC
S3150800C43084F83130527884F83220C4F809502946F5
S3150800C440042AA3F10203DBB208BF84F83360042A86
S3150800C450237263752375216184F830701BD0052A11
S3150800C4605CD0022A4AD0237F002B78D0012BE38B9D
S3150800C4707CD04BB904F12008BDF80A10C4F809802D
S3150800C48084F830600029B4D105B0BDE8F08394F88B
S3150800C4903220042AE3D10DF10A0203A904F110009F
S3150800C4A005F07AFD0028EFD094F82530E02BE1D18D
S3150800C4B094F82630012BDDD194F83830002B69D05A
S3150800C4C094F82730002BD5D094F8222084F83530FC
S3150800C4D0012194F8233084F8331084F8362084F840
S3150800C4E03730C7E7D4F8091094F8322094F8313079
S3150800C4F0A6E794F8322094F831309EE70DF10A0247
S3150800C50003A904F1100005F047FD0028BCD094F8F3
S3150800C510253084F8343004F12008ADE70DF10A021D
S3150800C52003A904F1100005F037FD0028ACD094F8F3
S3150800C5303330002B9ED0606800289BD094F83520B5
S3150800C540036804F12008CDE90028D3F8009094F890
S3150800C550362094F8373094F83410C8478CE794F8A6
S3150800C5603130023B9BB20122E383227783B1BDF8C7
S3150800C5700A20039903E0E383013182B22BB1013B20
S3150800C5809BB2501E002AF6D17EE7ADF80A20039129
S3150800C59026776FE794F82730012B7FF46BAF93E784
S3150800C5A0019A2BBB80F85910D37803F00303032BA9
S3150800C5B01FD0022B1CD192F902309178002BACBF08
S3150800C5C00323022303EB4303034401F00F0183F81B
S3150800C5D04D10918883F84E10937990F874209A42FA
S3150800C5E038BF80F8743090F85A30013380F85A30E2
S3150800C5F0704792F90230002BFADA90F852100123AC
S3150800C60063F3870180F852109178DBE770B54FF431
S3150800C610802104464FF48062C4E91512002543F6CA
S3150800C6200840042384F85150A4F8520084F85C307A
S3150800C63004F1640504F1740655F8043B184613B171
S3150800C6401B689B689847AE42F6D10025E06C84F8D3
S3150800C65050500123A4F8785084F85E30036884F8B3
S3150800C66041509B6884F84250A4F8465084F87D509F
S3150800C670256684F87A5029469847284670BD00BF33
S3150800C6802DE9F04F044690464FF480204FF480621F
S3150800C690C4E9150243F60845002699460423A4F87A
S3150800C6A0525089B00F4684F8516084F85C3004F122
S3150800C6B0640504F1740A55F8046B304616B13368FC
S3150800C6C09B6898475545F6D10025D4F84CA084F8C0
S3150800C6D050500123A4F8785084F85E30DAF8003018
S3150800C6E084F841501B6884F84250A4F8465084F8F0
S3150800C6F07D50256684F87A5029465046984706465E
S3150800C700002849D0D0F800B0BBF1000F3FD004F1A3
S3150800C710510303AA036080F80690009229462A4628
S3150800C720E06C122304F084FEC6F800B0054618BB78
S3150800C730DAF8002043465668394650462A46B04736
S3150800C74084F8500068B39DF81030092B2BD09DF85B
S3150800C75013009DF81D10BDF81420BDF8163084F896
S3150800C760520084F85410A4F87620A4F87430E02512
S3150800C770284609B0BDE8F08F23680D289B68204637
S3150800C78018BFE1259847284609B0BDE8F08FD72598
S3150800C790284609B0BDE8F08FD625284609B0BDE879
S3150800C7A0F08FD425E4E701462B462A46E06C04F0D0
S3150800C7B099FF236820469B689847D125D8E700BF8C
S3150800C7C02DE9F04F2DED028BD0F84C8090F854707F
S3150800C7D090F850104FF0000980F85490D8F80020CF
S3150800C7E09BB00446126840461E469047002800F053
S3150800C7F0918005464FF496702AF052FD494694F802
S3150800C8005030E06C4A4604F06DFF0146002840F0BF
S3150800C8108880D8F80030A87194F850101B684046F4
S3150800C8209847002876D0867194F85010E06C04F189
S3150800C8305103012208EE103A03F04AFA014600288D
S3150800C84071D1B4F8762040F24C539A4277D0002F33
S3150800C85000F0D68004F104094B460025DFF864820F
S3150800C860DFF864B209930DF12C0A13AE2946B946CE
S3150800C87029E00998DFF854C20C9094F85010E06C3F
S3150800C8808DF83420ADF840208DF84820ADF84A20C0
S3150800C890ADF85C208DF85E208DF86420CDF8356003
S3150800C8A00F961196CDF82CC004F062FE0135E9B258
S3150800C8B0002840F0CB8094F85E20032A00F2A4807A
S3150800C8C0894540F2C580606FCDF800A04FF0000C96
S3150800C8D040450B46624601D05845CAD1774F0B975B
S3150800C8E094F85010099FE06C0C978DF834C0ADF899
S3150800C8F040C08DF848C0ADF84AC0ADF85CC08DF8A8
S3150800C9005EC08DF864C0CDF835600F96119604F0B8
S3150800C9102FFECBE7D62108461BB0BDEC028BBDE83F
S3150800C920F08F85F80690236809919B6820469847FA
S3150800C930099908461BB0BDEC028BBDE8F08FB4F828
S3150800C9407430B3F51A7F08D040F22F42934204D0D0
S3150800C95040F2D53293427FF47AAF64202AF0A0FCE5
S3150800C96094F8501094F85120E06C012304F014FF59
S3150800C97001460028D7D163690BB9238B5BB3B4F89A
S3150800C9807430B3F51A7F6CD040F22F42934268D0C8
S3150800C9902346052053F8141F01909E88CDF82D10C4
S3150800C9A00B23CDE904330022079203920BAD032231
S3150800C9B00923069500930292414D8DF82C0094F8B0
S3150800C9C0512094F85010E06CADF831602123CDF871
S3150800C9D0335004F015F894F8512094F85010E06C90
S3150800C9E0002304F0D9FE002394F85010E06C1A4690
S3150800C9F004F078FE236820469B689847D1218AE789
S3150800CA0094F85E20032A23D994F85010E06C18EEA7
S3150800CA10103A03F05DF90146002884D194F85010C5
S3150800CA2094F85D3094F85120E06C04F0B5FE0146A8
S3150800CA3000287FF478AF4FF4C802012384F88100F8
S3150800CA402072C4F8822084F87A3064E701466AE7DF
S3150800CA50002394F85010E06C1A4604F043FED121E6
S3150800CA6061E70BAD08230320F521CDE90110CDE9D7
S3150800CA7005350022079203920922049300920120A9
S3150800CA80657E237EE27DA17DADF82C00607D8DF864
S3150800CA902E508DF82F30257D8DF830208DF83110E9
S3150800CAA08DF8320094F8512094F85010E06C8DF807
S3150800CAB03350212303F0A4FF8DE700BF7C9E0408B2
S3150800CAC010010212E8215C0A5A060D05889E040820
S3150800CAD070B54D4BC164044603F13402236000234C
S3150800CAE04A4D6260C4E91933C4E91B3301264FF481
S3150800CAF080204FF480610422C4E9145084F85E60F3
S3150800CB00A16584F85C2084F8413084F8433084F8C1
S3150800CB104630A4F848302366A4F8783084F87A308A
S3150800CB2004F1680504F1740655F8043B184613B178
S3150800CB301B689B689847B542F6D1E36C0022012131
S3150800CB4084F8412084F84220A4F8462084F87D2001
S3150800CB5084F850202266A4F8782084F87A2084F88D
S3150800CB605E106BB39A6F72B3DA6FAAB3D3F88020EC
S3150800CB70A2B3D3F884209AB3D3F8882092B3D3F813
S3150800CB808C202AB3D3F8902072B3D3F894206AB3D2
S3150800CB90D3F8982062B3D3F89C205AB3D3F8A020D0
S3150800CBA052B3D3F8A4204AB3D3F8A82042B3D3F893
S3150800CBB0AC203AB3D3F8B02022B1D3F8B4204AB1A6
S3150800CBC0204670BD0E221E32204643F8224070BD14
S3150800CBD00522F8E70F22F6E70A46F4E70222F2E70B
S3150800CBE00322F0E70422EEE70622ECE70722EAE74B
S3150800CBF00822E8E70922E6E70A22E4E70B22E2E749
S3150800CC000C22E0E70D22DEE7949E04080000083CAB
S3150800CC10F0B590F8783085B000F1C907CDE9007312
S3150800CC20054690F8572090F85010C06C40240DF136
S3150800CC300E03ADF80E4003F0C5FE68B105F16404B5
S3150800CC40743554F8043B184613B11B685B6898475B
S3150800CC50A542F6D105B0F0BDBDF80E3005F1640465
S3150800CC607435002BEDD0264656F8043B394618464F
S3150800CC7013B11B681B689847AE42F5D1E1E700BFC0
S3150800CC8070B513220C23064680F8892080F88A306E
S3150800CC9088B008460D46FBF7C5FA013086F88B00C2
S3150800CCA0002402E0EB5C82F88C302846FBF7BAFADF
S3150800CCB0E3B2984206EB030204F10104F2D83344C6
S3150800CCC0002483F88C402846FBF7ACFA0430B6F803
S3150800CCD08630079480B2CDE90400CDE90244CDE957
S3150800CCE0004406F1890223F00103A6F8863006926D
S3150800CCF096F8512096F85010F06C202303F080FE29
S3150800CD0008B070BDF0B590F8813089B00446132B91
S3150800CD1070D8DFE813F07900A400C400E9000F0119
S3150800CD201E01490157018301D3010202450214007D
S3150800CD3051026F00650274029502BE027100B0F8D6
S3150800CD408650290756D500F12206D94930460822C9
S3150800CD5038F034FF80B90127A4F8440084F87B0032
S3150800CD60D44984F842701622304638F027FF002846
S3150800CD7040F08C8384F8447094F8803033B9B4F862
S3150800CD807E2042F208539A4200F0AD8394F843306D
S3150800CD90002B40F01D8394F84830002B40F0188390
S3150800CDA0092140F20472208CE66984F88910A4F8F7
S3150800CDB08A2000230A2204F1890125F00305A4F834
S3150800CDC0900084F89230A4F88650C4F88C60CDE9B7
S3150800CDD00233CDE90033CDE90521079304922023D8
S3150800CDE094F8512094F85010E06C03F009FE0D23D6
S3150800CDF084F8813009B0F0BDB0F88630D907F9D586
S3150800CE00062384F88130F5E7B0F88230B0F884203C
S3150800CE1001339BB29A42A0F88230EBD20025032355
S3150800CE20A0F88650CDE90255CDE90055079580F85A
S3150800CE308930CDE9043300F189020C21A0F88A1063
S3150800CE40069290F8512090F85010C06C202303F0F9
S3150800CE50D7FD0123A4F8825084F88130CAE7B0F8D8
S3150800CE608230B0F8862001339BB2A0F88230D00712
S3150800CE7000F19082B4F884209342BBD902EB820376
S3150800CE805B009BB2B3F5FA6F88BF4FF4FA63A4F858
S3150800CE908430002384F88130A4F88230AAE7B0F8F9
S3150800CEA08630D907A6D5002223F0210303210925B8
S3150800CEB01020A4F8863084F88110CDE9041184F88E
S3150800CEC08950A4F88A00CDE90222CDE9002204F1AE
S3150800CED089030792069394F8512094F85010E06C51
S3150800CEE0202303F08DFD85E7B0F886309A0681D5B4
S3150800CEF023F04103A4F8863000220323102004F10E
S3150800CF0089010125A4F88A0084F88950CDE90531FC
S3150800CF10CDE90222CDE9002204930792202394F852
S3150800CF20512094F85010E06C03F06AFD042384F84D
S3150800CF3081305FE7B0F886305F067FF55BAFC16882
S3150800CF40002900F08982FFF79BFE052384F88130CB
S3150800CF5050E7B0F88630DE077FF54CAF90F84920E9
S3150800CF60002A3FF44DAF23F4007323F00103A4F81D
S3150800CF708630042200235048C4F8890004F1890148
S3150800CF80CDE90233CDE90033CDE9052107930492B3
S3150800CF90202394F8512094F85010E06C03F030FDEB
S3150800CFA0112384F8813025E790F84830002B40F0AB
S3150800CFB09E8190F84330002B40F099810A2384F82B
S3150800CFC0813017E7B0F886301A067FF513AF0025CB
S3150800CFD023F0010302200421032204F18906A4F8A0
S3150800CFE0863084F88900A4F88A10CDE90665CDE96B
S3150800CFF00255CDE90055CDE90422202394F85120A5
S3150800D00094F85010E06C03F0FBFC94F87C30002B8D
S3150800D01040F04982082384F88130EBE6B0F8863080
S3150800D020DF077FF5E7AE23F48173002123F00103C0
S3150800D030A0F88630057F407F84F87C1084F8981025
S3150800D040CDE900110522E37F84F88920A27F84F8C0
S3150800D0508C5084F88D0094F8205094F8210084F8B8
S3150800D0608E2084F88F304CF61842012340F6045679
S3150800D07084F8905084F89100A4F89220C4F894306B
S3150800D08094F85120A4F88A60CDE90211079104F1B9
S3150800D090890094F850100690E06C20231025CDE9FD
S3150800D0A0045503F0ADFC092384F88130A2E600BFDD
S3150800D0B0109E04081C9E040804100100B0F886306F
S3150800D0C0DE057FF597AE13F0020100F08781428BEB
S3150800D0D080F88C2023F00103A0F88630C2F30321E0
S3150800D0E00523002211264FF40175893084F88D1026
S3150800D0F084F88960A4F88A50CDE90530CDE9022282
S3150800D100CDE900220493079294F8512094F8501020
S3150800D110E06C202303F074FC50E790F84130002BB4
S3150800D1207FF468AE90F84330002B7FF463AE90F836
S3150800D1304630002B7FF45EAE90F84830002B7FF423
S3150800D14059AEC168B0F8862007930029CDE90233A5
S3150800D150CDE9003318BF03264FF0040308BF0226A3
S3150800D16022F011024FF4867004F189011A25A4F8F9
S3150800D1708620A4F88A0084F88C6084F88950CDE962
S3150800D1800531049394F8512094F85010E06C20234C
S3150800D19003F036FC01220B23227284F8813029E63B
S3150800D1A0B0F88630DD0600F1C68058077FF522AE56
S3150800D1B0102384F881301DE6B0F886309A077FF58B
S3150800D1C019AE90F87D3013B1012380F8463000235C
S3150800D1D00F2263726381A4F8863084F8812009E6F9
S3150800D1E0B0F8823001339BB2B3F57A7F7FF654AE3E
S3150800D1F000220A23A0F8822080F88130FAE5B0F8E8
S3150800D20086305B077FF5F6AD0025A0F886502946DF
S3150800D2104022893037F0CAFE2946402204F1C90067
S3150800D22037F0C4FE0A2384F84150A4F84250A4F803
S3150800D230465084F84850A4F87C5084F88130D9E5E3
S3150800D240B0F886309D057FF5D5AD90F87920002A8F
S3150800D2503FF4D6AD23F00103A4F886300422002358
S3150800D260AC48C4F8890004F18901CDE90233CDE957
S3150800D2700033CDE9052107930492202394F8512021
S3150800D28094F85010E06C03F0BBFB122384F881304D
S3150800D290B0E5B0F88630D8077FF5ACAD9E49C4F83E
S3150800D2A0891023F001034FF0FF32A4F88630C4F842
S3150800D2B08D2000230B22FF2004F189011F25A4F8E5
S3150800D2C0920084F89150CDE90233CDE90033CDE9D7
S3150800D2D0052107930492202394F8512094F85010BE
S3150800D2E0E06C03F08DFB132384F8813082E5B4F8F3
S3150800D2F086208A4BC4F889300821002322F081024F
S3150800D30004F18900864DA4F88620C4F88D50CDE92D
S3150800D3100233CDE90033CDE90510079304912023A4
S3150800D32094F8512094F85010E06C03F069FB072339
S3150800D33084F881305EE5002223F00903A0F88630E0
S3150800D340C569008C2272A4F894201927CDE9022217
S3150800D350CDE90022079240F60426012104F189024C
S3150800D36084F88970A4F88A60C4F88C50A4F89000F0
S3150800D370A4F892100D230692CDE90433202394F8DD
S3150800D380512094F85010E06C03F03AFB0C2384F813
S3150800D39081302FE5002322F00102A4F88620A4F8A4
S3150800D3A0823084F88E305F480793CDE90233CDE9A1
S3150800D3B0003302250623082104F1890284F88150E6
S3150800D3C0C4F8890084F88D10CDE90532049382E506
S3150800D3D094F87C30002B7FF41DAEE1E423F48173CE
S3150800D3E023F00103A0F88630057F407F84F8981063
S3150800D3F0CDE9011100910522E37F84F88920A27FF7
S3150800D40084F88C5084F88D0094F8205094F8210004
S3150800D41084F88E2084F88F3040F604564CF618426D
S3150800D4200123A4F88A6084F8905084F89100A4F83F
S3150800D4309220C4F8943094F851200791039194F8F7
S3150800D4405010E06C102504F189062023CDE9055615
S3150800D450049503F0D5FACDE490F84920002A3FF464
S3150800D460CFAC23F4007323F00103A4F886302E48CA
S3150800D4700791042304F18902CDE90211CDE90011CF
S3150800D480C4F88900CDE90532049381E527491622B7
S3150800D490304638F093FB90BB40F2011384F87B705A
S3150800D4A0A4F8443068E4B4F88630E069218CA4F81E
S3150800D4B0945023F00903CDE90665CDE90255CDE977
S3150800D4C00055192640F604250122A4F8863084F86A
S3150800D4D089600D23A4F88A50C4F88C00A4F890102B
S3150800D4E0A4F8922048E712493046132238F066FB22
S3150800D4F000287FF44BAC012384F87D3046E40D49BF
S3150800D5001322304638F05AFB00287FF435AC84F8ED
S3150800D5107B7031E4560C0101010C08FF0104053348
S3150800D5208B9E300A240C030404100100349E040860
S3150800D530609E04084C9E040870B50D2190F843506F
S3150800D540C269038C80F8891041F2047188B00446D8
S3150800D550A0F88A10C0F88C20A0F8903085B390F80F
S3150800D5607B30062280F89220002B4AD0034653F8D7
S3150800D570142FC0F893209B88A0F897300022C4F88F
S3150800D5809920C4F89D20A4F8A120B4F8865094F8F0
S3150800D590512094F85010E06C25F00105A4F8865047
S3150800D5A000231A258934CDE90233CDE900330793E0
S3150800D5B0CDE905540495202303F022FA08B070BD7E
S3150800D5C006693046FAF72EFE84F8920002E0F35C0C
S3150800D5D082F893303046FAF725FEEBB2984204EB10
S3150800D5E0030205F10105F2D80F2BCED8C3F10F02BD
S3150800D5F003F19300D2B201322044002137F0D6FC61
S3150800D600C3E7034653F81C2FC0F893209B88A0F85D
S3150800D6109730B3E7F0B590F878308BB000F189050C
S3150800D620CDE90053044690F8542090F85010C06C89
S3150800D63040260DF12603ADF8266003F0C3F910F075
S3150800D640FB0F5ED194F88920531E322B59D8DFE898
S3150800D65013F05A007400B100CA00E800F600090188
S3150800D6605800580058005800580058002201580021
S3150800D67058005800580058005800580049015401ED
S3150800D68058005800580058005800580058005800CC
S3150800D69058005800580058005800580058005800BC
S3150800D6A058005800580058005800580058005800AC
S3150800D6B058005D0158003300B4F88630E069218CC3
S3150800D6C0069523F001032C2240F20465A4F886305F
S3150800D6D084F8892000230922A4F88A50C4F88C000B
S3150800D6E0A4F89010CDE90233CDE90033CDE9042240
S3150800D6F0079394F8512094F85010E06C202303F017
S3150800D7007FF90BB0F0BD94F88830042B40F21A81EB
S3150800D71094F8431021B994F84810002900F01281B2
S3150800D72000230A2184F8413084F8433084F84630CF
S3150800D73084F8483084F8811006E194F88B60002E4E
S3150800D740DFD094F84310F300DBB2002940F049819A
S3150800D75094F848E0084606E00131C8B20333864229
S3150800D760DBB240F23781E21892F88E5092F88D704B
S3150800D77092F88FC005F00F02BEF1000FECD0052A13
S3150800D780EAD117F0C80FE7D0062303FB004084F858
S3150800D7907E7084F87F5084F880C0D0F88C20B4F866
S3150800D7A08630E261B0F89020228443F08003A4F822
S3150800D7B08630A6E7B4F8863094F88B2043F4807157
S3150800D7C0A4F88610002A40F0C28094F88D2094F8B8
S3150800D7D08C10120202F4706243F481730A43A4F8AF
S3150800D7E0863062838DE7234694F8922053F88B1F80
S3150800D7F0E1619988218402F00F0194F8913094F838
S3150800D800930084F87F20052984F87E3084F8800008
S3150800D81000F0A180B4F8863043F01003A4F88630EF
S3150800D8206FE794F88B30002B7FF46BAFB4F8863033
S3150800D83023F0020343F00403A4F8863061E794F862
S3150800D8408B30002B40F08E8094F84330002B00F08C
S3150800D850B38094F84130002B40F0AE80012384F861
S3150800D86041304EE794F88B30002B7FF44AAF04F131
S3150800D870210304F13F0101E08B4205D093F87120A2
S3150800D88003F8012F002AF7D1B4F8863043F00803CD
S3150800D890A4F8863035E794F88E30002B7FF431AF44
S3150800D8A0B4F88630B4F88C2041F2010143F0010047
S3150800D8B08A42A4F8860000F0DB8041F204018A421D
S3150800D8C000F0DF8041F209018A427FF41AAF22464E
S3150800D8D043F0210352F88F1F616192882283A4F8CE
S3150800D8E086300EE794F843301BB92369002B00F005
S3150800D8F0A2802046FFF720FE03E7B4F88630E069E9
S3150800D900218C069523F001030C22DDE6B4F8863057
S3150800D910E669208C069523F0010340F604122B25B0
S3150800D920A4F8863003210023A4F88A2084F88950B5
S3150800D9300C22C4F88C60A4F89000A4F8921084F81D
S3150800D9409430CFE60133DAB284F88820D9E6062384
S3150800D95084F88130D5E613F0C80F1CBF012384F87C
S3150800D960473057E7638BB4F886200695C3F303213F
S3150800D97084F88C3084F88D10002322F005021320D9
S3150800D98006214FF44175A4F8862084F88E00A4F881
S3150800D9908A50CDE90233CDE90033CDE90411079366
S3150800D9A094F8512094F85010E06C202303F028F8DE
S3150800D9B0102384F88130A4E694F84830002B3FF40D
S3150800D9C0A0AE94F84630002B7FF49BAE012384F872
S3150800D9D0463096E684F87E7084F87F5084F880C0D6
S3150800D9E08FE60021084605E00131C8B203338642B6
S3150800D9F0DBB2EFD9E21892F88E5092F88FC092F8FF
S3150800DA008D7005F00F0EBCF1000F01D1052D0AD05F
S3150800DA1094F84820002AE7D0BEF1050FE4D117F0A4
S3150800DA20C80FE1D0B0E617F00C0F3ED194F84820A5
S3150800DA30002AD9D0F3E7B4F88620E069218C079349
S3150800DA40CDE90233CDE90033069522F001020E2610
S3150800DA5040F204650923A4F8862084F88960A4F8AE
S3150800DA608A50C4F88C00A4F89010CDE9043340E637
S3150800DA7094F88F2084F8402043F04103A4F88630B8
S3150800DA803FE69A050AD494F88F203AB994F8972075
S3150800DA9012F0080218BF012284F8792043F40073B3
S3150800DAA043F00103A4F886302BE601EB410104EBB1
S3150800DAB04103012284F87C2084F87E7084F87F5024
S3150800DAC084F880C0D3F88C10B4F88620E161B3F8E6
S3150800DAD09030238442F08003A4F8863011E600BF14
S3150800DAE090F87A300BB90020704710B5044629F033
S3150800DAF0D1FB236EC01A00280EDB29F0CBFB94F865
S3150800DB007830184420662046FFF784FD2046FFF744
S3150800DB10F9F82046FFF77CF8002010BD30B503461B
S3150800DB200C46B0F8865090F8512090F85010C06C0A
S3150800DB3083F88C40C4F3032483F88D404FF4417472
S3150800DB4089B0A3F88A40132483F88E4025F005058A
S3150800DB5003F18904A3F8865006940625002483F861
S3150800DB608950CDE90455CDE90244CDE9004407942E
S3150800DB70202302F045FF09B030BD00BFF0B503F120
S3150800DB800F0404F4FC7483B002AFADEB040D02ACD1
S3150800DB9003F1040E8DF80810C1F3032C4FEA2E2169
S3150800DBA04CF0200C05460026387EE170397F84F853
S3150800DBB001C0237184F802E06671A071E171E3B1D6
S3150800DBC09EB2731E9BB2114604F108005A1C37F028
S3150800DBD0C5F906F10803009495F85A2095F85010EF
S3150800DBE0E86C02F0B7FC10B90437BD46F0BD6420F6
S3150800DBF029F056FB0437BD46F0BD0823EBE700BF06
S3150800DC00F0B587B00446BDF8305084F80A210220E2
S3150800DC10042284F8090184F80B212812002284F8CA
S3150800DC200D5184F80C2184F80E01187884F80F0138
S3150800DC305B7884F81031C1F303250B460826D4F81F
S3150800DC400D11D4F809018DF808308DF80B2045F030
S3150800DC5020038DF80D208DF80F200DEB060200929B
S3150800DC608DF809300C27012504AB8DF80A708DF85C
S3150800DC700C608DF80E5094F85A2003C394F850108F
S3150800DC80E06C102302F066FC08B907B0F0BD64200A
S3150800DC9029F006FB07B0F0BD70B50446002503263B
S3150800DCA0082084F8096184F80C5184F80A2184F85C
S3150800DCB00B0188B01A7884F80D215A780C9B84F8E1
S3150800DCC00E211A7884F80F215B789DF8342084F8A1
S3150800DCD01031C1F303260B46A4F8125184F81451E7
S3150800DCE08DF80C3084F8112146F02003D4F80D1174
S3150800DCF0D4F80901D4F811218DF80F508DF80D309C
S3150800DD008DF811508DF813500C2301258DF810301D
S3150800DD108DF81250102605AB03AD8DF80E6007C3BB
S3150800DD200095142394F85A2094F85010E06C02F0E9
S3150800DD3011FC08B908B070BD642029F0B1FA08B022
S3150800DD4070BD00BF70B5044600250426082084F877
S3150800DD50096184F80B0184F80C5184F80A211A78B1
S3150800DD6084F80D2188B05B7884F80E31C1F3032658
S3150800DD700B461B48C4F81001FF2284F80F5184F89B
S3150800DD8014218DF80C3046F02003D4F80D11D4F880
S3150800DD900901D4F811218DF80F508DF80D308DF842
S3150800DDA011508DF813500C2301258DF810308DF87D
S3150800DDB01250102605AB03AD8DF80E6007C300950B
S3150800DDC094F85A2094F85010E06C142302F0C2FB21
S3150800DDD008B908B070BD642029F062FA08B070BDB1
S3150800DDE0000102FF70B50446002505260A2084F8BE
S3150800DDF0096184F80B0184F80C5184F80A211A7811
S3150800DE0084F80D2188B05B7884F80E31C1F30326B7
S3150800DE100B468DF8083046F020038DF809304FF090
S3150800DE2080704AF202021223C4F8100184F80F51D6
S3150800DE30A4F814218DF80A300E23D4F80D11D4F85D
S3150800DE400901D4F811218DF80C3001238DF80E3014
S3150800DE5004AB8DF80B508DF80D508DF80F5007C395
S3150800DE60022284F81621B4F8155194F85A2094F829
S3150800DE705010E06C1D8002AC1623009402F06AFB79
S3150800DE8008B908B070BD642029F00AFA08B070BD58
S3150800DE90F0B50446062584F80A210420002284F8F1
S3150800DEA0095184F80C2184F80B0187B0187884F896
S3150800DEB00D0158780C9B84F80E01187884F80F0128
S3150800DEC05B7884F81031C1F303250B460826D4F88D
S3150800DED00D11D4F809018DF808308DF80B2045F09E
S3150800DEE020038DF80D208DF80F200DEB0602009209
S3150800DEF08DF809300C27012504AB8DF80A708DF8CA
S3150800DF000C608DF80E5094F85A2003C394F85010FC
S3150800DF10E06C102302F01EFB08B907B0F0BD6420C0
S3150800DF2029F0BEF907B0F0BDF0B50446072584F818
S3150800DF300A210420002284F8095184F80C2184F867
S3150800DF400B0187B0187884F80D0158780C9B84F873
S3150800DF500E01187884F80F015B7884F81031C1F344
S3150800DF6003250B460826D4F80D11D4F809018DF8B7
S3150800DF7008308DF80B2045F020038DF80D208DF81C
S3150800DF800F200DEB060200928DF809300C270125AB
S3150800DF9004AB8DF80A708DF80C608DF80E5094F865
S3150800DFA05A2003C394F85010E06C102302F0D2FAFA
S3150800DFB008B907B0F0BD642029F072F907B0F0BDC2
S3150800DFC070B5044688B00B260D4684F80961C1F37E
S3150800DFD0032684F80A2184F80D319DF830208DF83F
S3150800DFE00C500023082046F02005C4F8103184F8A8
S3150800DFF00E2184F80C3184F80F3184F8143184F832
S3150800E0000B018DF80D501025D4F80901D4F80D111F
S3150800E010D4F811218DF80F308DF811308DF81330A2
S3150800E0208DF80E500C2301258DF810308DF81250FE
S3150800E03005AB03AD07C3009594F85A2094F8501021
S3150800E040E06C142302F086FA08B908B070BD6420A3
S3150800E05029F026F908B070BD704700BF704700BFA9
S3150800E060704700BF90F871305BB970B50446806898
S3150800E07090F8463084B02BB92369DB071ED404B068
S3150800E08070BD7047437A002BF6D1637D002BF3D120
S3150800E09094F86920002AEFD1418B01231125437298
S3150800E0A084F86930A1812261227504F16B03009519
S3150800E0B0FFF7A6FD022384F87130E0E7012604F194
S3150800E0C01605CDE9005604F16B03227DA189039359
S3150800E0D0FFF7E2FD304629F0E3F8002200950192A9
S3150800E0E0227DA189039BA068FFF7D6FD237D3344D3
S3150800E0F03046237529F0D4F82B46227DA189A068DD
S3150800E100FFF720FE042384F8713004B070BD00BF09
S3150800E1100A2282760168002280F87120096A42750F
S3150800E12010B4074C80F86920A14280F86A20026181
S3150800E13002D15DF8044B70475DF8044B084700BFF1
S3150800E14061E0000810B590F86A3082B004463BBB1F
S3150800E150227DA189A0680132D2B204F16D0322752D
S3150800E160009304F11803FFF793FE22681649936893
S3150800E1708B4223D100230A21A17684F87130126AD2
S3150800E180124963758A4284F8693084F86A302361D3
S3150800E19017D10E220923A27684F8713002B010BD79
S3150800E1A0027D81898068013204F16F03D2B222753B
S3150800E1B0009304F11B03FFF76BFEC9E72046984757
S3150800E1C0E7E720469047E4E711E1000861E0000828
S3150800E1D030B4816039B14C6EDCB18C6EECB1CC6E6A
S3150800E1E0B4B10C6FDCB10F4C0F4D81F848200B61B0
S3150800E1F000220A214FF0E043C0E91A340560C0E95D
S3150800E200082230BC42750261A0F8702081767047FA
S3150800E210022401EB84046066E5E70124F9E7032498
S3150800E220F7E700BF00710050D49E040870B5837EDE
S3150800E2300B2B84B0044605D00E2B26D00A2B0ED005
S3150800E24004B070BD03699A05FAD523F40073012159
S3150800E2500A22036180F86A10827604B070BD0369E9
S3150800E26013F4807234D15905EAD500F11B0123F461
S3150800E2708063036180F86A200091027D818900F13C
S3150800E2806F038068FFF750FEDAE703695B04D7D5AA
S3150800E29081898068FFF742FC2268254993684FF612
S3150800E2A0FF708B42A0813ED100230A21A17684F813
S3150800E2B07130126A1F4963758A4284F8693084F896
S3150800E2C06A302361BCD0204604B0BDE870401047D0
S3150800E2D000F11B05012623F480720261CDE9005680
S3150800E2E000F16F03027D818980680393FFF7D4FCF0
S3150800E2F0304628F0D5FF002200950192227DA1899B
S3150800E300039BA068FFF7C8FC237D3344304623757A
S3150800E31028F0C6FF2B46227DA189A068FFF712FDCB
S3150800E3200B23A3768CE7204604B0BDE87040184757
S3150800E33011E1000861E0000870B590F87130023B01
S3150800E34086B00446072B27D8DFE813F03C004D00BB
S3150800E3507B009A00A900D6000800280003699906E0
S3150800E3601AD5036882681D696F48002182F846102D
S3150800E37082F8481085424FF00102627540F0CE805F
S3150800E38062680AB190472368DB69684A934240F09D
S3150800E390C880012384F8713006B070BD03691A0677
S3150800E3A0FAD5027D818980680132D2B204F16B0305
S3150800E3B02275009304F11603FFF76AFD052384F816
S3150800E3C07130E9E703695E07E6D5027D81898068D1
S3150800E3D00132D2B204F116032275FFF7B3FC032308
S3150800E3E084F87130D8E703699D07D5D590F8683069
S3150800E3F0C27D012B86BF002380F8683043F0700584
S3150800E400837DCDE9003288BF7025818980688DF8C3
S3150800E410175001230DF11702FFF7B0FB012028F072
S3150800E4203FFF227DA189A0680132D2B2132322754B
S3150800E430009304F16D03FFF7E3FB072384F87130BB
S3150800E440AAE703699A07A7D590F86830C27D012B19
S3150800E45086BF002380F8683043F07005837DCDE9D8
S3150800E460003288BF7025818980688DF8175001238E
S3150800E4700DF11702FFF782FB062384F871308BE74C
S3150800E48003691B0788D581898068FFF747FB002346
S3150800E4904FF6FF72A281236184F871307CE7036925
S3150800E4A0DB067FF579AF00F118050126CDE90056A0
S3150800E4B000F16D03027D818980680393FFF7ECFB09
S3150800E4C0304628F0EDFE002200950192227DA189B2
S3150800E4D0039BA068FFF7E0FB237D33443046237592
S3150800E4E028F0DEFE2B46227DA189A068FFF72AFCCC
S3150800E4F0082384F871304FE7036958067FF54CAF57
S3150800E500227DA189A0680132D2B204F118032275CE
S3150800E510FFF718FC082384F871303DE72046A84722
S3150800E52037E72046984734E79DB900085DE00008BC
S3150800E53070B5437D82B004460D4613B90B7A022B9B
S3150800E54044D0A068437A13B990F8473033B9A18903
S3150800E5502A78CBB29A4219D002B070BD637D002BDF
S3150800E560F5D194F86930002BF1D12A7A022AEED136
S3150800E570AA89112AEBD1418B80F8473001224272D1
S3150800E58084F86920A18184F87130E1E76A780B1272
S3150800E59043F020039A42DFD1EB88012B5BD0AB799D
S3150800E5A094F86F20EE799A4271D094F86D209A42C9
S3150800E5B019D094F86B209A4239D02046FFF736FED8
S3150800E5C0204602B0BDE87040FFF7B6BE8B89012B26
S3150800E5D0B7D18068827A002AB4D18372428BA2812D
S3150800E5E00A23A376AEE794F86E20B242E1D12B7ADD
S3150800E5F0A12BE2D128F04EFE2368BD4A5B6960670D
S3150800E60093422E7940F0E5816B7A012B00F0D08198
S3150800E610022BD2D1606A0028CFD002680A3500954D
S3150800E620B31E1568DBB200222146A847C5E794F851
S3150800E6306C30B342C1D12B7AA32BBED12368AD4A25
S3150800E6409B699342B9D029790139C9B205F1090202
S3150800E65020469847B1E72B7A012BAED0032B3CD046
S3150800E660022B63D0052B75D0042B00F09480062B63
S3150800E67000F0D180072B00F00A810A2B9DD16A7A17
S3150800E68022756B7B00932B7BFFF79AFC95E794F832
S3150800E6907020B24289D12B7A022B00F0A380042B7A
S3150800E6A000F0DD80062B88D16A7AAB7A84F82920B7
S3150800E6B0072284F82820904D227F84F82A300023E8
S3150800E6C084F82B302386E37EE562CDE900320A23FF
S3150800E6D004F12802FFF752FA6FE72B8A002B7FF422
S3150800E6E06CAF6B8A002B7FF468AFAB7B94F86F2016
S3150800E6F09A4200F0218194F86B209A4200F00B812F
S3150800E70094F86D209A427FF458AFEA7B94F86E30FD
S3150800E7109A427FF452AF6B7A23752A7B2369227655
S3150800E7206A7B627643F04003236146E7AB89012B97
S3150800E7304DD0112B00F0A080132B7FF43EAF6B7ADF
S3150800E7402375AA7B23692276EA7B627643F0100357
S3150800E750236132E72B8A002B7FF42FAF2B7B94F8AB
S3150800E7606F209A4200F0CA8094F86B209A4200F013
S3150800E770F78094F86D209A427FF41FAF6A7B94F86D
S3150800E7806E309A427FF419AF23696A7A227543F08C
S3150800E7902003236111E72B7B94F86F209A4200F03F
S3150800E7A08F8094F86B209A4200F0968094F86D203A
S3150800E7B09A427FF402AF6A7B94F86E309A427FF4ED
S3150800E7C0FCAE6A7A04F11803FFF70CFBF5E66B7AE0
S3150800E7D02375AA7B2369E276EA7B227743F4807362
S3150800E7E02361EAE6032384F828306B7A84F8293013
S3150800E7F0AB7AE27E84F82A30257F002384F82B3012
S3150800E80023860523E362CDE900250A2304F12802BD
S3150800E810FFF7B4F9D1E62B7B94F86F209A4200F003
S3150800E820AC8094F86B209A4200F0B48094F86D207E
S3150800E8309A427FF4C2AE6A7B94F86E309A427FF4AD
S3150800E840BCAE6A7A227504F11803009304F16D03CD
S3150800E850FFF76AFB236820469B689847ADE60523C1
S3150800E86084F828306B7A84F82930AB7A84F82A3011
S3150800E870214D227F002323E76B7A2375AA7B236920
S3150800E880A275EA7BE27543F00103236195E62B7BCB
S3150800E890E27E9A4200F09180A27D9A4200F0A08022
S3150800E8A0227E9A427FF489AE6A7B637E9A427FF41F
S3150800E8B084AE23696A7A227543F0800323617CE675
S3150800E8C06E7B94F8702096427FF46BAF6A7A04F1F7
S3150800E8D01B03FFF787FA70E66E7B94F86C20964266
S3150800E8E07FF464AF6A7A04F11603FFF77BFA64E6ED
S3150800E8F059E00008B5B9000805000235697B94F8A7
S3150800E900702091427FF430AF23696A7A227543F406
S3150800E9100073236151E6E97B94F86C2091427FF4F9
S3150800E920EFAE6B7A23752A7B2369A2756A7BE2753B
S3150800E93043F00403236140E6EE7B94F87020964288
S3150800E9407FF4D9AE6B7A23752A7BE2760133DAB285
S3150800E9506B7B2377227504F11B03FFF7F3F92CE68B
S3150800E960697B94F86C2091427FF403AF23696A7A35
S3150800E970227543F0020323611FE66E7B94F870202C
S3150800E98096427FF44EAF23696A7A227543F4806310
S3150800E990236112E66E7B94F86C2096427FF446AFAC
S3150800E9A06A7A227504F11603009304F16B034FE7A4
S3150800E9B0206A00287FF431AEFFE5697B227F914209
S3150800E9C07FF46AAF23696A7A227543F48043236128
S3150800E9D0F3E5711EC9B205F109022046984713E608
S3150800E9E0697BE27D91427FF45BAF23696A7A22757F
S3150800E9F043F008032361E0E551B9037A03F00F02F7
S3150800EA00072A56D013F00E0F0CBF012000207047BE
S3150800EA10132931D0012931D014292DD002293FD00C
S3150800EA20152929D0032932D0162925D0A1F10803A2
S3150800EA30DBB21E2B3FD84C4A22FA03F3DB073CD441
S3150800EA4001F0EF03092B40D0A1F12703012B3CD994
S3150800EA500A293CD029293AD00B293AD02A2938D074
S3150800EA60A1F10E03DBB21D2B35D8404A22FA03F377
S3150800EA70DA0730D50A2321E000207047007A00F033
S3150800EA800F00013802288CBF002001207047007A49
S3150800EA9000F00F00053802288CBF002001207047BF
S3150800EAA0007A00F00F00033802288CBF00200120EE
S3150800EAB07047012070473329C2D10C238068C0F300
S3150800EAC01700D84000F0010070470D23F6E70E2323
S3150800EAD0F4E70F23F2E7A1F10F03DBB21D2B09D9E7
S3150800EAE00C290ED02D290CD00D2901D02E2924D180
S3150800EAF00923E3E71D4A22FA03F3DB0703D50B23B1
S3150800EB00DCE70823DAE71E2919D0052927D01D29AD
S3150800EB1025D0062925D01F2923D007291DD020292D
S3150800EB201BD0A1F11003DBB21F2B0AD8104A22FA18
S3150800EB3003F3DA0705D51023C0E70429E3D1072331
S3150800EB40BCE7A1F11103DBB21F2B95D8094A22FABB
S3150800EB5003F3DB0790D51123B0E70423AEE70623BA
S3150800EB60ACE70523AAE700BF01800942010040205F
S3150800EB700100048001020480B1B3132934D00129AD
S3150800EB8049D0142947D0022949D0152947D0032945
S3150800EB9050D016294ED0A1F10803DBB21E2B42D85D
S3150800EBA05E4A22FA03F3DB073FD401F0EF03092B91
S3150800EBB044D0A1F12703012B40D90A2943D029299A
S3150800EBC041D00B2944D02A2942D0A1F10E03DBB249
S3150800EBD01D2B42D8524A22FA03F3DA073DD54FF4E1
S3150800EBE080616FF4806302E001216FF0010310B4C5
S3150800EBF0B0F8444090F8432042EA042213401C0A25
S3150800EC000A42A0F8444080F843305DF8044B14BF2C
S3150800EC1001200020704702216FF00203E7E7042174
S3150800EC206FF00403E3E73329BFD14FF480516FF443
S3150800EC308053DCE708216FF00803D8E74FF400514A
S3150800EC406FF40053D3E74FF480416FF48043CEE767
S3150800EC504FF400416FF40043C9E7A1F10F03DBB29B
S3150800EC601D2B0CD90C2914D02D2912D00D2901D011
S3150800EC702E2930D14FF400716FF40073B7E7284A94
S3150800EC8022FA03F3DB0709D54FF400616FF400633A
S3150800EC90ADE74FF480716FF48073A8E71E291CD086
S3150800ECA0052931D01D292FD0062931D01F292FD06B
S3150800ECB0072925D0202923D0A1F11003DBB21F2B69
S3150800ECC00FD8184A22FA03F3DA070AD54FF4803127
S3150800ECD06FF480338BE70429E0D180216FF080033D
S3150800ECE085E7A1F11103DBB21F2B15D80E4A22FACC
S3150800ECF003F3DB0710D54FF400316FF4003376E7E2
S3150800ED0010216FF0100372E740216FF040036EE7A1
S3150800ED1020216FF020036AE700207047018009422E
S3150800ED200100402001000480010204801B2920D92B
S3150800ED30A1F12103DAB2122A05D8134BD340DB43DB
S3150800ED4013F001031BD0A1F10E03DBB21D2B04D86F
S3150800ED500E4A22FA03F3DA0713D4A1F10F03DBB242
S3150800ED601D2B0CD8094A22FA03F3DB0707D5007BCB
S3150800ED707047074BCB40DB4313F00103E3D1002078
S3150800ED807047C07A704700BFE103040001004020C5
S3150800ED900F0FF80B01440879704700BF012910B519
S3150800EDA00B4604463FD91146002A3CD01278012A60
S3150800EDB057D0112A42D1032B40D9033BDAB23C2A59
S3150800EDC028BF3C220331043036F0C8F8A168236C0A
S3150800EDD0C1F31701C3F31703994224D021EA0303A9
S3150800EDE084F84330227A206C02F00F021B0A61F382
S3150800EDF01700072AA4F84430206400D0FAB9012382
S3150800EE00053A022A98BF43F0080394F84E209A421E
S3150800EE1009D094F8431084F84E3023EA020363F3CA
S3150800EE20030184F8431094F84D303BB1214620463F
S3150800EE3051F8463BBDE810401B68184710BD511EE7
S3150800EE40A2F10103B3FA83F302294FEA5313A2F19D
S3150800EE50030110D8022943F00203D6D843F004036D
S3150800EE60CEE7013BDAB23C2A28BF3C220131043006
S3150800EE7036F074F8AAE70229F0D9C1E7F0B4036CB2
S3150800EE8090F82F6090F826C090F82A7090F83350C2
S3150800EE9090F8384090F83C104FF07F3203F07043FA
S3150800EEA046F0800647F0800745F0800544F0800468
S3150800EEB042604CF0800C43F0080241F080010023C8
S3150800EEC080F82F60082680F82A7080F8335086600C
S3150800EED080F8384080F826C0F0BC80F83C10026400
S3150800EEE00373C0F84630A0F84A30A0F84C3080F8D2
S3150800EEF04E30704751B9C37E03F00F02072A56D029
S3150800EF0013F00E0F0CBF012000207047132931D0D3
S3150800EF10012931D014292DD002293FD0152929D00D
S3150800EF20032932D0162925D0A1F10803DBB21E2BFE
S3150800EF303FD8524A22FA03F3DA073CD401F0EF032A
S3150800EF40092B41D0A1F12703012B3DD90A293DD030
S3150800EF5029293BD00B293BD02A2939D0A1F10E0308
S3150800EF60DBB21D2B36D8464A22FA03F3DB0731D526
S3150800EF700A2221E000207047C07E00F00F00013809
S3150800EF8002288CBF002001207047C07E00F00F00C9
S3150800EF90053802288CBF002001207047C07E00F08B
S3150800EFA00F00033802288CBF00200120704701207B
S3150800EFB070473329C2D10C22C37E808B43EA0020D6
S3150800EFC0D04000F0010070470D22F5E70E22F3E766
S3150800EFD00F22F1E7A1F10F03DBB21D2B09D90C298A
S3150800EFE00ED02D290CD00D2901D02E2924D1092285
S3150800EFF0E2E7234A22FA03F3DA0703D50B22DBE713
S3150800F0000822D9E71E2919D005292CD01D292AD06E
S3150800F01006292AD01F2928D0072922D0202920D01E
S3150800F020A1F11003DBB21F2B0AD8164A22FA03F302
S3150800F030DB0705D51022BFE70429E3D10722BBE782
S3150800F040A1F11103DBB21F2B11D9A1F11203DBB217
S3150800F0501F2B8FD80C4A22FA03F3DB078AD5122214
S3150800F060AAE70422A8E70622A6E70522A4E7074A94
S3150800F07022FA03F3DA07E8D511229DE7018009424F
S3150800F0800100402001000480010400800102048080
S3150800F090B1B3132934D0012949D0142947D00229FC
S3150800F0A049D0152947D0032950D016294ED0A1F1A9
S3150800F0B00803DBB21E2B42D8664A22FA03F3DA07A4
S3150800F0C03FD401F0EF03092B44D0A1F12703012B0C
S3150800F0D040D90A2943D0292941D00B2944D02A29C5
S3150800F0E042D0A1F10E03DBB21D2B42D85A4A22FAAE
S3150800F0F003F3DB073DD54FF480616FF4806302E0CC
S3150800F10001216FF0010310B4B0F8404090F83F2099
S3150800F11042EA042213401C0A0A42A0F8404080F83A
S3150800F1203F305DF8044B14BF0120002070470221D0
S3150800F1306FF00203E7E704216FF00403E3E73329DE
S3150800F140BFD14FF480516FF48053DCE708216FF08C
S3150800F1500803D8E74FF400516FF40053D3E74FF490
S3150800F16080416FF48043CEE74FF400416FF40043CB
S3150800F170C9E7A1F10F03DBB21D2B0CD90C2914D05A
S3150800F1802D2912D00D2901D02E2930D14FF4007126
S3150800F1906FF40073B7E7304A22FA03F3DA0709D5A2
S3150800F1A04FF400616FF40063ADE74FF480716FF4BC
S3150800F1B08073A8E71E291CD0052936D01D2934D00E
S3150800F1C0062936D01F2934D007292AD0202928D045
S3150800F1D0A1F11003DBB21F2B0FD8204A22FA03F342
S3150800F1E0DB070AD54FF480316FF480338BE70429A7
S3150800F1F0E0D180216FF0800385E7A1F11103DBB22E
S3150800F2001F2B1CD9A1F11203DBB21F2B15D8144AE8
S3150800F21022FA03F3DB0710D54FF480216FF480231D
S3150800F22071E710216FF010036DE740216FF040037E
S3150800F23069E720216FF0200365E700207047094A37
S3150800F24022FA03F3DA07DDD54FF400316FF4003301
S3150800F25059E700BF018009420100402001000480EF
S3150800F26001040080010204801B2920D9A1F1210391
S3150800F270DAB2122A05D8134BD340DB4313F0010345
S3150800F2801BD0A1F10E03DBB21D2B04D80E4A22FABD
S3150800F29003F3DA0713D4A1F10F03DBB21D2B0CD845
S3150800F2A0094A22FA03F3DB0707D5407E7047074B66
S3150800F2B0CB40DB4313F00103E3D100207047007E07
S3150800F2C0704700BFE1030400010040200F0FF80B50
S3150800F2D00144087D704700BF012910B50B46044656
S3150800F2E044D91146002A41D01278012A62D0312A1F
S3150800F2F04DD1022B4BD0023BDAB2282A28BF28224E
S3150800F3000231143035F02AFEE27EA18BE36B42EA25
S3150800F3100121C3F31703994223D021EA030384F892
S3150800F3203F30E06B02F00F021B0A61F31700072A51
S3150800F330A4F84030E06300D052BB0123053A022A04
S3150800F34098BF43F0080394F84B209A4209D094F8E2
S3150800F3503F1084F84B3023EA020363F3030184F871
S3150800F3603F10B4F84C300133A4F84C3094F84A30C6
S3150800F3703BB12146204651F8423BBDE810401B6888
S3150800F3801847E37A002BF4D1E37C002BF1D110BDAA
S3150800F390511EA2F10103B3FA83F302294FEA53136C
S3150800F3A0A2F1030110D8022943F00203CBD843F097
S3150800F3B00403C3E7013BDAB2282A28BF2822013111
S3150800F3C0143035F0CBFD9FE70229F0D9B6E700BF28
S3150800F3D030B4C36B90F8344090F83810082203F024
S3150800F3E070434FF07F3544F08004C27641F08001C7
S3150800F3F01A430023456180F8344080F8381030BC41
S3150800F400C26383830371C3720373C3740383C0F82F
S3150800F4104230C0F84630A0F84A3070470378262BA9
S3150800F42012D00BD8012B01D0022B23D10B704378B5
S3150800F4304B7083788B700023C3717047FC2B19D1EE
S3150800F4400B700023C37170470B704378DB434B7016
S3150800F45083780BB102238B70C3780B7103794B71D8
S3150800F46043798B7183795B0808BF01234B720023AC
S3150800F470C371704700230B704B708B700023C371E8
S3150800F480704700BF00207047002070470020704773
S3150800F490002070470020704711F0800F42D1072BDB
S3150800F4A040D830B4044612B1C079072837D0E07C7A
S3150800F4B0002869D0A07E002868D094F8210000288A
S3150800F4C066D094F82800002864D094F82F00002805
S3150800F4D062D094F83600002860D094F83D000028E1
S3150800F4E05ED094F8440000285CD094F84B000028BD
S3150800F4F05AD094F85200002858D094F85900002899
S3150800F50056D094F86000002854D094F86700002874
S3150800F51052D094F86E0038B194F8750000B3002004
S3150800F52030BC7047002070470E25D9B1C1F30201DF
S3150800F5304FF0000061F3C500FAB1E1790131C9B2B3
S3150800F540E17101F00701C5EBC50541EA82132C44B8
S3150800F55003F047031843207300F07F0030BC704760
S3150800F5600F25E2E7C5EBC50552B1621941231373AE
S3150800F570E27901321846E271D2E703F00701E2E7C1
S3150800F5802C4401202073CBE70125CEE70225CCE7E2
S3150800F5900325CAE70425C8E70525C6E70625C4E7FF
S3150800F5A00725C2E70825C0E70925BEE70A25BCE7FF
S3150800F5B00B25BAE70C25B8E70D25B6E7C1EBC1025E
S3150800F5C002442DE9F843072303FB0103127B1D7B45
S3150800F5D05306884604464FEAC10940F1CF8005F034
S3150800F5E0070501260827BB1B23441B7BC3F3C2035D
S3150800F5F0AB4200F0D480731CDBB2102B00F0BB804A
S3150800F600C3EBC3022244DF00127BC2F3C202AA4242
S3150800F61000F0C480B31CDBB2102B00F0AC80C3EB47
S3150800F620C3022244DF00127BC2F3C202AA4200F0E0
S3150800F630B580F31CDBB2102B00F09D80C3EBC30230
S3150800F6402244DF00127BC2F3C202AA4200F0A6805F
S3150800F650331DDBB2102B00F08E80C3EBC3022244AD
S3150800F660DF00127BC2F3C202AA4200F09780731D24
S3150800F670DBB2102B7FD0C3EBC3022244DF00127B20
S3150800F680C2F3C202AA4200F08980B31DDBB2102B76
S3150800F69071D0C3EBC3022244DF00127BC2F3C2025D
S3150800F6A0AA427BD0F31DDBB2102B64D0C3EBC30296
S3150800F6B02244DF00127BC2F3C202AA426ED006F1D0
S3150800F6C00803DBB2102B56D0C3EBC3022244DF007B
S3150800F6D0127BC2F3C202AA4260D006F10903DBB26A
S3150800F6E0102B48D0C3EBC3022244DF00127BC2F3BF
S3150800F6F0C202AA4252D006F10A03DBB2102B3AD054
S3150800F700C3EBC3022244DF00127BC2F3C202AA4241
S3150800F71044D006F10B03DBB2102B2CD0C3EBC3028B
S3150800F7202244DF00127BC2F3C202AA4236D006F197
S3150800F7300C03DBB2102B1ED0C3EBC3022244DF003E
S3150800F740127BC2F3C202AA4228D006F10D03DBB22D
S3150800F750102B10D0C3EBC3022244DF00127BC2F386
S3150800F760C202AA421AD0022E05D094F87530C3F305
S3150800F770C203AB421BD0E379AB4215D0A9EB08080C
S3150800F780A04401220023043488F80D20C8F8084054
S3150800F79088F80C3088F80E30BDE8F8831E463146E6
S3150800F7A02046FFF70BFF1EE7013DE571E6E70F264A
S3150800F7B07827F4E7D9B3C37C8B4240D0837E8B424B
S3150800F7C03FD090F821308B423DD090F828308B42BC
S3150800F7D03BD090F82F308B422BD090F836308B42A6
S3150800F7E035D090F83D308B4233D090F844308B4278
S3150800F7F031D090F84B308B422FD090F852308B4254
S3150800F8002DD090F859308B422BD090F860308B422F
S3150800F81029D090F867308B4227D090F86E308B420B
S3150800F82025D090F875308B4223D0002070470830D9
S3150800F83070470523C3EBC3030830184470470123F8
S3150800F840F8E70223F6E70323F4E70423F2E706239F
S3150800F850F0E70723EEE70823ECE70923EAE70A239C
S3150800F860E8E70B23E6E70C23E4E70D23E2E70E239C
S3150800F870E0E70F23DEE700BF41292DE9F8430446F8
S3150800F88049D0C37C8B4200F08E81837E8B4200F088
S3150800F8908D8190F821308B4200F08B8190F82830CA
S3150800F8A08B4200F0898190F82F308B4200F08781D7
S3150800F8B090F836308B4200F0858190F83D308B42C7
S3150800F8C000F0838190F844308B4200F0818190F8F3
S3150800F8D04B308B4275D090F852308B4200F07B81CA
S3150800F8E090F859308B4200F0798190F860308B425D
S3150800F8F000F0778190F867308B4200F0758190F8B8
S3150800F9006E308B4200F0738190F875308B4200F0B0
S3150800F9107181BDE8F883021D002301214FF4807030
S3150800F920C4F80F20C4F81620C4F81D206262C4F873
S3150800F9302B20C4F83220C4F839202264C4F84720A2
S3150800F940C4F84E20E374237784F8213084F82A30EB
S3150800F95084F82F3084F8383084F83D3084F84630FF
S3150800F96084F84B3084F8543084F85930A182618485
S3150800F9702186E187A4F84C10A4F85A1060832085E4
S3150800F980E086A4F84400A4F85200C4F85520A4F868
S3150800F9906000A4F86810A4F86E00A4F87610E37165
S3150800F9A084F86230E26584F86730C4F8632084F826
S3150800F9B07030C4F86A2084F87530C4F87120BDE840
S3150800F9C0F8834FF00908C8EBC80323444FEAC8096F
S3150800F9D01B7B03F007065B0640F1CF80012508274D
S3150800F9E07B1B23441B7BC3F3C203B34200F0D680C0
S3150800F9F06B1CDBB2102B00F0BB80C3EBC3022244A6
S3150800FA00DF00127BC2F3C202B24200F0C680AB1C12
S3150800FA10DBB2102B00F0AC80C3EBC3022244DF003C
S3150800FA20127BC2F3C202B24200F0B780EB1CDBB213
S3150800FA30102B00F09D80C3EBC3022244DF00127B2B
S3150800FA40C2F3C202B24200F0A8802B1DDBB2102B13
S3150800FA5000F08E80C3EBC3022244DF00127BC2F3A0
S3150800FA60C202B24200F099806B1DDBB2102B7FD028
S3150800FA70C3EBC3022244DF00127BC2F3C202B242C6
S3150800FA8000F08B80AB1DDBB2102B71D0C3EBC30229
S3150800FA902244DF00127BC2F3C202B2427DD0EB1DC4
S3150800FAA0DBB2102B64D0C3EBC3022244DF00127B07
S3150800FAB0C2F3C202B24270D005F10803DBB2102BC2
S3150800FAC056D0C3EBC3022244DF00127BC2F3C20244
S3150800FAD0B24262D005F10903DBB2102B48D0C3EB62
S3150800FAE0C3022244DF00127BC2F3C202B24254D0E0
S3150800FAF005F10A03DBB2102B3AD0C3EBC30222444A
S3150800FB00DF00127BC2F3C202B24246D005F10B03F4
S3150800FB10DBB2102B2CD0C3EBC3022244DF00127BCE
S3150800FB20C2F3C202B24238D005F10C03DBB2102B85
S3150800FB301ED0C3EBC3022244DF00127BC2F3C2020B
S3150800FB40B2422AD005F10D03DBB2102B10D0C3EB5D
S3150800FB50C3022244DF00127BC2F3C202B2421CD0A7
S3150800FB60022D05D094F87530C3F3C203B34244D0CE
S3150800FB70E379B34201D1013EE671A9EB0808A04436
S3150800FB8001220023043488F80D20C8F8084088F8B4
S3150800FB900C3088F80E30BDE8F8831D462946204605
S3150800FBA0FFF70CFD1CE74FF001080CE74FF00208C1
S3150800FBB009E74FF0030806E74FF0040803E74FF09C
S3150800FBC0050800E74FF00608FDE64FF00708FAE6D5
S3150800FBD04FF00808F7E64FF00A08F4E64FF00B086E
S3150800FBE0F1E64FF00C08EEE64FF00D08EBE64FF0A5
S3150800FBF00E08E8E64FF00F08E5E60F257827CDE76B
S3150800FC0070B4304A304C314E0260011D00224FF468
S3150800FC108075446001248160C0F80F10C0F8161082
S3150800FC20C0F81D104162C0F82B10C0F83210C0F899
S3150800FC3039100164C0F84710858145830585C58656
S3150800FC40A0F84450848244840486C4878273C274AC
S3150800FC50027780F8212080F82A2080F82F2080F863
S3150800FC60382080F83D2080F8462080F84B20A0F800
S3150800FC704C40C0F84E10C0F85510C165C0F8631066
S3150800FC80C0F86A10C0F871101121A0F85250A0F8F7
S3150800FC905A40A0F86050A0F86840A0F86E50A0F846
S3150800FCA07640317080F8542070BC80F8592080F86E
S3150800FCB0622080F8672080F8702080F8752080F828
S3150800FCC0B8207047009F040800083C00910F0020E8
S3150800FCD0002B46D000293ED010B4C47C8C424ED0AE
S3150800FCE0847E8C424DD090F821408C423BD090F8CF
S3150800FCF028408C4247D090F82F408C4245D090F847
S3150800FD0036408C4243D090F83D408C4241D090F822
S3150800FD1044408C423FD090F84B408C423DD090F8FE
S3150800FD2052408C423BD090F859408C4239D090F8DA
S3150800FD3060408C4237D090F867408C4235D090F8B6
S3150800FD406E408C4233D090F875408C4231D0D62024
S3150800FD505DF8044B7047083001710360427100205A
S3150800FD607047D82070470324C4EBC40408302044E5
S3150800FD704271017103605DF8044B0020704701244D
S3150800FD80F2E70224F0E70424EEE70524ECE706246C
S3150800FD90EAE70724E8E70824E6E70924E4E70A246B
S3150800FDA0E2E70B24E0E70C24DEE70D24DCE70E246B
S3150800FDB0DAE70F24D8E700BFF0B5054683B00C464E
S3150800FDC000294BD0C17CA14200F01781877EA7424B
S3150800FDD000F01C8190F82110A14200F0198190F8DA
S3150800FDE02810A14200F0168190F82F10A14200F0C9
S3150800FDF0B58090F83610A14200F00E8190F83D10BB
S3150800FE00A14200F00B8190F84410A14200F00A814B
S3150800FE1090F84B10A14200F0098190F85210A142C7
S3150800FE2000F0088190F85910A14200F0078190F877
S3150800FE306010A14200F0068190F86710A14200F018
S3150800FE40058190F86E10A14200F0048190F87510B3
S3150800FE50A14200F00381D62003B0F0BD80680028D7
S3150800FE6000F0C88005F1080637467979002900F0C0
S3150800FE70BC800139C9B2013101EB4101014403E0FB
S3150800FE800330884200F0B18007789742F8D182782B
S3150800FE90186093080F2B28BF0F230127089A754867
S3150800FEA007FA03F3013B13801021002228F0DEF93C
S3150800FEB04FF0E20C4FF0FF3301A902226E488DF88D
S3150800FEC004C08DF805402BF061FC6A483A461021BB
S3150800FED028F0CCF9D82367488DF803300022102182
S3150800FEE028F0C4F93A464FF0FF330DF10301624892
S3150800FEF02BF04CFC00244FF0FF333A4601A95E482C
S3150800FF008DF804402BF0ECFE5A483A46102128F0AA
S3150800FF10ADF9B3799DF80440EBB195F8B8301C43B8
S3150800FF2044F0020453480022102128F09FF9DA25EC
S3150800FF3001A94FF0FF3302224F488DF805408DF88E
S3150800FF4004502BF023FC4B480122102128F08EF98F
S3150800FF50002003B0F0BD04F0F904E3E70521C1EB86
S3150800FF60C10105F1080046184158002942D0A742A8
S3150800FF7056D095F82110A14256D095F82810A142DE
S3150800FF8056D095F82F10A14256D095F83610A142B2
S3150800FF9056D095F83D10A14256D095F84410A14286
S3150800FFA056D095F84B10A14256D095F85210A1425A
S3150800FFB056D095F85910A14254D095F86010A14230
S3150800FFC052D095F86710A14250D095F86E10A1420C
S3150800FFD04ED095F87510A14207D10F21C1EBC1018A
S3150800FFE04718405800287FF440AF0022DB201A60EB
S3150800FFF003B0F0BDD72003B0F0BDD0F80F1005F15F
S315080100000F0608300029F5D00121E7E70221A6E706
S315080100100321A4E70421A2E70621A0E707219EE719
S315080100200221DBE708219AE70321D7E7092196E7A9
S315080100300421D3E70A2192E70521CFE70B218EE7B1
S315080100400621CBE70C218AE70721C7E70D2186E7B9
S315080100500821C3E70E2182E70921BFE70F217EE7C1
S315080100600A21BBE70B21B9E70C21B7E70D21B5E753
S315080100700E21B3E700100240ACB001202DE9F04F84
S315080100804D788BB08B46691E3F290592029300F283
S315080100905882984627F0FEF89BF80220074612F088
S315080100A0010F96484FF000024FF0100114BF802649
S315080100B04026EA2428F0DAF84FF0FF3309A902228C
S315080100C08F488DF825608DF824402BF05FFB8B480F
S315080100D00122102128F0CAF807F59C57434608372C
S315080100E0002B00F03382ABB2844CDFF814820693FE
S315080100F00DF1230A4FF0000900970022102120462E
S3150801010028F0B4F8029B069A934228BF13461E4666
S31508010110079312254FF0FF33012209A940468DF8AE
S3150801012024502BF033FB4FF0FF33324614994046E7
S315080101302BF02CFB01221021204628F097F80022EB
S315080101401021204628F092F8F3B21E4601933A256B
S315080101504FF0FF33022209A940468DF825608DF834
S3150801016024502BF013FB01221021204628F07EF89B
S315080101709BF8005000221021204628F077F845F018
S315080101802005022209A9F2264FF0FF3340468DF8D1
S3150801019025508DF824602BF0F9FA0122102120460A
S315080101A028F064F8C8230022102120468DF8213052
S315080101B028F05CF84FF0FF3301220DF1210140468A
S315080101C02BF0E4FA4FF0FF33012209A940468DF8D6
S315080101D024902BF085FD01221021204628F046F8AF
S315080101E09DF92430002BDDDA00221021204628F063
S315080101F03DF848F2CA054FF0FF33022209A94046E5
S31508010200ADF824502BF0C2FA01221021204628F01D
S315080102102DF8F8270022102120468DF8237028F0A2
S3150801022025F84FF0FF330122514640462BF0AEFA2E
S315080102304FF0FF33012209A940468DF824902BF08F
S315080102404FFD01221021204628F010F89DF8245070
S3150801025015F00F0500F051810023CDE9033327F08E
S3150801026019F8009BC01A002880F24881062D49D04A
S315080102700E2D00F05E81042D00F04F811F480022EB
S31508010280102127F0F3FF3A24022209A91C48ADF8E8
S3150801029024404FF0FF332BF079FA18480122102138
S315080102A027F0E4FFF82315488DF8233000221021A2
S315080102B027F0DCFF51464FF0FF33012210482BF09F
S315080102C065FA002409A94FF0FF3301220C488DF87D
S315080102D024402BF005FD09480122102127F0C6FF0D
S315080102E09DF824309BF80220C3F3401363F3000200
S315080102F028468BF802200BB0BDE8F08F00100240AB
S31508010300ACB001200022102120468DF8237027F079
S31508010310ADFF4FF0FF330122514640462BF036FA26
S315080103204FF0FF33012209A940468DF824902BF09E
S31508010330D7FC01221021204627F098FF9DF824308A
S315080103409BF8022083F02003C3F3401363F30002F2
S3150801035012F0010F8BF802204FF010014FF0000246
S31508010360204614BF80254025EA2627F07FFF022272
S3150801037009A94FF0FF3340468DF825508DF82460C2
S315080103802BF004FA01221021204627F06FFF0022E4
S315080103901021204627F06AFF3A254FF0FF33022243
S315080103A009A94046ADF824502BF0F0F90122102195
S315080103B0204627F05BFF149B0022102120461E7859
S315080103C027F054FF4FF0120C4FF0FF33022209A910
S315080103D040468DF824C08DF825602BF0D7F9012207
S315080103E01021204627F042FF00221021204627F03F
S315080103F03DFF4FF0FF33022209A98DF824504046EC
S31508010400019D8DF825502BF0C1F9012210212046B6
S3150801041027F02CFF9BF8005000221021204627F0D8
S3150801042025FF45F02005022209A9F2264FF0FF33E0
S3150801043040468DF825508DF824602BF0A7F9012246
S315080104401021204627F012FFC8230022102120463A
S315080104508DF8223027F00AFF4FF0FF3301220DF104
S31508010460220140462BF092F94FF0FF33012209A9E8
S3150801047040468DF824902BF033FC012210212046AA
S3150801048027F0F4FE9DF92430002BDDDA0022102135
S31508010490204627F0EBFE48F2CA054FF0FF33022249
S315080104A009A94046ADF824502BF070F90122102114
S315080104B0204627F0DBFE0022102120468DF8237006
S315080104C027F0D4FE4FF0FF330122514640462BF068
S315080104D05DF94FF0FF33012209A940468DF82490B2
S315080104E02BF0FEFB01221021204627F0BFFE9DF8C6
S315080104F0245015F00F057FF4B2AE0025029B079A2A
S3150801050014999B1A9BB2114402931491002B7FF400
S31508010510F4AD002D3FF4C6AEB0E6049B059A01334F
S315080105209BB20493002A3FF432AF93427FF42FAF74
S31508010530A4E6039B0133DBB2032B03937FF427AFB6
S315080105409CE6DA2528460BB0BDE8F08F029D0DF131
S31508010550230AA7E670B584B00DF10A051C460026E4
S31508010560009503AB254603960446ADF80A60FFF7E6
S3150801057023FC40B9089B0093BDF80A2003992B4632
S315080105802046FFF77BFD04B070BD00BF2DE9F04F93
S3150801059085B015468946019326F07CFE4FF0000A80
S315080105A000F59C57504C49EA05090837D346554684
S315080105B026F070FEC01B002870DA002210212046A2
S315080105C027F054FEF22503A94FF0FF3302224748CC
S315080105D08DF80D908DF80C502BF0D8F801221021CA
S315080105E0204627F043FE414E4FF0C8081DE08DF81E
S315080105F00A8027F03BFE4FF0FF3301220DF10A0175
S3150801060030462BF0C3F84FF0FF33012203A93046D9
S315080106108DF80C502BF064FB01221021204627F09F
S3150801062025FE9DF90C30AB423CDB26F033FE034632
S315080106300025DB1BAB422A464FF010012046D6DBCC
S31508010640F8230022102120468DF80B3027F00EFEE4
S315080106504FF0FF3301220DF10B0124482BF096F8D8
S31508010660002503A94FF0FF33012220488DF80C50CD
S315080106702BF036FB01221021204627F0F7FD9DF8C5
S315080106800C5005F00F05042D22D00E2D06D10BF1C5
S31508010690010B5FFA8BFBBBF1030F89D1284605B025
S315080106A0BDE8F08F2A462046102127F0DFFD48F2E3
S315080106B0CA0503A94FF0FF3302220C48ADF80C50C6
S315080106C02BF064F801221021204627F0CFFDB7E769
S315080106D0019B0AF1010A1FFA8AFA002B3FF468AF57
S315080106E09A457FF465AFD9E700100240ACB0012006
S315080106F02DE9F04F2DED028B9B4687B00B46AF4E89
S315080107005B7800918978029300249DF84C30BBF8F8
S3150801071000A0019311F0020F054613464FF0100190
S3150801072022463046ABF8004008EE105A08EE903AD9
S315080107300CBF0D462025DDF84890A14F27F096FD00
S31508010740EA2005A94FF0FF3302228DF814009C48D0
S315080107508DF815502BF01AF801221021304627F092
S3150801076085FD0394009A18EE903A127818EE100A4D
S315080107700021FFF70BFF0628054600F0A180002897
S3150801078040F00E81C8230246102130468DF81130FB
S3150801079027F06CFD4FF0FF3301220DF111013846A8
S315080107A02AF0F4FF4FF0FF33012205A938468DF8E8
S315080107B014502BF095FA01221021304627F056FDE8
S315080107C09DF814305B0740F1F18030232A46102149
S315080107D030468DF8133027F049FD0DF113014FF01E
S315080107E0FF33012238462AF0D1FF4FF0FF330122A9
S315080107F005A938468DF814502BF072FA01221021FA
S31508010800304627F033FDBBF800409DF81480AAEB6B
S315080108100404D04524B224EAE474C8BF5FFA8AF80E
S3150801082044454FF008034FF000024FF010013046DF
S31508010830A8BF44468DF8123027F018FD4FF0FF3354
S3150801084001220DF1120138462AF0A0FF22460021A5
S31508010850484634F0ABFB4FF0FF334946A2B238465F
S315080108602BF03EFA01221021304627F0FFFC002228
S315080108701021304627F0FAFC40F2CA4C4FF0FF33FC
S31508010880022205A93846ADF814C02AF07FFF0122D5
S315080108901021304627F0EAFCBBF80030029A43449F
S315080108A09BB29045A144ABF8003051D353454FD282
S315080108B0019B002B3FF456AF184626F0F1FC51E791
S315080108C0F8233046002210218DF8133027F0CEFC8C
S315080108D00DF113014FF0FF33012238462AF056FF76
S315080108E0039C8DF814404FF0FF3305A901223846C1
S315080108F02BF0F6F930460122102127F0B7FC0099B2
S315080109009DF814308A7883F01003C3F3001363F358
S31508010910410212F0020F8A7030464FF010014FF073
S3150801092000020CBF0C462024EA2527F09FFC05A9E6
S315080109304FF0FF33022238468DF815408DF81450D2
S315080109402AF024FF01221021304627F08FFC09E7FF
S31508010950F8231A488DF813300022102127F086FC57
S315080109600DF113014FF0FF33012215482AF00EFF4E
S3150801097000244FF0FF3305A9012211488DF81440D0
S315080109802BF0AEF9012210210C4827F06FFC0099D3
S315080109909DF814308A78C3F3001363F341028A7011
S315080109A0284607B0BDEC028BBDE8F08FF025284636
S315080109B007B0BDEC028BBDE8F08F00BF0010024006
S315080109C0ACB0012070B584B00DF10A051C460026AD
S315080109D0009503AB25460396ADF80A6004469DF8D3
S315080109E02460FFF7E9F948B9089B0093BDF80A2086
S315080109F0039901962B462046FFF77AFE04B070BD8F
S31508010A002DE9F04F2DED028B8BB000260DF1160462
S31508010A109DF85C7000940796ADF816601D469DF822
S31508010A205860029607AB03979DF86090BDF86480FD
S31508010A30BDF868B0BDF86C701D9E04469246FFF776
S31508010A40BBF9844628B160460BB0BDEC028BBDE804
S31508010A50F08F029B8DF821300246039B61488DF881
S31508010A60223010218DF820508DF82390ADF824807E
S31508010A70ADF826B027F0FAFB4FF0220C0DF11A015A
S31508010A804FF0FF33012258488DF81AC02AF07EFE2E
S31508010A904FF0FF33082208A953482AF077FE514838
S31508010AA00122102127F0E2FBBDF81630524610212B
S31508010AB02046FFF76BFD84460028C4D11C9B6DB206
S31508010AC0002B00F08580002D079938DA8B7843F0E2
S31508010AD002038B70BBF1000F7CD0B84608EE104AB2
S31508010AE01C9FCDF808A081465D46BDF81620ADF8D5
S31508010AF0188006ABCDE9007918EE100AFFF7F8FD64
S31508010B00062801468446ABEB050E0DF11A033A4653
S31508010B10304632D0002996D13EB13468BDF8181056
S31508010B20D4F800A0ADF81AE0D047BDF81830ED1A90
S31508010B304345ADB250D3002D4ED00799D5E78878F5
S31508010B40BDF8162040F0010088701C9800903B46BD
S31508010B502046FFF793FA844600287FF474AF802174
S31508010B60BDF8163052462046FFF710FD844660460A
S31508010B700BB0BDEC028BBDE8F08FF82319488DF850
S31508010B8015300022102127F071FB4FF0FF330122A7
S31508010B900DF1150114482AF0F9FD4FF0FF33012232
S31508010BA00DF11A0110488DF81A902BF099F80122C7
S31508010BB010210C4827F05AFB9DF81A30079983F043
S31508010BC020038A78C3F3401363F341028A708CE7E2
S31508010BD0002DC4DAA021C3E718EE104ADDF808A0F3
S31508010BE0F8E700BF00100240ACB001202DE9F0473C
S31508010BF00446806888B000284FD00806A37347D4F6
S31508010C00072A45D8E07C002800F02582A07E002826
S31508010C1000F0258294F82100002800F0248294F837
S31508010C202800002800F0238294F82F00002800F0FD
S31508010C30228294F83600002800F0218294F83D00BB
S31508010C40002800F0208294F84400002800F01D8254
S31508010C5094F84B00002800F01A8294F852000028F4
S31508010C6000F0178294F85900002800F0148294F8CD
S31508010C706000B8B194F86700002800F00E8294F875
S31508010C806E00002800F00B8294F87500002867D0E2
S31508010C90D426304608B0BDE8F087D726304608B0D6
S31508010CA0BDE8F0870C2000295CD0C1F3020502F0EB
S31508010CB00702C0EBC00042EAC505204405F07F05DE
S31508010CC00573002DE4D0E27CAA4251D0A27EAA4245
S31508010CD000F0B18194F82120AA4200F0AE8194F87F
S31508010CE02820AA4200F0AB8194F82F20AA4200F0EE
S31508010CF0A88194F83620AA4200F0A58194F83D20EF
S31508010D00AA4200F0A28194F84420AA4200F09F81E9
S31508010D1094F84B20AA4200F09C8194F85220AA42EA
S31508010D2000F09B8194F85920AA4200F09A8194F820
S31508010D306020AA4200F0998194F86720AA4200F03F
S31508010D40988194F86E20AA4200F0978194F875204C
S31508010D50AA4200F09681D626304608B0BDE8F0874B
S31508010D600F20A0E7C0EBC000204401250573AAE7C0
S31508010D700122C2EBC202A118052700228B73204665
S31508010D80CDE90622CDE90422CDE9022201951346D1
S31508010D9011460097FFF734FE06464FF4967026F083
S31508010DA07FFA002E3FF475AFE37CAB4200F0798100
S31508010DB0A37EAB4200F0778194F82130AB4200F074
S31508010DC0748194F82830AB4200F0718194F82F3081
S31508010DD0AB4232D094F83630AB4200F06A8194F8CF
S31508010DE03D30AB4200F0678194F84430AB4200F0E5
S31508010DF0648194F84B30AB4200F0618194F852302B
S31508010E00AB4200F05E8194F85930AB4200F05B8149
S31508010E1094F86030AB4200F0588194F86730AB42E1
S31508010E2000F0558194F86E30AB4200F0528194F887
S31508010E307530AB427FF42DAF0F27C7EBC7032344A9
S31508010E404FEAC70A1B7B03F007085B0640F1E280FD
S31508010E5001254FF00809A9EB050323441B7BC3F3BE
S31508010E60C203434500F0E2806B1CDBB2102B00F095
S31508010E70CA80C3EBC30222444FEAC309127BC2F3F9
S31508010E80C202424500F0D180AB1CDBB2102B00F048
S31508010E90BA80C3EBC30222444FEAC309127BC2F3E9
S31508010EA0C202424500F0C180EB1CDBB2102B00F0F8
S31508010EB0AA80C3EBC30222444FEAC309127BC2F3D9
S31508010EC0C202424500F0B1802B1DDBB2102B00F0A7
S31508010ED09A80C3EBC30222444FEAC309127BC2F3C9
S31508010EE0C202424500F0A1806B1DDBB2102B00F057
S31508010EF08A80C3EBC30222444FEAC309127BC2F3B9
S31508010F00C202424500F09180AB1DDBB2102B7AD0AC
S31508010F10C3EBC30222444FEAC309127BC2F3C202DE
S31508010F20424500F08280EB1DDBB2102B6BD0C3EB80
S31508010F30C30222444FEAC309127BC2F3C2024245E5
S31508010F4073D005F10803DBB2102B5CD0C3EBC302E7
S31508010F5022444FEAC309127BC2F3C202424564D056
S31508010F6005F10903DBB2102B4DD0C3EBC3022244B2
S31508010F704FEAC309127BC2F3C202424555D005F1B5
S31508010F800A03DBB2102B3ED0C3EBC30222444FEA5D
S31508010F90C309127BC2F3C202424546D005F10B03CF
S31508010FA0DBB2102B2FD0C3EBC30222444FEAC3098D
S31508010FB0127BC2F3C202424537D005F10C03DBB2FC
S31508010FC0102B20D0C3EBC30222444FEAC309127B7C
S31508010FD0C2F3C202424528D005F10D03DBB2102B3C
S31508010FE011D0C3EBC30222444FEAC309127BC2F3F1
S31508010FF0C202424519D0022D05D094F87530C3F3C3
S31508011000C203434567D0E379434503D108F1FF3865
S3150801101084F80780AAEB0707274400230434012232
S31508011020BC607A733B73BB7333E61D46294620467B
S31508011030FEF7C4FA0FE702229BE6032299E6042289
S3150801104097E6052295E6062293E6072291E6082207
S315080110508FE609228DE6012025E60A2289E6022085
S3150801106021E60B2285E603201DE60C2281E60420F3
S3150801107019E60D227DE6052015E60E2279E60620FB
S3150801108011E60F2275E607200DE608200BE6092072
S3150801109009E60A2007E60B2005E60D2003E60E20E1
S315080110A001E60127C9E60227C7E60327C5E604279D
S315080110B0C3E60627C1E60727BFE60827BDE60927CF
S315080110C0BBE60A27B9E60B27B7E60C27B5E60D27CF
S315080110D0B3E60E27B1E60F254FF07809A6E700BF5C
S315080110E02DE9F04F85B0DFF830819DF838B0DFF88B
S315080110F02C91019000EB810617469A460024B06FA1
S3150801110003685D68454507D11D684D451BD1002516
S31508011110284605B0BDE8F08F5B4652463946A847D2
S31508011120E02805461ED137B307F11E030199374A50
S3150801113051F8230003685B69934237D1B06F03689E
S315080111401D684D45E3D05B4652463946A8470D28EA
S31508011150054630D1E3B2022B2FD8642026F0A0F839
S315080111600134CCE70D284ED1E3B2022BF5D9284636
S3150801117005B0BDE8F08F26483A46102127F076F8E3
S315080111804FF4F5754FF0FF33022203A92148ADF854
S315080111900C502AF0FBFA1E480122102127F066F8A6
S315080111A0662026F07DF8B06F0368ADE7514698478B
S315080111B0B06F0368A8E70028A9D05FB1019B134A5D
S315080111C01E3753F8270003685B699342A0D051463E
S315080111D098479DE73A460E48102127F047F84FF4FD
S315080111E0F5744FF0FF3303A902220A48ADF80C4003
S315080111F02AF0CCFA06480122102127F037F8662092
S3150801120026F04EF884E7002898D081E721C1000826
S3150801121000100240ACB001201DC1000885F4000889
S315080112202DE9F04F2DED068B93B01D4609930DF16F
S31508011230300E002385730DF1340C856807930F462C
S31508011240C0F808E019460393019316461A46062381
S315080112501224CDF818C000934FF0010C4FF4006327
S31508011260CDE90444ADF83030CDF808C03C248023DC
S3150801127080468DF83240FFF7C3FBC8F808500028AE
S315080112805FD1BDF83C30DFF8A0A1DFF8A0B109EEC7
S31508011290903ABDF83E300AEE103A9DF838300B9375
S315080112A09DF83930B94608EE106A08F1740608EE59
S315080112B0907A34460A9609EE103A054608F1B407BB
S315080112C04E460FE0136A5B451ED1936954498B421A
S315080112D025D1D369534A934240F08780A74205F145
S315080112E0010533D054F8040F5FFA85F90028F5D0C3
S315080112F0026813695345E5D098470028EED120685E
S315080113000268136A5B45E0D019EE101A984700285F
S31508011310E4D020684249026893698B42D9D01AEE13
S31508011320102A19EE901A9847002875D0099B009340
S31508011330494618EE103A32464046FFF7D1FED12803
S31508011340CCD013B0BDEC068BBDE8F08F0A9EDFF852
S31508011350D890DFF8D8A0DFF8C8B0002403E0B74278
S3150801136004F1010446D056F8040FE5B20028F6D078
S31508011370026813694B451CD1136A534521D19369F8
S315080113805B4528D1D369274A934240D1099B0093EB
S3150801139018EE902A18EE103A29464046FFF7A0FEA5
S315080113A000F0F703D12BDAD013B0BDEC068BBDE8FC
S315080113B0F08F98470028D2D130680268136A5345DE
S315080113C0DDD019EE101A98470028DFD03068026878
S315080113D093695B45D6D01AEE102A19EE901A9847EA
S315080113E00028BCD130680268CCE70B9998470028D9
S315080113F09CD173E7099B18EE102A18EE901A4046FD
S31508011400FFF7F4FB13B0BDEC068BBDE8F08F0B9923
S3150801141098470028A3D1B9E72068026859E700BFB1
S3150801142095F4000825C1000891F4000829C10008AF
S315080114302DE9F04F89B004AD1C46009505AB002592
S31508011440129F059506469046ADF81050FEF7B4FC76
S3150801145010B109B0BDE8F08F0246424B4248ADF8DB
S315080114601C2010210693ADF81E40222526F0FEFE0B
S315080114700DF112014FF0FF3301223C488DF812504D
S315080114802AF084F94FF0FF33082206A937482AF0D3
S315080114907DF935480122102126F0E8FEBDF8103005
S315080114A0424610213046FFF771F80028D1D11FB303
S315080114B005998B7843F002038B70ECB1DFF8A8B07D
S315080114C0DFF8A8A081462546CDE90079BDF81020A8
S315080114D0ADF812400DF112033046FFF709F9062857
S315080114E014D00028B5D1BDF81230ED1A9C42ADB220
S315080114F002D80DB10599E7E7BDF8103042463046E6
S31508011500A021FFF743F809B0BDE8F08FF8230022C0
S31508011510102158468DF80E3026F0A8FE4FF0FF33FD
S3150801152001220DF10E0150462AF030F94FF0FF3332
S3150801153001220DF10F0150468DF80F902AF0D0FBCC
S3150801154001221021584626F091FE05999DF80F3083
S315080115508A7883F02003C3F3401363F341028A7048
S31508011560B2E700BF8006000100100240ACB00120BE
S315080115702DE9F04F9FB00AAC0025984600940BABB5
S315080115800B95044689461646ADF82850FEF714FC15
S3150801159010B11FB0BDE8F08F02464FF4D06700F1D5
S315080115A080404FF410230225102100F50430ADF8D0
S315080115B030700EAF8DF833500D938DF83280222599
S315080115C026F054FE39464FF0FF33012243488DF881
S315080115D038502AF0DBF84FF0FF3308220CA93F48B0
S315080115E02AF0D4F83E480122102126F03FFEBDF824
S315080115F02830324610212046FEF7C8FF0028C8D1F8
S315080116000B998B78092543F002038B70AB464FF093
S31508011610000ACDE9007ABDF82820ADF82AB00DF107
S315080116202A032046FFF764F806282CD00028B0D1F3
S31508011630BDF82A30ED1A082BADB202D90DB10B99B6
S31508011640E5E7BDF828303246A0212046FEF79EFF81
S3150801165000289ED1289B0390CDE90673BDF83A7000
S31508011660CDF804804FF0400C022506230093CDE9FE
S31508011670047C32464946204602958023FFF7C0F985
S315080116801FB0BDE8F08FF82315488DF8263052466D
S31508011690102126F0EBFD4FF0FF3301220DF1260153
S315080116A00E482AF073F84FF0FF3301220DF1270196
S315080116B00A488DF827A02AF013FB012210210848B1
S315080116C026F0D4FD0B999DF827308A7883F02003FC
S315080116D0C3F3401363F341028A7098E7ACB0012063
S315080116E000100240F0B587B00DF10A0400941F46B8
S315080116F0002403AB0394ADF80A4006461546FEF7E7
S315080117005BFB044630B14FF4967025F0C9FD2046BF
S3150801171007B0F0BD02464FF4A0631D488DF813408B
S3150801172010210594ADF8103022248DF8127026F098
S315080117309DFD4FF0FF3301220DF1090115488DF882
S3150801174009402AF023F84FF0FF33082204A911486B
S315080117502AF01CF80E480122102126F087FDBDF853
S315080117600A302A4610213046FEF710FF04460028A3
S31508011770C9D1BDF80A302A4680213046FEF706FF50
S3150801178004464FF4967025F08BFD204607B0F0BD50
S3150801179000100240ACB00120F0B587B00DF10A0483
S315080117A000941F46002403AB154606460394ADF87C
S315080117B00A40FEF701FB024610B1104607B0F0BD1C
S315080117C04FF410631B488DF8132010210592ADF8CC
S315080117D010308DF81270222426F048FD4FF0FF33A1
S315080117E001220DF1090114488DF8094029F0CEFFAF
S315080117F04FF0FF33082204A90F4829F0C7FF0D4807
S315080118000122102126F032FD2A46BDF80A301021A0
S315080118103046FEF7BBFE02460028CED12A46BDF861
S315080118200A3030468021FEF7B1FE0246104607B05F
S31508011830F0BD00BF00100240ACB0012030B583B046
S31508011840F82362488DF803300022102126F00EFD98
S315080118500DF103014FF0FF3301225D4829F096FF90
S31508011860002501A94FF0FF33012259488DF804508C
S315080118702AF036FA55480122102126F0F7FC9DF880
S31508011880044004F0C004802C49D041D8002C00F053
S315080118908380402C3AD1D8234C488DF803302A4608
S315080118A0102126F0E3FC0DF103014FF0FF3301226D
S315080118B0474829F06BFF4FF0FF33012201A944483D
S315080118C08DF804502AF00CFA01224048102126F01E
S315080118D0CDFC9DF8042012F0020244D02A463B486A
S315080118E0102126F0C3FC4CF6DA144FF0FF3301A998
S315080118F002223748ADF8044029F048FF012233484F
S31508011900102126F0B3FC334B02221A7003B030BD06
S31508011910C02CFBD12F4B01221A7003B030BDD8233E
S315080119202A488DF803302A46102126F09FFC0DF12E
S3150801193003014FF0FF330122254829F027FF4FF015
S31508011940FF33012201A922488DF804502AF0C8F96B
S3150801195001221E48102126F089FC9DF8042012F068
S315080119600202BCD02A461948102126F07FFC4CF603
S31508011970DA3401A94FF0FF3302221548ADF80440C5
S3150801198029F004FF11480122102126F06FFC114BA2
S3150801199003221A7003B030BD22460C48102126F0E6
S315080119A065FC4DF2DA1501A94FF0FF33022208480A
S315080119B0ADF8045029F0EAFE04480122102126F068
S315080119C055FC044B1C7003B030BD00BF001002402B
S315080119D0ACB00120900F002070B54FF4005182B0D1
S315080119E004466D4826F03CFC002800F0BA816B4B92
S315080119F01B78032B00F2C482DFE803F0C3BEBC02E6
S31508011A000126674D2B7803F0F003102B00F08B822B
S31508011A10A06F28B10368634ADB68934240F06B8282
S31508011A20E06F28B103685F4ADB68934240F0618240
S31508011A30D4F8800028B103685A4ADB68934240F01B
S31508011A405682D4F8840028B10368564ADB68934263
S31508011A5040F04B82D4F8880028B10368514ADB6804
S31508011A60934240F04082D4F88C0028B103684D4A6D
S31508011A70DB68934240F03582D4F8900028B10368B8
S31508011A80484ADB68934240F02A82D4F8940028B188
S31508011A900368444ADB68934240F01F82D4F89800F1
S31508011AA028B103683F4ADB68934240F01482D4F8B0
S31508011AB09C0028B103683B4ADB68934240F00982DF
S31508011AC0D4F8A00028B10368364ADB68934240F08F
S31508011AD0FE81D4F8A40028B10368324ADB68934230
S31508011AE040F0F381D4F8A80028B103682D4ADB68D1
S31508011AF0934240F0E881D4F8AC0028B10368294A3A
S31508011B00DB68934240F0DD81D4F8B00028B1036860
S31508011B10244ADB68934240F0D281D4F8B40028B154
S31508011B200368204ADB68934240F064812B78402B96
S31508011B3000F0658100F2D380202B00F0E981302B7B
S31508011B4036D119480022102126F090FB4FF4F5747E
S31508011B504FF0FF33022201A91448ADF8044029F0D9
S31508011B6015FE11480122102126F080FB40232B7017
S31508011B7002B070BD002644E7094D13232B700026D9
S31508011B8046E7074D2B7803F0F003102B00F0288168
S31508011B9011232B7000263BE700080240900F002016
S31508011BA0910F00208DF4000800100240ACB001200E
S31508011BB0112BDDD1A06F002384F8B83028B1036852
S31508011BC0884A9B68934240F0D981E06F28B103683F
S31508011BD0844A9B68934240F0CF81D4F8800028B1AB
S31508011BE00368804A9B68934240F0C481D4F8840014
S31508011BF028B103687B4A9B68934240F0B981D4F8BF
S31508011C00880028B10368774A9B68934240F0AE8101
S31508011C10D4F88C0028B10368724A9B68934240F055
S31508011C20A381D4F8900028B103686E4A9B68934251
S31508011C3040F09881D4F8940028B10368694A9B68F2
S31508011C40934240F08D81D4F8980028B10368654A1B
S31508011C509B68934240F08281D4F89C0028B10368BE
S31508011C60604A9B68934240F07781D4F8A00028B176
S31508011C7003685C4A9B68934240F06C81D4F8A400DF
S31508011C8028B10368574A9B68934240F06181D4F8AA
S31508011C90A80028B10368534A9B68934240F05681CD
S31508011CA0D4F8AC0028B103684E4A9B68934240F0C9
S31508011CB04B81D4F8B00028B103684A4A9B6893421D
S31508011CC040F04081D4F8B40028B10368454A9B68BE
S31508011CD0934240F0358112232B7002B070BD512B0F
S31508011CE000F00B81802B0DD1002233462046114688
S31508011CF0FFF796FA002870D0D2283FF439AFA0230F
S31508011D002B7035E7502B7FF433AFC82336488DF84F
S31508011D1004300022102126F0A9FA4FF0FF330122E0
S31508011D2001A9324829F032FD00244FF0FF33012280
S31508011D300DF103012D488DF8034029F0D1FF2A48FA
S31508011D400122102126F092FA9DF803305B067FF5F1
S31508011D500FAF51232B7025F09DFA254B14301860CF
S31508011D6006E70546C823024610211F488DF80230AA
S31508011D7026F07CFA4FF0FF3301220DF102011B48D0
S31508011D8029F004FD4FF0FF3301A9012217488DF808
S31508011D90045029F0A5FF14480122102126F066FAFD
S31508011DA09DF8043013F0200540F0C5800E48002246
S31508011DB0102126F05BFACA2601A94FF0FF33022249
S31508011DC00A488DF805508DF8046029F0DFFC0648AD
S31508011DD00122102126F04AFA09E690232B70C7E65C
S31508011DE0002615E689F4000800100240ACB001206F
S31508011DF0940F002098472B78402B7FF49BAEE8235D
S31508011E0061488DF803300022102126F02FFA0DF1D2
S31508011E1003014FF0FF3301225C4829F0B7FC002487
S31508011E204FF0FF3301A9012258488DF8044029F0E3
S31508011E3057FF55480122102126F018FA9DF804305B
S31508011E4013F001047FF494AED82322464E488DF848
S31508011E500330102126F00AFA0DF103014FF0FF3382
S31508011E6001224A4829F092FC4FF0FF33012201A9C9
S31508011E7046488DF8044029F033FF434801221021D2
S31508011E8026F0F4F99DF804603F482246102126F011
S31508011E90EDF946F008064FF0FF3301A902223B4847
S31508011EA08DF80560DA248DF8044029F06FFC364870
S31508011EB00122102126F0DAF950232B7058E69847AB
S31508011EC02BE6984720E6984715E698470AE6984785
S31508011ED0FFE59847F4E59847E9E59847DEE5984729
S31508011EE0D3E59847C8E59847BDE59847B2E59847C9
S31508011EF0A7E598479CE5984792E525F0CBF9244B49
S31508011F001B68C01A0028FFF633AE80232B70EBE658
S31508011F1025F0C0F91E4B1B68C01A0028FFF628AE2B
S31508011F2030232B700DE625F0B5F9194AC830202360
S31508011F3010602B706CE52046FFF780FC202535E7FD
S31508011F409847C8E69847BDE69847B2E69847A7E690
S31508011F5098479CE6984791E6984786E698477BE630
S31508011F60984770E6984765E698475AE698474FE6D0
S31508011F70984744E6984739E698472EE6984724E66F
S31508011F80044D002644E500BF00100240ACB0012014
S31508011F90940F0020910F00200368FBB170B40479F7
S31508011FA0A4B11388BBB143790E68056836781B1B43
S31508011FB0EE540379013B037113880C68013B013424
S31508011FC09BB213800C600479002CEBD14379037121
S31508011FD070BC01207047002070BC70470020704714
S31508011FE000B583B0481EADF8062007280DD8DFE8EE
S31508011FF000F02B04424C5A10101DBDF8062002B100
S3150801200001223348202126F031F9012003B05DF879
S3150801201004FB3049BDF80620086819464FF47A735F
S3150801202029F0B4FB012003B05DF804FB2949BDF88A
S3150801203006200868194629F05FFF012025F030F9C6
S31508012040012003B05DF804FB00221021204826F088
S315080120500DF9022025F024F91D480122102126F048
S3150801206005F91D4801224FF4004126F0FFF8012029
S3150801207003B05DF804FBBDF806300BBB1648012218
S315080120804FF4004126F0F2F8BFE7BDF8062002B189
S31508012090012210210E4826F0E9F827F0ABFC0120B1
S315080120A003B05DF804FB0B4A4FF47A7310680DF11F
S315080120B00601012229F06AFB012003B05DF804FB41
S315080120C0054800224FF4004126F0D0F89DE700BFED
S315080120D000040240980F00200000024025F0E0B8F5
S315080120E010B5094B044601224FF4004107481C600C
S315080120F026F0BCF80A2025F0D3F8BDE81040044ABA
S315080121000449054800F0B6BC980F002000000240BB
S31508012110E11F0108000000202CAE01202DE9F04F37
S3150801212087B08146BDF840A0CDF800A0119E0D46A6
S3150801213014461F4600F0B2F800287BD0BAF1000F0A
S3150801214078D0A7F108039AB2C3F3CC0305F10F01BE
S31508012150013322F00702A24407350493531807F105
S31508012160070B1FFA8AF00593ABB202900393CBF3E0
S31508012170CC0B072F70D9049B039D06EB030AB046C7
S3150801218018F8013B0093294602232246484600F0E7
S3150801219033FD0835D045ADB2F2D1BDF8148007F04C
S315080121A00705002D40D09AF800A0A8F107011AF0FA
S315080121B0010F89B241D1A8F10601012D89B24FEA71
S315080121C05A0331D0DA073DD4A8F10501022D89B2A7
S315080121D04FEA9A0328D0DB0739D4A8F10401032D65
S315080121E089B24FEADA031FD0D8073AD4A8F1030116
S315080121F0042D89B24FEA1A1316D0DA0736D4053DEB
S31508012200A8F10201ADB289B24FEA5A1365B1DB07EB
S3150801221031D408F1FF38012D1FFA88F14FEA9A1ACD
S3150801222002D01AF0010F2BD1029B0134A4B29C42B1
S315080122305E449ED107B0BDE8F08F2246484600F0BD
S31508012240CFFCB8E72246484600F0CAFCBCE722465E
S31508012250484600F0C5FCC0E7DDF80C803D46B246AD
S315080122609FE72246484600F0BBFCBFE722464846A0
S3150801227000F0B6FCC3E72246484600F0B1FCC8E7C1
S315080122802246484600F0ACFCCEE700BF10B4BDF8C4
S31508012290044001945DF8044BFFF740BF70B4BDF8E4
S315080122A00C40B0F84260C58F013C14449642A4B272
S315080122B018D3A54201D9A24211D9B0F84040828F5C
S315080122C0013B0B448C429BB207D39A420FD99942E0
S315080122D094BF0020012070BC70479A42F7D90020AC
S315080122E070BC7047A542FAD8A242F8D9E5E70120A1
S315080122F0F6E700BF10B48C680023A44601215DF8F7
S31508012300044B604710B48C680023A44603215DF88A
S31508012310044B604710B48C680023A44602215DF87B
S31508012320044B604710B48C680023A44605215DF868
S31508012330044B60472DE9F0411446127880460E4653
S31508012340FF2A0AD0B568002305214046A84700B3ED
S315080123506278FF2A04F10104F4D16578FF2D0FD0C4
S31508012360FE2D4AD0EF2D11D8DF2D15D905F00F0214
S315080123700023B56802214046A84702342278DFE7E0
S31508012380B568002305214046A84710B1A278023452
S31508012390D6E70020BDE8F081CF2D09D905F00F0257
S315080123A00023B56803214046A84702342278C7E7C7
S315080123B0BF2D18D92D01002302351A460421B76805
S315080123C005F0FE054046B8472846FFF787FE012275
S315080123D000230421B7684046B8472846FFF77EFE22
S315080123E002342278ACE7BD2DD0D82B06CED42846A8
S315080123F0FFF774FE02342278A2E70120BDE8F081D6
S31508012400013AF8B51FFA82FE0EF1010E0E4F0F4E74
S315080124109E44002213F8014B04F00F0C551C2409A5
S3150801242016F80CC007F802C0ADB2345D7C5502320D
S31508012430734592B2EED18C68034B4FF48062082142
S31508012440A0470120F8BD00BF9C0F00200C9F04087F
S31508012450013AF8B55FFA82FE0EF1010E0D4F0E4EE6
S315080124609E44002213F8014B04F00F0C551C240955
S3150801247016F80CC007F802C0EDB2345D7C5502327D
S315080124807345D2B2EED18C68024B80220621A04751
S315080124900120F8BD9C1300200C9F040801207047F9
S315080124A02DE9F04F85B017460A3A04468846019346
S315080124B00C2A58D8DFE802F0605757575769888FB2
S315080124C05757579607004B68B3F80A901A88D3F8F6
S315080124D00CA04FEA49091FFA89F9002A43D0029745
S315080124E0DFF8ACB15746184600269A4602E0D8F8F6
S315080124F004000288057A02FB056505F0FF055A46C0
S3150801250041462046FFF716FF2A4641462046FFF771
S3150801251009FF05F10802D2B241462046FFF702FF3C
S31508012520002241462046FFF7F5FE5C224146204639
S31508012530FFF7F8FE012241462046FFF7EBFE3B4630
S315080125404A4641462046FFF75BFF002241462046A0
S31508012550FFF7D8FE0836BAF80010F2B291424F4496
S315080125601646C4D8029F019B3A464146204605B005
S31508012570BDE8F04F00F054BC0222FFF7BBFE414A0A
S3150801258041462046FFF7D6FEEDE70122FFF7BAFEE0
S31508012590414620460022FFF7BDFE4146C12220469C
S315080125A0FFF7C0FE414620460122FFF7B3FE019B15
S315080125B01A78414652082046FFF7B4FE00224146E2
S315080125C02046FFF79FFECEE72F4AFFF7B3FE01200D
S315080125D005B0BDE8F08F2D4AFFF7ACFE012005B026
S315080125E0BDE8F08F4B6858891A88D3F80C90810892
S315080125F00291002AB7D00397DFF894B04F465FFAE5
S3150801260081FA18460026994602E0D8F8040002889D
S31508012610057A02FB056505F0FF055A46414620463F
S31508012620FFF788FE2A4641462046FFF77BFE6A1CCD
S31508012630D2B241462046FFF775FE002241462046A2
S31508012640FFF768FE5C2241462046FFF76BFE012232
S3150801265041462046FFF75EFE3B4652464146204626
S31508012660FFF7F6FE002241462046FFF74BFE0136EC
S31508012670B9F80010029BF2B291421F441646C4D81B
S31508012680039F70E71C9F0408B89F0408AC9F0408C1
S315080126909C9F04084218435C507800EB032080B2E3
S315080126A0704700BF0020704790F92900013080B2B9
S315080126B0704700BF704700BF08B5FFF7FBFF10F072
S315080126C0FD0F14BF0320062008BD00BF0621FFF732
S315080126D0E1BF00BF0821FFF7DDBF00BF807A704761
S315080126E0C07A70472DE9F84FD0F808B09BF800A0DA
S315080126F0054650468946FFF7DDFF01280746584635
S3150801270014BFFF260F26FFF7E9FF04465846FFF7D1
S31508012710E7FF60298046584630D9FFF7DBFF28B323
S315080127200BEB00026124C84519D3444517D8504616
S31508012730FFF7C2FF0AE04C4528D09378334003449B
S3150801274044451A4404F1010409D0E4B21378FF2B75
S31508012750F1D1444502F1010204F10104F5D1002247
S31508012760EA6185F820201046BDE8F88F5846FFF73C
S31508012770ADFF40B10BEB00024124D4E7FFF7A6FFFA
S31508012780B9F1400FF5D80BF11102CCE717F0FD0F9F
S3150801279012D003F00F0102391B09A9776B77537819
S315080127A003F00F011B0985F82010EB7793781B09B5
S315080127B02B771046BDE8F88FEB77537885F82030EC
S315080127C0D3782B7713796B775379AB771046BDE8B6
S315080127D0F88F00BF2DE9F04F8A4685B01946914614
S315080127E00646FFF77FFF044600284CD096F820706E
S315080127F096F91E2096F91D30B168F57F91F800808B
S3150801280000973A44A9EB02029A441FFA82FB1FFA7F
S315080128108AFA5A4651462B463046FFF73FFD80B3A2
S31508012820E91DC1F3C40167B34046FFF745FF251803
S3150801283039B37B1E01F1FF38DBB25FFA88F8013341
S3150801284008F101085B4405EB08099BB203934F465F
S31508012850544615F8013B0093214600235A46304653
S3150801286000F0CAF90834BD42A4B2F2D1039B0BF1B8
S31508012870010B1FFA8BFB9B4547444D4601D0C144CA
S31508012880E6E796F91C0005B0BDE8F08F2DE9F041A1
S315080128901D46436A904607460C4698472B7840449E
S315080128A09BB11FFA80F80026214642463846FFF7B3
S315080128B091FF15F8013F80B204443044A4B286B2B0
S315080128C0002BF1D13046BDE8F0811E463046BDE801
S315080128D0F08100BF8268002380F828309AB192F906
S315080128E0053080F8293092F90C1090F82B2080F8E1
S315080128F02A105B1A402A9BB203D0DBB202FB03F310
S315080129009B0980F82C3070478268012380F82830AB
S315080129109AB192F90F3080F8293092F9101090F88F
S315080129202B2080F82A105B1A402A9BB203D0DBB20F
S3150801293002FB03F39B0980F82C307047014B436275
S31508012940704700BFA5260108014B4362704700BFC7
S31508012950A926010870B50D46097871B10646002405
S315080129603046FFF7BFFE96F91C3015F8011F1C44C7
S31508012970A4B20029F4D1204670BD0C46204670BD8C
S3150801298083688B421AD08160B1B190F82830B3B907
S3150801299091F9053080F8293091F90C1080F82A1040
S315080129A090F82B205B1A402A9BB203D0DBB202FBBC
S315080129B003F39B0980F82C300B4B43627047012BBC
S315080129C008D091F90D3080F8293091F90E1080F868
S315080129D02A10E5E791F90F3080F8293091F910109E
S315080129E080F82A10DCE700BFA526010810B40C6898
S315080129F0A4465DF8044B604710B582B00C680DF12A
S31508012A0006034622A047BDF8060002B010BD00BF66
S31508012A1010B582B00C680DF106034722A047BDF830
S31508012A20060002B010BD00BF30B54168044683B048
S31508012A300D680DF106034622A8476168BDF8063000
S31508012A400D68238020460DF106034722A8476168D1
S31508012A50BDF806300D686380204600234822A84742
S31508012A606168E0740D6804F13C0320461722A84703
S31508012A7003B030BD2DE9F041222300254FF00108AE
S31508012A8004460E468374C0E902558561A0F8108094
S31508012A9080F834801746FFF751FF104A104B6660DD
S31508012AA0A262A36384F82C500220B76000F05CFC94
S31508012AB0314637682B460A222046B847A36B064695
S31508012AC003209847A36B284698471EB12046FFF76F
S31508012AD0ABFF46463046BDE8F08100BF0100004025
S31508012AE06933010870B5044602206568A36B9847E7
S31508012AF0A36B012098472E682946204600231422F5
S31508012B00B04704F13C032E68294620461722B047F0
S31508012B10A36B0020BDE87040184700BFF8B583696C
S31508012B20044603B198476668A36B02209847A36BCE
S31508012B300120984735683146002315222046A847C3
S31508012B40054630B13768314604F13C031722204661
S31508012B50B847A36B002098472846F8BDF8B583699E
S31508012B60044603B198476668A36B02209847A36B8E
S31508012B700120984735683146002316222046A84782
S31508012B80054630B13768314604F13C031722204621
S31508012B90B847A36B002098472846F8BD10B582B000
S31508012BA043688DF807101C6819460F220DF10703B3
S31508012BB0A04702B010BD00BF416810B40C680023DD
S31508012BC0A44610225DF8044B604700BF416810B463
S31508012BD00C680023A44611225DF8044B604700BF28
S31508012BE030B44468C1852568028603462146AC4649
S31508012BF02E3330BC3222604770B445689DF80C60AC
S31508012C0080F8333080F832602C68C18502862946FF
S31508012C10A44600F12E0370BC3B22604780F83410AD
S31508012C20704700BFC37C302B08D0282B0AD0022B53
S31508012C3014BF0123032380F8343070474FF6FF731E
S31508012C4083867047FF23F6E703880022013B8280CB
S31508012C50C3800272704700BF838802884188134483
S31508012C609BB28B42838012D210B4C488037A224461
S31508012C7092B2914298BF01F1FF3203F10103037247
S31508012C8098BF92B2C2805DF8044B012070470020BC
S31508012C90704700BF4389C28810B4013B84884C80C1
S31508012CA000205DF8044B08808B80CA80704700BFFE
S31508012CB030B44B794A88012B1ED0032B19D1A2F1C6
S31508012CC008039BB29A4214462CBF002101211A46D9
S31508012CD0C3888588934234BF0023012343EA010050
S31508012CE0A5428CBF002000F001000B40184330BC00
S31508012CF0704714460021EBE702F10804A4B2A24288
S31508012D0094BF00210121E3E730B485884489C0686E
S31508012D10521BA408D2B29DF8085012FB04F28C0883
S31508012D20490014FA82F201F0060145B1845C03F008
S31508012D30030303FA01F12143815430BC704703258B
S31508012D40845C8D40EDB224EA0504F0E7F0B50C7910
S31508012D5083B00D460646002723061BD46B79032B41
S31508012D6006D8DFE803F0130B0F026B88013B6B8073
S31508012D70640014F0FF04EFD103B0F0BD6B88013392
S31508012D806B80F5E72B88013B2B80F1E72B88013314
S31508012D902B80EDE76A88B3889342DFD8F38893429C
S31508012DA0DCD3298873898B42D8D90097AB79304609
S31508012DB0FFF7AAFFD2E700BFF0B50C7983B00D463D
S31508012DC006460127A309AB71B1886A8891420AD8D8
S31508012DD0F188914207D3708929888842304602D9F9
S31508012DE00097FFF791FF6B79032B06D8DFE803F00D
S31508012DF00F130B026B88013B6B80A40014F0FF04D0
S31508012E00E0D103B0F0BD2B88013B2B80F5E72B8879
S31508012E1001332B80F1E76B8801336B80EDE700BF47
S31508012E2030B5143A4D6885B0342A27D8DFE802F060
S31508012E30451B1B2926262626262626262626262617
S31508012E4026262626262626266149262626264E268D
S31508012E50262626262626262F2626262626262626FA
S31508012E6026263D4176002846FFF7F6FE002853D070
S31508012E706A89E8685200002132F098F8012005B005
S31508012E8030BD28461946FFF705FF0120F7E7194621
S31508012E9028460393FFF70CFF039B0028EED028462C
S31508012EA01946FFF753FF0120E9E76A891A800120CD
S31508012EB0E5E76A881A800120E1E72846FFF7C4FE9C
S31508012EC0D6E719462846FFF777FFD7E75A88A9882C
S31508012ED09142D3D8E9889142D0D319886889884222
S31508012EE0CCD900209B7900902846FFF70DFF0120D9
S31508012EF0C5E75A88A9889142C0D8E9889142BDD3C5
S31508012F00198868898842B9D901249B790094284689
S31508012F10FFF7FAFE2046B2E70020B0E70220AEE747
S31508012F202DE9F04F87B00746BDF8405000950C468D
S31508012F3090461E46FFF7B2F910B907B0BDE8F08F03
S31508012F40072E40F2E980A6F1080A2AF0070A0AF1D3
S31508012F50080AA2441FFA8AFAA1464FF0FF0B49460E
S31508012F6009F10809CDF800B00023424638461FFA90
S31508012F7089F9FFF741FED145F1D106F00703002B88
S31508012F8040F08B80072D40F2AA80A5F1080323F0B3
S31508012F90070AC2441FFA8AFA03930AF108039BB285
S31508012FA00593C1464FF0FF0B01234A46CDF800B001
S31508012FB021463846FFF720FE4B46534509F10809D5
S31508012FC01FFA89F9F0D105F00703049315F00703F1
S31508012FD074D1039B23F00709C1441FFA89F9711EAD
S31508012FE009F1080321449BB289B20593C2464FF001
S31508012FF0FF0B01235246CDF800B038460391FFF77F
S31508013000FBFD53464B450AF1080A03991FFA8AFA4A
S31508013010EFD1BDF8103073B183F007030133FF22F6
S3150801302003F0070302FA03F3DBB20093059A0123BF
S315080130303846FFF7E1FD013DA844072E1FFA88F837
S3150801304065D9A6F1080929F0070909F10809A14472
S315080130501FFA89F9FF2521460834009500234246BF
S315080130603846A4B2FFF7C8FDA145F4D106F0070614
S31508013070002E3FF462AF86F00706731C03F00706BD
S31508013080FF23B340DBB21093424649463846002334
S3150801309007B0BDE8F04FFFF7AFBD83F00703013373
S315080130A0FF2203F0070302FA03F3DBB2009351464A
S315080130B0002342463846FFF79FFD63E783F007037F
S315080130C0013303F007030BFA03FB5FFA8BF3009353
S315080130D0059A012321463846FFF78EFD79E7002D2B
S315080130E0A9D085F00703013303F00702FF239340B4
S315080130F0DBB200932146012342463846FFF77CFDA1
S31508013100711E214489B22B46CDF8148083E7A14666
S31508013110002E3FF412AFAEE73346A2462FE700BFB3
S315080131202DE9F04F85B0A3F10806BDF838901F4682
S3150801313026F0070601F108031E4491448A461546FE
S31508013140B6B21FFA89F9072F2CD9B34654464FF060
S31508013150FF0821460834CDF8008000232A46A4B288
S315080131600390FFF749FDB4420398F2D107F007032C
S3150801317033B90135ADB24D45E5D105B0BDE8F08F9E
S3150801318083F007030133FF2203F0070302FA03F36F
S31508013190DBB20093594600232A460390FFF72CFD1C
S315080131A00398E6E73B46D346E2E700BF2DE9F0413F
S315080131B082B00446BDF82080CDF800800D4616463B
S315080131C01F46FFF76BF810B902B0BDE8F0813B4620
S315080131D0324629462046CDF8208002B0BDE8F041A6
S315080131E0FFF79EBF002070472DE9F041A2F11705B0
S315080131F0496882B0174606461C46302D1AD8DFE8BC
S3150801320005F066191919191919191919191919190F
S31508013210191919191919191F39191919191F1919E3
S3150801322019191919191939191919191919191919DF
S3150801323019585F00234602B0BDE8F041FFF7D6BB37
S315080132400191FFF7E5FB65880199ED430544304691
S31508013250FFF7D2FB23880199DB430344ADB22380F0
S3150801326065803A4630462346FFF7C0FB012002B087
S31508013270BDE8F0810191FFF7CBFB65880199ED4324
S3150801328005443046FFF7B8FB228863790199ADB248
S3150801329065800233D543054403F0030363713A4657
S315080132A0304625802346FFF7A1FB012002B0BDE881
S315080132B0F081FFF7A1FB2080012002B0BDE8F08173
S315080132C0FFF7A6FB2080012002B0BDE8F081234666
S315080132D017220191FFF78AFB01993046FFF78CFB0C
S315080132E0B4F8048001996FEA080880443046FFF76C
S315080132F083FB27880199FF4307443046FFF788FB7C
S31508013300E3880199DB43054630461D44FFF780FBF8
S315080133106388DB4318441FFA88F8BFB2ADB2E08070
S315080133200120A4F80080A780658002B0BDE8F0817D
S31508013330044942688A4200D0704752684260FFF7E2
S3150801334073BB00BF1C000020054B42689A4218BF98
S315080133505A60044A18BF43601A60FFF765BB00BF8D
S315080133601C000020E9310108704700BFF8B5084E76
S31508013370084F0223054633700A2400E038B10122BA
S31508013380294638462FF014F8013C3070F6D1F8BDBD
S315080133901C1600202016002070B5084E022305468B
S315080133A033700A2400E038B10122294600202EF0A4
S315080133B0FFFF013C3070F6D170BD00BF1C1600201E
S315080133C0024B312283F87820704700BF5418002039
S315080133D030B40F4D0F4C104A017040F6B8314561B3
S315080133E0846141F28835022401864263082100225C
S315080133F0C0E90E54C0E9032230BCC0E90722C0E97E
S315080134000922A0F84010427042804260C2627047A9
S31508013410006CCA8800943577801A0600F0B52F4BE0
S315080134202F4E304F044693E8030087B0C823009017
S315080134308DF80410052269462B4828F0A7F9237848
S315080134402A4836F81310012224F010FF2378284859
S3150801345037F81310012224F009FF0A2023F020FF70
S315080134602578A1230022042D02938DF80C2010D86B
S3150801347036F815101D4824F0F9FE052202A91A4846
S31508013480C82328F083F936F815101848012224F0C4
S31508013490EDFE0A2023F004FF2578AD230022042D32
S315080134A004938DF8142011D836F815100F4824F016
S315080134B0DDFEC823052204A90B4828F067F936F86A
S315080134C015100A48012224F0D1FE257837F815107F
S315080134D00748002224F0CAFE07B0F0BD78DF0408C9
S315080134E09C070020A407002004B10120000C02401B
S315080134F00008024030B56A4B024693E8030091B0D2
S31508013500147800908DF80410D3E9060102908DF81D
S315080135100C10D3E9080104908DF81410D3E90201BF
S3150801352006908DF81C10D3E90A0108908DF824102D
S31508013530D3E90C010A908DF82C10D3E90E010C90F1
S315080135408DF83410D3E91001042C0E908DF83C1037
S3150801355000F2A380534D544835F81410002224F084
S3150801356085FEC82369460522504828F00FF935F823
S3150801357014104D48012224F079FE35F814104A48F2
S31508013580002224F073FEC82369460522474828F01D
S31508013590FDF835F814104448012224F067FE35F881
S315080135A014104148002224F061FEC823052202A90D
S315080135B03E4828F0EBF835F814103B48012224F070
S315080135C055FE35F814103848002224F04FFEC8235A
S315080135D0052204A9354828F0D9F835F814103248D7
S315080135E0012224F043FE35F814102F48002224F056
S315080135F03DFEC823052206A92C4828F0C7F835F848
S3150801360014102948012224F031FE35F814102648F1
S31508013610002224F02BFEC823052208A9234828F0F6
S31508013620B5F835F814102048012224F01FFE35F8A4
S3150801363014101D48002224F019FEC82305220AA9E0
S315080136401A4828F0A3F835F814101748012224F06F
S315080136500DFE35F814101448002224F007FEC8237D
S3150801366005220CA9114828F091F835F814100E48CE
S31508013670012224F0FBFD35F814100B48002224F032
S31508013680F5FD05220EA90948C82328F07FF835F863
S3150801369014100548012224F0E9FD11B030BD00BF20
S315080136A0B89504089C070020000C024004B10120CB
S315080136B030B5474B024693E803008BB01478009067
S315080136C08DF80410D3E902018DF80C100290D3E9A4
S315080136D01A018DF814100490D3E906018DF81C100F
S315080136E00690D3E91C01042C8DF8241008906CD897
S315080136F0384D394835F81410002224F0B7FDC8238F
S3150801370069460522354828F041F835F8141032483B
S31508013710012224F0ABFD35F814102F48002224F0BD
S31508013720A5FDC823694605222C4828F02FF835F847
S3150801373014102948012224F099FD35F81410264859
S31508013740002224F093FDC823052202A9234828F064
S315080137501DF835F814102048012224F087FD35F8A4
S3150801376014101D48002224F081FDC823052204A94E
S315080137701A4828F00BF835F814101748012224F0D6
S3150801378075FD35F814101448002224F06FFDC8237E
S31508013790052206A9114827F0F9FF35F814100E4835
S315080137A0012224F063FD35F814100B48002224F099
S315080137B05DFD052208A90948C82327F0E7FF35F862
S315080137C014100548012224F051FD0BB030BD00BF8D
S315080137D0989504089C070020000C024004B10120BA
S315080137E030B5304B024693E8030087B01478009051
S315080137F08DF80410D3E91E018DF80C100290D3E957
S315080138002001042C8DF81410049048D8264D274819
S3150801381035F81410002224F029FDC823694605222B
S31508013820234827F0B3FF35F814102048012224F065
S315080138301DFD35F814101D48002224F017FDC82374
S31508013840694605221A4827F0A1FF35F814101748CA
S31508013850012224F00BFD35F814101448002224F037
S3150801386005FDC823052202A9114827F08FFF35F85F
S3150801387014100E48012224F0F9FC35F814100B48EF
S31508013880002224F0F3FC052204A90948C82327F0DD
S315080138907DFF35F814100548012224F0E7FC07B02E
S315080138A030BD00BF989504089C070020000C024013
S315080138B004B1012030B583B004788DF804100816D8
S315080138C00A14AD230912032C8DF801008DF8022084
S315080138D08DF803108DF8003013DC0B4D0B4835F8C5
S315080138E01410002224F0C2FC0522694608484FF448
S315080138F07A7327F04BFF35F814100448012224F097
S31508013900B5FC03B030BD00BF9C070020000C024087
S3150801391004B1012030B5164B04789942A8BF19465F
S3150801392083B00D1608140A12A723032C8DF8041068
S315080139308DF801508DF802008DF803208DF80030BE
S3150801394013DC0C4D0C4835F81410002224F08EFCBB
S315080139500522694609484FF47A7327F017FF35F8A7
S3150801396014100548012224F081FC03B030BD00BFC4
S3150801397000FE7F009C070020000C024004B10120D4
S315080139802DE9F04301290B464FF6FF78B8BF01230D
S3150801399083B043450778A8BF43468DF80430A6226D
S315080139A01B120026032F8DF80330ADF800208DF881
S315080139B0026002DD03B0BDE8F083DFF888900C46AB
S315080139C0054639F817101D48324624F04FFC4FF4C6
S315080139D07A73694605221A4827F0D8FE39F817106E
S315080139E01648012224F042FC44452D78A8BF4446D6
S315080139F0211622148DF80440A8232412032D8DF8CC
S31508013A0001108DF802208DF803408DF80030D1DCC5
S31508013A1039F815100948324624F028FC69464FF44E
S31508013A207A730522064827F0B1FE39F815100348BE
S31508013A30012224F01BFC03B0BDE8F083000C024010
S31508013A4004B101209C07002030B54FF6FF73994257
S31508013A500478A8BF194683B00D1608140A12A823BC
S31508013A60032C8DF804108DF801508DF802008DF89D
S31508013A7003208DF8003013DC0A4D0B4835F8141075
S31508013A80002224F0F3FB0522694608484FF47A73AD
S31508013A9027F07CFE35F814100348012224F0E6FBD2
S31508013AA003B030BD9C070020000C024004B1012080
S31508013AB02DE9F04F067883B04FF0A0080423032EB2
S31508013AC0CDF800808DF8043002DD03B0BDE8F08F33
S31508013AD03D4D0C46074635F816103C48002224F0A1
S31508013AE0C5FB4FF47A7369460522394827F04EFE1D
S31508013AF035F816103548012224F0B8FB3E784FEA0E
S31508013B00146BC4F3074AC4F30729A123E4B2032EAD
S31508013B108DF801B08DF802A08DF803908DF8044058
S31508013B208DF80030D1DC35F816102848002224F02B
S31508013B309DFB4FF47A7305226946254827F026FE30
S31508013B4035F816102148012224F090FB3E788DF8AD
S31508013B5001B0AD23032E8DF802A08DF803908DF8E0
S31508013B6004408DF80030B0DC35F8161017480022ED
S31508013B7024F07CFB4FF47A7305226946144827F032
S31508013B8005FE012235F81610104824F06FFB3C7823
S31508013B90CDF800800022032C8DF8042095DC35F839
S31508013BA014100A4824F062FB69464FF47A73052219
S31508013BB0074827F0EBFD35F814100448012224F0D4
S31508013BC055FB03B0BDE8F08F9C070020000C0240AE
S31508013BD004B1012070B56C4B024693E8030092B01C
S31508013BE0147800908DF80410D3E9020104908DF839
S31508013BF01410D3E9040106908DF81C10D3E90601C7
S31508013C0008908DF82410D3E908010A908DF82C1034
S31508013C10D3E90A010C908DF83410D3E90C0100267A
S31508013C20A522A023042C109002928DF80C608DF821
S31508013C303C600E938DF8441000F2A380534D54480E
S31508013C4035F81410324624F011FBC82305226946BB
S31508013C50504827F09BFD35F814104D48012224F0F1
S31508013C6005FB35F814104A48324624F0FFFAC823F2
S31508013C70052202A9474827F089FD35F8141044485A
S31508013C80012224F0F3FA35F814104148324624F09B
S31508013C90EDFAC823052204A93E4827F077FD35F831
S31508013CA014103B48012224F0E1FA35F8141038487B
S31508013CB0324624F0DBFAC823052206A9354827F03F
S31508013CC065FD35F814103248012224F0CFFA35F88B
S31508013CD014102F48324624F0C9FAC823052208A928
S31508013CE02C4827F053FD35F814102948012224F0F1
S31508013CF0BDFA35F814102648324624F0B7FAC82317
S31508013D0005220AA9234827F041FD35F81410204851
S31508013D10012224F0ABFA35F814101D48324624F076
S31508013D20A5FAC82305220CA91A4827F02FFD35F84C
S31508013D3014101748012224F099FA35F8141014487A
S31508013D40324624F093FAC82305220EA9114827F012
S31508013D501DFD35F814100E48012224F087FA35F8AE
S31508013D6014100B48324624F081FA052210A9094895
S31508013D70C82327F00BFD35F814100548012224F055
S31508013D8075FA12B070BD00BF209604089C07002082
S31508013D90000C024004B101202DE9F04F83B001293E
S31508013DA09DF830909DF834809DF838A014461E463B
S31508013DB0054600F0AB80022900F0A5802846FFF7EA
S31508013DC009FF544A2F786C63A242A8BF22461316EC
S31508013DD08DF8013013148DF804208DF80230121273
S31508013DE0A723032F8DF803208DF8003007DD2E86D3
S31508013DF085F8409085F8418003B0BDE8F08F464CC0
S31508013E00464834F81710002224F030FA4FF47A7332
S31508013E1069460522424827F0B9FC34F817103F488D
S31508013E20012224F023FA012E95F800B02E86334696
S31508013E30B8BF01231912A6220027BBF1030F8DF87B
S31508013E4004308DF80310ADF800208DF80270CFDC30
S31508013E5034F81B1031483A4624F008FA4FF47A73BD
S31508013E60052269462E4827F091FC34F81B102B4889
S31508013E70012224F0FBF995F800B08DF80270321290
S31508013E80A823BBF1030F8DF804608DF80320ADF864
S31508013E900030ADDC34F81B1020483A4624F0E6F928
S31508013EA04FF47A73052269461D4827F06FFC34F8EA
S31508013EB01B101A48012224F0D9F92E7885F840906A
S31508013EC09023032E85F841808DF802A08DF8039082
S31508013ED08DF80480ADF800308EDC34F816100F48E2
S31508013EE03A4624F0C3F969464FF47A7305220C4819
S31508013EF027F04CFC34F816100848012224F0B6F9CC
S31508013F0003B0BDE8F08FFFF7F5FA57E7FFF7D0FBE7
S31508013F1054E700BF00FE7F009C070020000C02400A
S31508013F2004B1012030B583B004788DF80310032C51
S31508013F304FF090018DF804208DF80230ADF800108D
S31508013F4013DC0B4D0B4835F81410002224F08EF9BA
S31508013F500522694608484FF47A7327F017FC35F8A5
S31508013F6014100448012224F081F903B030BD00BFC2
S31508013F709C070020000C024004B1012030B58DB029
S31508013F800024264B00941A6B254842F001021A6355
S31508013F901A6B02F001020092009A01945A6C42F4DB
S31508013FA080725A645B6C089403F48073019302224D
S31508013FB0032306A9CDE90623019D23F09BFF194892
S31508013FC0194B1A4A03604FF480310123CDE90344A2
S31508013FD00294059484600461047680F82040C462E2
S31508013FE0C46080F8304041608262C361436123F056
S31508013FF069F960B90122012300240A48049402A937
S31508014000CDE9022323F0FEFA20B90DB030BD1EF02A
S315080140108BFCEFE71EF088FC0DB030BD003802407E
S315080140200000024070AE0120002001400100000F8F
S3150801403010B50168164A88B000239142CDE90233CA
S31508014040CDE90433069301D008B010BD02F58C32D0
S315080140500093516C0F4841F480715164516C01F41D
S315080140608071009100990193116B41F0010111636F
S31508014070126B049302F0010201920323062202A99C
S31508014080CDE90223019C23F035FF08B010BD00BF1E
S3150801409000200140000002400A4808B50A4B0360A7
S315080140A000231022C0E905338383C0E90123C0E94F
S315080140B0033323F061FB00B908BDBDE808401EF0D3
S315080140C033BC00BFB8AE01200064004030B50168BA
S315080140D0184A89B000239142CDE90233CDE9043368
S315080140E0069301D009B030BD02F5EA320093116C8E
S315080140F0114841F000711164116C01F000710091D1
S3150801410000990193136B43F008031363136B03F0D0
S31508014110080301930923019A06930022032302A99E
S3150801412003240225CDE90245CDE9042323F0E2FE65
S3150801413009B030BD00640040000C024030B5134898
S31508014140134B036083B00023CDE9003323F02EFC23
S3150801415088B93C2400250D4800226946CDE9004569
S3150801416023F03AFC70B909486946102223F034FC59
S3150801417020B903B030BD1EF0D7FBEAE71EF0D4FB29
S3150801418003B030BD1EF0D0FBEDE700BFE0AE012065
S315080141900074004010B50168164A88B000239142A0
S315080141A0CDE90233CDE90433069301D008B010BD39
S315080141B002F5E2320093116C0F4841F00051116487
S315080141C0116C01F00051009100990193116B41F0B6
S315080141D001011163126B049302F001020192032398
S315080141E0302202A9CDE90223019C23F083FE08B0FF
S315080141F010BD00BF007400400000024010B582B037
S315080142000024304B00941A6B42F480021A631A6B2D
S3150801421002F480020092009A01941A6B42F4001289
S315080142201A631B6B03F400132246019307210C2022
S31508014230019B23F037FB0C2023F06CFB2246082157
S315080142400E2023F02FFB0E2023F064FB22460921C2
S31508014250102023F027FB102023F05CFB22460A21BD
S31508014260112023F01FFB112023F054FB224621467F
S315080142702F2023F017FB2F2023F04CFB2246052184
S315080142803A2023F00FFB3A2023F044FB2246032170
S315080142903B2023F007FB3B2023F03CFB224604216D
S315080142A0452023F0FFFA452023F034FB2246062158
S315080142B0462023F0F7FA462002B0BDE8104023F065
S315080142C029BB00BF003802402DE9F04F00248DB00C
S315080142D0CDE90644CDE90844654B00940A941A6B66
S315080142E0DFF89481DFF894B1DFF89491614DDFF836
S315080142F094A142F010021A631A6B02F0100200929E
S31508014300009A01941A6B42F004021A631A6B02F0BE
S3150801431004020192019A02941A6B42F080021A630E
S315080143201A6B02F080020292029A03941A6B42F007
S3150801433001021A631A6B02F001020392039A0494AA
S315080143401A6B42F002021A631A6B02F00202049215
S31508014350049A05941A6B42F008021A631B6B03F060
S3150801436008030593404601221021059B23F07EFF91
S315080143702246584642F2C32123F078FF2246484690
S3150801438048F2010123F072FF224628464FF61061D2
S3150801439023F06CFF28460122802123F067FF22467D
S315080143A050464FF44C7123F061FF224640460321E3
S315080143B023F05CFF0026002706A9404613220123A5
S315080143C0CDE90623CDE9086723F094FD584606A9E9
S315080143D042F2C3220123CDE90623CDE9086723F07A
S315080143E089FD06A9484648F201020123CDE90623BB
S315080143F0CDE9086723F07EFD4FF0010C404606A97A
S315080144004FF680720023CDF820C0CDE9062323F0AC
S3150801441071FD06A928464FF690620123CDE90623C8
S31508014420CDE9086723F066FD484606A94FF4807270
S315080144300223CDE90623CDE908670A9423F05AFD3C
S31508014440284606A908220023CDE90623089423F065
S3150801445051FD4FF44C72012306A95046CDE9086770
S31508014460CDE9062323F046FD0DB0BDE8F08F00BF68
S3150801447000380240000C02400010024000080240C9
S3150801448000000240000402400B480C4908B50C4BD9
S3150801449003604FF480420023C0E90233C0E90533C3
S315080144A0C0E907334160026124F0C8F800B908BDC4
S315080144B0BDE808401EF038BAF4AE0120801A06009D
S315080144C00054004070B50268184B88B000249A421F
S315080144D0CDE90244CDE90444069401D008B070BD83
S315080144E0134D00942B6B134843F002032B632B6B7C
S315080144F003F002030093C0221223CDE9022301220D
S315080145000323CDE9042302A904230693009E23F07D
S31508014510F1FC01942B6C43F400132B642B6C03F40C
S3150801452000130193019B08B070BD00BF0054004001
S315080145300038024000040240BFF34F8F0549064B7D
S31508014540CA6802F4E0621343CB60BFF34F8F00BF22
S31508014550FDE700BF00ED00E00400FA05704700BF63
S31508014560F8B5B94B93F90030F3B9B84C2378002B59
S3150801457000F0BC80012B00F08180B548B54DB64EE0
S31508014580B0F900302968B6F90020052BDBBF0623F0
S315080145900380D81E0320132963DC14218242296073
S315080145A067DB043B3380F8BD012BFCD1A74C22788D
S315080145B0002A00F0CC80012A7CD0A84AA84DA94936
S315080145C01068B5F90070B1F90060A74B0E2800F321
S315080145D0A78093ED007ADFEDA56AB4EEE67AF2EEEE
S315080145E0067A0F20F1EE10FA67EE277A106011DDD0
S315080145F0FDEEE77A17EE900AB8EEE77AC2ED007A91
S31508014600DFED9B7AB4EEE77AF1EE10FA40F3B88063
S3150801461098481060002FC0F29780C82FC4BFC823DE
S315080146202B80002EC0F28D80C82EC4BFC8230B80F4
S31508014630F3F7A8FF82A3D3E90023F4F70DF88E4E0A
S3150801464004460D463068F3F79DFF22462B46F4F7DC
S3150801465075FA0028A7D020462946F4F7ADFA306046
S31508014660F8BDB1F5B45FC4BF4FF4B45129608242B5
S3150801467097DA012A97DC02233380F8BD7F4B1B7832
S315080146800B3B082B3FF679AF01A252F823F000BF86
S31508014690B3480108D3480108194801089148010897
S315080146A0F74701087B450108D14701087B45010801
S315080146B0A5470108714B1B780B3B082B3FF67DAFCD
S315080146C001A252F823F000BFC3490108A74901080E
S315080146D05D49010831490108E3490108BB4501085B
S315080146E07F490108BB450108F548010863490A786D
S315080146F00C2A00F087810E2A00F098810B2A7FF494
S315080147003CAF5348534D544EDFF880C1B0F90030E1
S315080147102968B6F9002001278CF80070277034E75C
S31508014720D3ED007AB2EE067A67EE877A07EE100ABB
S31508014730B8EEC77AB4EEE77AF1EE10FA7FF560AF14
S3150801474056E700230B8073E700232B8069E74B4864
S3150801475001780C2900F090810E2900F07A810B2945
S315080147607FF42BAF3D4A3E4D3E49DFF820C1106824
S31508014770B5F90070B1F9006023708CF8003024E7B0
S31508014780B0F5167FFFF646AF3D4CC31784FB00C450
S31508014790C3EBA40303EB8303B0EB43031CBFC01AAB
S315080147A0106037E7374B93F90030002B40F0D6817C
S315080147B02748354A03881478264D274E2968B6F9BD
S315080147C000201B1B1BB20380304C01272770DCE637
S315080147D02C4B93F90030002B40F07B811C482A4B67
S315080147E004881B781B4D1C4E2968B6F90020234402
S315080147F01BB20380E8E7234B93F90030002B40F006
S31508014800BC811348134D0388134E2968B6F9002055
S3150801481014331BB20380D7E71A4B93F90030002BE8
S3150801482040F066810A480B4D03880B4E2968B6F994
S315080148300020143B1BB20380C6E700BFAFF300801C
S31508014840BA490C022B87863F6C070020F81B00200B
S3150801485048060020AC070020280B0020B00B0020DA
S3150801486040AB01203EAB01206C310020A38BAE3F4B
S3150801487000BA5B49A0BB0D00B80B0020E4A90120D2
S3150801488067666666712D0020C80200209807002019
S31508014890A54B93F90030002B40F03881A348A44D6D
S315080148A00388A44E2968B6F90020013B1BB2038090
S315080148B08AE7A14F9D489E4D9E4EB0F90030296862
S315080148C0B6F900204FF0010C87F800C000272770C1
S315080148D05BE6954B93F90030002B40F05C819348D9
S315080148E0934D0388934E2968B6F9002001331BB20C
S315080148F0038069E7914B93F90030002B40F0B081B2
S315080149008F4A106844F24F6398428E4B1B7840F3E6
S315080149104C826FF0270101FB030010608A4D8B4919
S31508014920B5F90070B1F90060834B01241C704CE69F
S31508014930824B93F90030002B40F0B081804A106811
S31508014940B0F5167FACBF053800F1FF307E4D7F49C3
S31508014950B5F90070B1F900601060E5E7774B93F996
S315080149600030002B40F04281754A774D106877492F
S31508014970B5F90070B1F9006014381060D4E76F4BCF
S3150801498093F90030002B40F07A816D4A106844F2A1
S315080149904F6398426B4B1B7840F31182282111FB18
S315080149A003001060BAE7654B93F90030002B40F01D
S315080149B08F81634A1068B0F5167FACBF0A300130A3
S315080149C0C4E75D4B5E4A604D60491068B5F90070F1
S315080149D0B1F900604FF0010C83F800C00023237081
S315080149E0F3E5564B93F90030002B40F06481544AA5
S315080149F0554D10685549B5F90070B1F90060143084
S31508014A00106091E7484A92F90030002B47D0013BE4
S31508014A105BB249494548464D464E137001230B7012
S31508014A20B6F90020B0F900302968AEE53E480278AB
S31508014A30013252B2022A38DC02703F4A3B483C4DE9
S31508014A403C4EB0F90030296801241470B6F90020EB
S31508014A509BE53A490B7801335BB2022B2CDC0B70D0
S31508014A60354B374A384D39491068B5F90070B1F9EF
S31508014A70006001241C70A8E5304C94F9003013B38A
S31508014A80013B5BB22C482E4A2F4D30492370012336
S31508014A900370B5F900701068B1F9006095E52C4C02
S31508014AA002252A2025700870B3E72A4D03242922F6
S31508014AB02B7004700A70C0E7274D032429232A7036
S31508014AC00C700370CCE7224902252A220D70027068
S31508014AD0D8E7012B6CD11B4B164E1A78348813482C
S31508014AE0134DB0F900302968224412B232806BE6C0
S31508014AF0012B40F089800F4E0C4832880C4DB0F9D5
S31508014B0000302968143A12B232805DE6012B40F072
S31508014B108980084E05483288054DB0F90030296864
S31508014B20013A12B232804FE6712D00204806002064
S31508014B30AC070020280B002098070020722D0020C2
S31508014B40B00B0020C802002040AB01203EAB01207B
S31508014B50702D0020732D0020742D0020012B6FD19C
S31508014B609B4E9C4B32881C789B489C4DB0F9003073
S31508014B702968121B12B2328026E6012B40F0B58055
S31508014B80934E95483288954DB0F90030296814320C
S31508014B9012B2328018E6012B1AD18D4E8E48328810
S31508014BA08E4DB0F900302968013212B232800BE617
S31508014BB0022B40F02D81874B884D1C782968864841
S31508014BC0834EB0F90030B6F9002021442960FBE58F
S31508014BD0022B40F01D81814D7F4829687C4EB0F932
S31508014BE00030B6F9002001312960EDE5012B40F0CE
S31508014BF08A807B4D7B4A2F887B491068B1F9006012
S31508014C000A3F3FB22F808FE6022B40F00181734D98
S31508014C10714829686E4EB0F90030B6F9002014398A
S31508014C202960D1E5022B40F0F3806C4D6A4829686A
S31508014C30674EB0F90030B6F9002001392960C3E59D
S31508014C40022B40F0E580654D624B2C681978624865
S31508014C505F4EB0F90030B6F90020611A2960B3E554
S31508014C60012B5DD15E4D5B4B2F881B785E495D4AF2
S31508014C70B1F900601068FF1A3FB22F8054E6012B84
S31508014C805DD1544B564D1F782B885749554AB1F972
S31508014C90006010681F443FB22F8045E6012B5DD1A5
S31508014CA04F4D504A2F8850491068B1F90060053FA9
S31508014CB03FB22F8038E6012B6AD1494D494A2F88E0
S31508014CC049491068B1F900600A373FB22F802BE6CF
S31508014CD0012B50D1424D434A2F8843491068B1F9F7
S31508014CE0006005373FB22F801EE6022B40F0908008
S31508014CF03A4D39482968364EB0F90030B6F90020E0
S31508014D001431296060E5022B70D13749354A0E887E
S31508014D10334D1068B5F900700A3E36B20E8003E6C7
S31508014D20022B6CD130492B4B0E881B782C4D2D4A02
S31508014D30B5F900701068F61A36B20E80F4E5022B42
S31508014D405DD1244B28491E780B88254D254AB5F98E
S31508014D50007010681E4436B20E80E5E5022B45D177
S31508014D602149204A0E881E4D1068B5F90070053E86
S31508014D7036B20E80D8E5022B38D11B49194A0E885E
S31508014D80174D1068B5F90070053636B20E80CBE5B9
S31508014D90022B2BD11449134A0E88114D1068B5F907
S31508014DA000700A3636B20E80BEE5B0F5167FA6BF8C
S31508014DB06FF0090101FB0300C01A1060AEE5B0F5FA
S31508014DC0167FA6BF0A2111FB0300C0181060A5E5CE
S31508014DD0280B0020C802002048060020AC07002046
S31508014DE040AB0120B00B00203EAB01200D4A0E4D11
S31508014DF00E491068B5F90070B1F9006094E50A4DDD
S31508014E000A49084AB5F90070B1F9006010688BE5DE
S31508014E100748084D084EB0F900302968B6F9002050
S31508014E20D2E400BFB00B002040AB01203EAB01200D
S31508014E3048060020AC070020280B002008B5F6F725
S31508014E402BFD00F0FD03012B03D0042818BF002019
S31508014E5008BD032008BD00BF2DE9F04F6049614830
S31508014E60614F624D91B0FDF78BFD5E48FDF732FD4E
S31508014E705C48FDF769FD5B4890F82A3090F829608F
S31508014E800321F61AFDF7CAFE594B56489B6A0022BA
S31508014E901146FDF7FBFC97F90030F6B2002B40F0FE
S31508014EA0898003AC2968204630F080FEB6B22346D5
S31508014EB04C4832464121FDF7E9FC97F90130002BB0
S31508014EC06ED12968204630F071FE234645487200A6
S31508014ED04121FDF7DBFC97F902304FEA4608002B22
S31508014EE054D12968204630F061FE23463D4806EB39
S31508014EF008024121FDF7CAFC97F90330002B3BD183
S31508014F002968204630F052FE3648DFF8F490DFF87B
S31508014F10F4A0DFF8F4B02346B20041218046FDF73C
S31508014F20B5FC3546002759F8041B4046FDF712FD26
S31508014F300321C0F13C044046FDF770FE9AF90030A2
S31508014F40BB42A4B20ED02A4659F8043C2146404633
S31508014F500137FDF79BFC3544042FADB2E3D111B0FF
S31508014F60BDE8F08F9BF800102A46404669BB214BE5
S31508014F701B68FDF78BFCE6E71F4A55F8233092F9C3
S31508014F8000201E49204630F0A1FDBDE71A4A55F812
S31508014F90233092F900201949204630F097FDA4E7FD
S31508014FA0154A55F8233092F900201449204630F065
S31508014FB08DFD8AE7104A55F8233092F900200F49EA
S31508014FC003AC204630F082FD70E700963C230021B1
S31508014FD0FEF7ECF800214046FDF720FEB3E700BFD7
S31508014FE010A704082CAE0120280300207007002012
S31508014FF03C070020FC0A0020700B002084010508EC
S315080150009C0A0020792D0020F81B00202DE9F04F7D
S31508015010DFF8CC9399F9005093B02DB1012D00F02A
S31508015020088113B0BDE8F08FDFF8B8B3DFF8B8A38D
S31508015030D74CBBF90030DAF80070D64AD649039244
S31508015040204607FB03F7FDF79BFC20460121FDF7E8
S31508015050E5FDD248D24ADFF880C3D24EDFF88C8309
S31508015060A0FB0731A2FB07E24FF41673890903FB7C
S315080150701171D20B48F6A043ACFB01C103FB1273B5
S31508015080C908A0FB030300919B09C74905A830F08D
S315080150901DFD05AB36220A212046FDF7F7FBDAF896
S315080150A00000C249C24B81FB00C183FB0072014467
S315080150B0C717C7EB2111C7EBA20202EB420CC1EBE2
S315080150C00117A0EBCC0CA0EB4700BA4F00910CEBF3
S315080150D08C0C87FB00174FEA4C0C83FB0C13A7EBD0
S315080150E0E0704FEAEC7CCCEBA303B349019005A829
S315080150F030F0ECFC3E2205AB0A212046FDF7C6FB43
S31508015100AE492046FDF73CFC2046FDF7E3FB204669
S31508015110FDF71AFC94F82A3094F8297020460321E1
S31508015120FF1AFDF77BFD9B4A2946936820462A46C6
S31508015130FDF7ACFBBBF90030A14986FB0320DA1762
S31508015140C2EBA00202EB8200A3EB4003FFB2BFB29F
S315080151501BB212B205A830F0B9FC3A4605AB7D215F
S315080151602046FDF793FBBBF900C0964B9649B3F968
S31508015170003086FB0C024FEAEC70C0EBA20086FBFE
S31508015180032600EB8002ACEB420CDA17C2EBA6024F
S3150801519002EB820E0FFA8CF6A3EB4E0300B2CDE9B1
S315080151A000061BB212B205A830F090FC05AB7A00D6
S315080151B07D212046FDF76AFB7E00DAF80020834947
S315080151C0DFF82CA205A830F081FCBA1905AB7D21C0
S315080151D02046FDF75BFB79492046FDF7D1FB2046C2
S315080151E00321FDF71BFDAB463E4658F8041B204636
S315080151F0FDF7B0FB0321C0F178052046FDF70EFD4A
S315080152009AF900305B45ADB200F0FC80324658F899
S31508015210043C294620460BF1010BFDF737FB3E44BA
S31508015220BBF1030FB6B2E0D199F90050012D7FF415
S31508015230F8AE574C6149574D03952046FDF7A0FB3B
S315080152402046FDF747FB2046FDF77EFB94F82A30FA
S3150801525094F8296020460321F61AFDF7DFFC00229F
S31508015260AB6820461146FDF711FB594B1868B0F596
S31508015270167FF6B2C0F2D080DFF87881554FB8F9BB
S315080152800030B7F90010454C454A534D03440B44C9
S31508015290A4FB0301A2FB03C24FF41670890900FBA4
S315080152A01131D20B48F6A04000FB1233A5FB015180
S315080152B0A4FB0303C90805AC00919B09474920468D
S315080152C030F004FCB6B2324623467D213048354DCE
S315080152D0DFF82491DFF824A1DFF824B1FDF7D6FA27
S315080152E0B8F900303649DFF8A88085FB0320DA17BC
S315080152F0C2EBA00202EB8200A3EB40031BB212B27F
S31508015300204630F0E3FB720023467D212048FDF755
S31508015310BDFAB7F900302A4985FB0325DA17C2EB2E
S31508015320A50202EB8200A3EB40031BB212B2204690
S3150801533030F0CCFB7200234632447D214046FDF70E
S31508015340A5FA1E494046FDF71BFB03214046FDF71A
S3150801535065FC3546002759F8041B4046FDF7FAFA5D
S315080153600321C0F178044046FDF758FC9AF900304C
S31508015370BB42A4B263D02A4659F8043C21464046AA
S315080153800137FDF783FA3544032FADB2E3D148E679
S315080153902CAE01203C070020C49F0408B5814E1B92
S315080153A0D55204E96766666614EE04088988888812
S315080153B0ABAAAA2A565555552CEE040810A7040877
S315080153C0F0FA0408280B002050EE040864EE0408DD
S315080153D0B00B00203EAB0120CDCCCCCC70EE04083E
S315080153E06C07002048060020AC070020E8060020CC
S315080153F0712D002040AB0120F4060020722D0020FB
S31508015400F81B00201D4B19783246204609BB039B21
S315080154101B68FDF73BFAF9E6194B1A49DFF86C8068
S31508015420194F83FB0023C217C2EBA30202EB8203C7
S3150801543005ACA0EB4303204630F048FB42E79BF856
S3150801544000102A46404671B9039B1B68FDF71EFAF0
S3150801545091E7009778230021FDF7A8FE0021204651
S31508015460FDF7DCFBD2E6009678230021FDF79EFEC8
S3150801547000214046FDF7D2FB7DE700BFF81B00205F
S3150801548067666666F0FA04083EAB012040AB012068
S315080154902DE9F04FA74DA849DFF8E4A293B02846B5
S315080154A0FDF76EFA2846FDF715FA2846FDF74CFA78
S315080154B095F8293095F82A209AF900409B1ADBB20B
S315080154C0029324B1012C76D013B0BDE8F08F9B4B23
S315080154D003931E4603212846FDF7A0FBF3682246DF
S315080154E021462846FDF7D2F9954BBDF808901A686A
S315080154F0944905AC204630F0E9FA23464A46692123
S315080155002846FDF7C3F9904B8E49B3F9002020468A
S3150801551030F0DCFA23464FEA490269212846FDF7AD
S31508015520B5F98A4B8749B3F9002020464FEA49065F
S3150801553030F0CCFA2346284609EB06026921FDF725
S31508015540A5F9834B93F90030022B00F0E1808149DC
S315080155509A1E204630F0BAFA7648DFF82882DFF834
S3150801556028B223464FEA890269210746FDF78EF9D3
S315080155704D46002658F8041B3846FDF7EBF903217A
S31508015580C0F164043846FDF749FB9BF90030B34284
S31508015590A4B200F097802A4658F8043C21463846BA
S315080155A00136FDF773F94D44042EADB2E2D19AF9ED
S315080155B00040012C88D1614B5E4803931C460321A8
S315080155C0FDF72CFB0022E3685A481146FDF75EF900
S315080155D0614B624A1C68624BBDF808901D686149B7
S315080155E082FB0423E217C2EBA30202EB82036420C7
S315080155F0A4EB430300FB04F005AC90FBF5F0009027
S31508015600204630F063FA23464A4669214948FDF7A0
S315080156103DF9554A554B92F90020204653F8221078
S3150801562030F054FA234643484FEA49026921FDF707
S315080156302DF9474B93F90030022B4FEA49054BD018
S3150801564044499A1E204630F041FA09EB05022346E1
S3150801565069213848374FDFF83481DFF834A1DFF89C
S3150801566018B1FDF713F9424A424B92F90020204638
S3150801567053F8221030F02AFA23464FEA89026921A3
S315080156803846FDF703F94D46002658F8041B3846F7
S31508015690FDF760F90321C0F164043846FDF7BEFA47
S315080156A09AF90030B342A4B21DD02A4658F8043CF0
S315080156B0214638460136FDF7E9F84D44042EADB2C8
S315080156C0E3D101E72C4B19782A463846A9B9039B39
S315080156D01B68FDF7DBF85EE7284B93E803000590A6
S315080156E08DF81810B1E79BF800102A463846B1B96B
S315080156F0039B1B68FDF7CAF8D7E7CDF8009064232A
S315080157000021FDF753FD00213846FDF787FA42E7E8
S315080157101A4B93E8030005908DF818101CE7CDF88D
S31508015720009064230021FDF741FD00213846FDF76D
S3150801573075FABAE72CAE012010A704083C07002029
S315080157400C09002064EE04087C2D00207E2D002023
S31508015750700B002084EE0408B80B002067666666A5
S31508015760B00B002094EE0408782D002024070020B1
S31508015770752D002020070020F81B00207CEE040868
S315080157806C07002000070020732D00201007002059
S31508015790742D00202DE9F04F6F49704891B0FDF73F
S315080157A0EFF86E48FDF7D0F86C480321FDF736FA95
S315080157B06B4B1B78002B00F097806A496748FDF709
S315080157C0DFF86648FDF786F86448FDF7BDF86348D3
S315080157D00321FDF723FA644B6048DB6A0022114670
S315080157E0FDF754F85E4B1B78002B00F09680012BD1
S315080157F000F0AA80DFF8949199F90030F6224FF665
S31508015800FB78002B18FB032803F1FF3298FBF2F80B
S315080158101FFA88F83CDD0024DFF874B14F4FDFF832
S3150801582074A1264613E0ADB2721C514603A830F0A6
S315080158304DF9A91D03AB89B210223846FDF726F8A2
S31508015840013499F90030E4B29C42264620DA032154
S315080158503846FDF7E3F99BF90030B34214FB08F526
S31508015860E1D13F4B1B78012B14FB08F513D0022B12
S3150801587020D0002BD7D114FB08F5ADB2691D0E2334
S31508015880009389B20A230F223846FDF749FBCBE775
S3150801589011B0BDE8F08FADB2691D0E2300933846ED
S315080158A089B20A230F22FDF781FC00213846FDF74C
S315080158B0B5F9B9E714FB08F5ADB2691D0E230093D6
S315080158C0384689B20A230F22FDF770FC291D1023D9
S315080158D0009338460E2289B20C23FDF721FB0021DD
S315080158E03846FDF79BF99FE7204B1C482D220521D9
S315080158F0FCF7CCFF1E4B19482D220F21FCF7C6FFDA
S315080159001C4B164839220521FCF7C0FF1A4B1348D0
S3150801591039226421FCF7BAFF4FE7184B0F482822B2
S315080159201821FCF7B3FF164B0C4834220F21FCF75C
S31508015930ADFF144B094834227021FCF7A7FF084B29
S315080159401B78012B7FF456AF0F4B044828221821E8
S31508015950FCF79CFF4EE700BF78AF04082CAE012088
S31508015960F81B002010A704083C070020A8EE04082D
S3150801597080030508F4E20408AC980408ACEE0408B0
S31508015980CCEE0408D4EE0408E0EE0408700B0020FF
S315080159907A2D002038FC04082DE9F04F2DED028BF5
S315080159A0C94CCA49DFF880A3DFF880B393B0204613
S315080159B0FCF7E6FF2046FCF78DFF2046FCF7C4FFFF
S315080159C094F82A3094F8296020460321F61AFDF73F
S315080159D025F9BF4B002211465B682046FCF756FFA6
S315080159E020460321FDF71AF9BA4ABB4B92F9002062
S315080159F0F6B253F82210B6B205A830F067F805AB2F
S31508015A00204632466E21FCF741FF9AF8003023B151
S31508015A109BF90020012A00F08D81B04BB04AB149AB
S31508015A20750005A830F052F805ABA7482A466E213D
S31508015A30FCF72CFF9AF80030012B2C4600F0B381B5
S31508015A40022B00F0FD80002B40F07981A34BA44A7C
S31508015A50A449344405A830F039F805AB9A482246DA
S31508015A606E21FCF713FF9AF80030012B00F095819F
S31508015A70022B00F0ED8094480121FDF7CFF89AF842
S31508015A8000303BB19BF90030012B00F0F881022B65
S31508015A9000F00A82944A9FED950A136AD2699B1A05
S31508015AA0002BB8BF5B4207EE903AF8EEE77AB400EE
S31508015AB067EE807A9FED8E0ABDEEE78A0234B8EE6C
S31508015AC0C87A77EEC77A27EE800A2EF0B7F8FDEE88
S31508015AD0C07A18EE102A17EE903A092BCCBF8549E1
S31508015AE0854905A82FF0F2FF05AB77482246002124
S31508015AF0FCF7CCFE9AF800303BB19BF90030012B3C
S31508015B0000F0C781022B00F0CA817C4A9FED7C0A0E
S31508015B10136AD2699B1A002BB8BF5B4207EE903A0B
S31508015B20F8EEE77A67EE807A9FED710ABDEEE78AAD
S31508015B30B8EEC87A77EEC77A27EE800A2EF07EF895
S31508015B40FDEEC07A18EE102A17EE903A092BCCBF53
S31508015B506C496D4905A82FF0B9FF05AB5A4822468D
S31508015B604B21FCF793FE694B93F90030002B40F06B
S31508015B70F780674BDFED676AC3ED006A9AF8003074
S31508015B803BB19BF90030012B00F07F81022B00F01D
S31508015B909081614A136AD2699FED550ADFF890919F
S31508015BA09B1A002BB8BF5B4207EE903AF8EEE77AEC
S31508015BB0354687EEA67A0027BDEEC78AF8EEC87A7B
S31508015BC037EE677A27EE000A2EF038F8FDEEC07A2E
S31508015BD018EE102A17EE903A092BCCBF4F495049B7
S31508015BE005A82FF073FF05AB224696213648FCF728
S31508015BF04DFE354803218046FDF710F859F8041B78
S31508015C004046FCF7A7FE0321C0F164044046FDF7B0
S31508015C1005F89BF90030BB42E4B200F097802A46AA
S31508015C2059F8043C214640460137FCF72FFE354416
S31508015C30032FADB2E2D113B0BDEC028BBDE8F08FF4
S31508015C409BF90030012B00F03881022B7FF4FEAE60
S31508015C509BF90030022B7FF40EAF06EB4604204A6F
S31508015C6030491E4D05A82FF031FF224605AB6E219E
S31508015C7015480394FCF70AFE05A91348FCF76AFEC2
S31508015C80294604461048FCF765FEE4B2C3B2039AF6
S31508015C900D480096013304F16D01FDF787FA0A48AC
S31508015CA00021FCF7BBFF95E80300039AADF818102D
S31508015CB0059004F16E0105AB0348FCF7E7FD0248C0
S31508015CC00321FCF7ABFFD6E62CAE012010A704088A
S31508015CD03C0700206C070020E00600208CDF040842
S31508015CE080DF0408FCEE0408EC2E00203F11A039E1
S31508015CF00000C84214EF040820EF0408302F0020E2
S31508015D009694F1382CEF040838EF0408F43F002084
S31508015D102C1D002074D13546201A002044EF0408B2
S31508015D2050EF04080CEF0408F81B0020702D002022
S31508015D30D4060020012B6FD0022B00F0BD809BF901
S31508015D400020022A00F0F18074007FE69AF800101C
S31508015D502A464046B9B9AA4B1B68FCF797FD5EE788
S31508015D60022B05D1A74BDFEDA86AC3ED006A05E74B
S31508015D70012B40F04181DFEDA57AA24BF0EE676A6F
S31508015D80C3ED007AFAE6009664230021FDF70EFAC0
S31508015D9000214046FCF742FF41E79BF90030022B00
S31508015DA07FF469AE07E09BF90030012B36D0022B50
S31508015DB07FF44CAE3444964B18680368DB6B9847FE
S31508015DC00546002800F0E880924B934A934905A8B6
S31508015DD02FF07CFE05A99248FCF7BCFD0321054678
S31508015DE08F48FCF71BFFEBB2013322468C4800961D
S31508015DF06D21FDF7DBF98A480021FCF70FFF05AB9A
S31508015E0022466E218648FCF741FD85480321FCF7A9
S31508015E1005FF9AF800302BE6740025467C4B186876
S31508015E200368DB6B98470746002800F08380794BA7
S31508015E30794A7A4905A82FF049FE05A97848FCF759
S31508015E4089FD032107467648FCF7E8FEFBB20133D4
S31508015E502A46734800966D21FDF7A8F97048002176
S31508015E60FCF7DCFE05AB2A466E216D48FCF70EFDF4
S31508015E706B480321FCF7D2FE9AF80030E0E5694A3F
S31508015E809FED690A5368126A09E6684A5368126AF5
S31508015E9082E6674A9FED670A5368126A3AE6644AD8
S31508015EA09FED640A536834E65E4A9FED5F0A5368BC
S31508015EB0F4E55E4A53686EE67400A5B2564A5E4931
S31508015EC0544F05A82FF002FE2A4605AB6E21544809
S31508015ED00395FCF7DBFC05A95148FCF73BFD394660
S31508015EE005464F48FCF736FDEDB2C3B2039A4C4856
S31508015EF00096013305F16D01FDF758F9484800216F
S31508015F00FCF78CFE97E8030005AB039AADF8181069
S31508015F10059005F16E014248FCF7B8FC404803219B
S31508015F20FCF77CFE9AF800308DE5012B7FF4A0ADD5
S31508015F3074003FE7DFF8E08039484146FCF70AFD7F
S31508015F405FFA80F909F101032A46354800966D2161
S31508015F50FDF72CF939463248FCF760FE98E8070048
S31508015F6005AF03C705AB3A706E212A462C48FCF7E4
S31508015F708DFC2B480321FCF751FE264A2F4905A81B
S31508015F802FF0A4FD05AB26482A4609F16E01FCF758
S31508015F907DFC9AF8003053E5DFF87C8020484146BD
S31508015FA0FCF7D8FCC7B27B1C22461D4800966D211A
S31508015FB0FDF7FCF829461A48FCF730FE98E8070071
S31508015FC005AD03C505AB2A706E2122461448FCF7B8
S31508015FD05DFC13480321FCF721FE0E4A174905A863
S31508015FE02FF074FD05AB0E48224607F16E01FCF74A
S31508015FF04DFC9AF800303BE5024BD3ED006ABDE54E
S315080160003C0700202C1D0020DBAC2D47E4385E46FA
S315080160100C1C00208CDF040880DF0408FCEE040851
S315080160202CAE0120EC2E00203F11A039201A0020A9
S31508016030302F00209694F1380CEF040804EF040879
S315080160402DE9F04FA04FA14C97F90030A049032B39
S31508016050A9B040F36381072B40F39A800B2B40F3D9
S31508016060EF820F2B40F3A183132B40F3FF81162BED
S3150801607040F39A842046FCF783FC2046FCF764FC2F
S3150801608020460321FCF7CAFD0522924BDFF87892D8
S31508016090914DDFF87882F3212046FCF7F7FB8F490B
S315080160A02046FCF76DFC2046FCF714FC2046FCF75D
S315080160B04BFC94F82A3094F8296020460321F61AF5
S315080160C0FCF7ACFD864B87495A681BA82FF0FEFCE6
S315080160D0002211461BAB2046FCF7D8FB824B8349AD
S315080160E01F68A9FB07235B09A5FB0320C3EB031C58
S315080160F000097A0900EB4000A7EB8C07A3EBC00364
S31508016100A8FB02C200971BA800272FF0DFFC1BAAD9
S315080161100323012107A80097F4F770FD744B75490D
S315080161201868A9FB00235B09A5FB0325C3EB031C20
S315080161302D09420905EB4505A0EB8C00A3EBC50328
S31508016140A8FB02C200901BA82FF0C0FC03231BAAC0
S315080161501946009711A8F4F751FD07A8F4F730FE80
S3150801616011A8F4F72DFE644BF6B219681BA82FF097
S315080161701DFD1BABB20028212046FCF787FB11A8A1
S31508016180F4F766FD07A8F4F763FD29B0BDE8F08FBB
S31508016190534B02932046FCF7F3FB2046FCF7D4FB4E
S315080161A020460321FCF73AFD4A4BDFF86481534D3B
S315080161B0DFF860910522F3212046FCF767FB0522EB
S315080161C04F4BF9212046FCF761FB44492046FCF771
S315080161D0D7FB2046FCF77EFB2046FCF7B5FB94F877
S315080161E02A3094F8296020460321F61AFCF716FD91
S315080161F0029B44495A681BA82FF068FC00221146E5
S315080162001BAB2046FCF742FB98F90030F6B2B6B252
S3150801621055F823101BA82FF059FC32461BAB412118
S315080162202046FCF733FB98F901301BA855F82310D3
S315080162302FF04CFC72001BAB41212046FCF726FBD4
S3150801624098F902304FEA460A55F823101BA82FF091
S315080162503DFC06EB0A021BAB41212046FCF716FB67
S3150801626098F90330DFF8B0A055F823101BA82FF0D2
S315080162702DFC1BABB20020464121FCF707FBA346C8
S3150801628035464FF0040859F8041B5846FCF762FBDB
S315080162900321C0F13C045846FCF7C0FC97F90030CD
S315080162A04345A4B200F0D6802A4659F8043C214653
S315080162B0584608F10108FCF7E9FA3544B8F1080F20
S315080162C0ADB2E0D161E700BFA83D00202CAE0120A8
S315080162D078AF0408F4E20408ABAAAAAA10A704082E
S315080162E0FC0A002068EF0408D01A00206CEF0408A5
S315080162F0083800207CEF0408AC0B0020D80A0020DF
S31508016300AC980408A0EF040889888888065BB0055C
S3150801631024030020500A0020F81B0020B54D0295E1
S315080163202046FCF72DFB2046FCF70EFB20460321F1
S31508016330FCF774FC0522B04BDFF8FC92DFF8F4A2F7
S31508016340F9212046FCF7A2FAAC492046FCF718FBCE
S315080163502046FCF7BFFA2046FCF7F6FA94F82A30ED
S3150801636094F8296020460321F61AFCF757FC6A6857
S31508016370A3491BA82FF0AAFB002211461BAB2046F6
S31508016380FCF784FA9F4AA04B92F90020F6B2B6B2FE
S3150801639053F822101BA82FF099FB32461BAB8A2112
S315080163A02046FCF773FA994B99491A781BA82FF0DE
S315080163B08DFB72001BAB8A212046FCF767FA954BC9
S315080163C093491A7875001BA82FF080FB72191BAB2D
S315080163D08A212046FCF75AFA8F4A904B92F90020F7
S315080163E01BA853F822102FF071FB1BABB2002046F5
S315080163F08A21FCF74BFAA34635464FF0000859F8AF
S31508016400041B5846FCF7A6FA0321C0F1870458462F
S31508016410FCF704FC97F900304345A4B20ED02A468E
S3150801642059F8043C2146584608F10108FCF72EFAAA
S315080164303544B8F1040FADB2E1D1A6E69AF80010D9
S315080164402A465846002940F0A681029B1B68FCF79C
S315080164501DFAE4E79AF800102A465846002940F042
S315080164605F82029B1B68FCF711FA1DE7614B0293D9
S315080164702046FCF785FA2046FCF766FA20460321F2
S31508016480FCF7CCFB664BDFF8B0B10522F3212046B9
S31508016490FCF7FCF90522584BF9212046FCF7F6F9D9
S315080164A056492046FCF76CFA2046FCF713FA2046B3
S315080164B0FCF74AFA94F82A3094F829802688049633
S315080164C020460321A8EB0308FCF7A8FB494B5549CD
S315080164D05A681BAD28462FF0F9FA002211462B46B9
S315080164E02046FCF7D3F9504A504B92F900205FFA3F
S315080164F088F853F822104FEA48094FEA560A2846FF
S315080165002FF0E4FA4A462B460AF10A012046FCF71F
S31508016510BDF9DBF840102046FCF71CFA301A00EBEF
S31508016520D07603212046FCF779FB97F900301FFA4C
S3150801653088F2102BC6F34F060392C84600F0508323
S31508016540DBF84030039A3A483146FCF79FF9DBF805
S3150801655044103748FCF7FEF90321AAEB0004344836
S31508016560FCF75CFB97F90030112BA4B200F02C83E1
S315080165702F48DBF84430DFF8C0A0DFF8C0B0214669
S315080165804A460646FCF782F9039B1224984430468C
S315080165900321FCF743FB97F900309C42304640F053
S315080165A0B682244B1B7859462846002B00F0CA822E
S315080165B0DAF848202FF08AFA29463046FCF7CAF954
S315080165C0039B00934246049B814600213046FCF713
S315080165D0EDFD30460021FCF721FB049BA3EB0909DD
S315080165E009EBD979C9F34F012B4642463046FCF7E8
S315080165F04DF99CE2FC0A0020AC98040810A704088F
S315080166005CEF040875030020100A002038030020F7
S3150801661060EF040839030020F43F0020C80A00206F
S31508016620F4E2040894EF0408E0370020AC0A0020DD
S315080166302CAE0120F81B0020400A0020BCEF0408FC
S31508016640C14B02932046FCF79BF92046FCF77CF9DF
S3150801665020460321FCF7E2FABC4B0522F32120462A
S31508016660FCF714F90522BA4BF9212046FCF70EF975
S31508016670B8492046FCF784F92046FCF72BF9204651
S31508016680FCF762F994F82A3094F829602046032128
S31508016690F61AFCF7C3FA029BAF495A681BAD28469E
S315080166A02FF014FA002211462B462046FCF7EEF885
S315080166B0AA4AAB4B92F90020F6B253F82210B6B2A9
S315080166C028462FF003FA32462B4620468A21FCF744
S315080166D0DDF8A44B1A78002A40F02C81A24B0FCB87
S315080166E085E80F002B4672008A21A048DFF87C92C4
S315080166F0DFF8A4A2DFF8A4B2FCF7C8F89C4A9D4BC0
S3150801670092F90020284653F8221074002FF0DEF97A
S315080167102B4632198A219548FCF7B8F8964A974BC1
S3150801672092F90020284653F822102FF0CFF92B466C
S31508016730B2008A214846FCF7A9F835464FF0080801
S315080167405AF8041B4846FCF705F90321C0F18704EA
S315080167504846FCF763FA97F900304345A4B20ED0D0
S315080167602A465AF8043C2146484608F10108FCF72E
S315080167708DF83544B8F10C0FADB2E1D105E59BF8BA
S3150801678000102A464846002940F0B781029B1B683B
S31508016790FCF77CF8E4E7009687230021FCF706FD61
S315080167A000215846FCF73AFA39E6674B0293204628
S315080167B0FCF7E6F82046FCF7C7F820460321FCF764
S315080167C02DFA624BDFF8D8B10522F3212046FCF7F2
S315080167D05DF805225E4BF9212046FCF757F85D491D
S315080167E02046FCF7CDF82046FCF774F82046FCF75E
S315080167F0ABF894F82A3094F82960258820460321B5
S31508016800F61AFCF70BFA029B5D495A681BA82FF08A
S315080168105DF9002211461BAB2046FCF737F8594AA9
S31508016820594B92F90020049569080D4605F10A08A5
S31508016830F6B203911BA853F822102FF047F906EB7D
S31508016840460241461BAB2046FCF720F84F4A504BFF
S3150801685010787500ADB253F8203041462A462046D5
S31508016860FCF714F8DBF830102046FCF773F8049BA4
S31508016870181A00EBD07803212046FCF7CFF997F9CF
S3150801688000300C2BC8F34F08B6B200F0CA81414656
S31508016890DBF830303548DFF80C91DFF8D080324626
S315080168A0FBF7F4FF4FF00D0A59F8041B4046FCF7B5
S315080168B051F8039B03211C1A4046FCF7AFF997F9D7
S315080168C000305345A4B200F00C812A4659F8043C1D
S315080168D021464046FBF7DAFF3544BAF10E0FADB251
S315080168E01BD1DBF83C102148FCF734F8049B181A35
S315080168F000EBD07403211D48FCF790F997F9003095
S315080169000F2BC4F34F0400F08081B200DBF83C3052
S3150801691016482146FBF7BAFF37E44FF00E0AC3E7DC
S3150801692000963C230021FCF741FC00215846FCF760
S3150801693075F9B9E402EB82021649C2EB021228463E
S315080169402FF0C4F8CEE600BFFC0A0020F4E20408E2
S31508016950AC98040810A704089CEF0408442C0020EE
S315080169601C0A002010A90120A4EF04082CAE01205E
S31508016970281D0020080A0020F43C0020C00A002037
S3150801698098EF04081E1A0020F8090020F4090020CF
S31508016990B40A0020B4EF0408600A0020F81B00209E
S315080169A0400A0020740A0020BD4D02952046FBF7D7
S315080169B0E7FF2046FBF7C8FF20460321FCF72EF91F
S315080169C00522B84BDFF8F8B2F3212046FBF75EFF44
S315080169D0B5492046FBF7D4FF2046FBF77BFF204647
S315080169E0FBF7B2FF94F82A3094F82960B4F80080CE
S315080169F020460321F61AFCF711F96A68AB491BA868
S31508016A002FF064F8002211461BAB2046FBF73EFF28
S31508016A10A74AA84B92F9002053F822104FEA5803C7
S31508016A201D46F6B21BA84FEA460A03932FF04EF805
S31508016A3029461BAB52460A312046FBF727FFDBF8EE
S31508016A4050102046FBF786FFA8EB000000EBD07537
S31508016A5003212046FCF7E2F897F90030142B1FFAB8
S31508016A6086F9C5F34F05564600F0A380DBF850308A
S31508016A7091484A462946FBF709FFDBF854108E4828
S31508016A80FBF768FF039B03211C1A8B48FCF7C6F822
S31508016A9097F90030152BA4B27FD0DBF8543086481D
S31508016AA052462146FBF7F2FEDBF858108248FBF7FF
S31508016AB051FFA8EB000000EBD07303217E48C3F316
S31508016AC04F04FCF7ABF897F90030162B57D009EBB2
S31508016AD00602DBF8583078482146FBF7D7FEFFF760
S31508016AE054BB764B19782A464046002940F08380E4
S31508016AF0029B1B68FBF7CAFEE7E60096872300217F
S31508016B00FCF754FB00214846FCF788F828E6DAF832
S31508016B104810FBF71FFF049B181A00EBD070C0F34F
S31508016B204F01DAF8483042463046FBF7AFFE039B81
S31508016B30132C98441FFA88F80AF1040A3FF425AB86
S31508016B40132424E5DAF8481005933046FBF702FFCB
S31508016B50059B1946029B42461B6881463046FBF750
S31508016B6095FE049BA3EB090909EBD979DAF84830B4
S31508016B70C9F34F0142463046FBF788FED7E74F4B2C
S31508016B80197809EB060200297BD1029B4A481B6842
S31508016B900292FBF77BFE029A9BE7484B197800297C
S31508016BA040F09080029B44481B685246FBF76EFEF4
S31508016BB073E7424B1978002956D1029B20461B6878
S31508016BC04A46FBF763FE51E73C4B1978002940F02A
S31508016BD08680334B38481B684A46FBF757FEC7E49D
S31508016BE0364B1978002940F087802D4B20461B68C3
S31508016BF0FBF74CFEA4E4039B00960021FCF7D6FAAA
S31508016C0000214046FCF70AF85FE62C4B1978B200DA
S31508016C1089B9029B28481B680292FBF737FE029A3C
S31508016C2074E6264B197899B9029B20461B683246A9
S31508016C30FBF72CFE2BE6049B1F48009600210292C7
S31508016C40FCF7B4FA1C480021FBF7E8FF029A5DE657
S31508016C502046049B009632460021FCF7A7FA2046F7
S31508016C600021FBF7DBFF12E62046CDF800904346EC
S31508016C704A460021FCF79AFA20460021FBF7CEFF87
S31508016C80F4E60D48CDF80090434600210292FCF740
S31508016C908DFA09480021FBF7C1FF029A19E700BFDF
S31508016CA0FC0A0020F4E2040810A7040890EF04087F
S31508016CB049AA0120D40A00202CAE0120F81B002085
S31508016CC0400A0020039B1248CDF800905246002145
S31508016CD0FCF76CFA0E480021FBF7A0FFDDE6039BE3
S31508016CE000930B4853464A460021FCF75FFA0848C9
S31508016CF00021FBF793FF3BE42046049B0092002109
S31508016D00FCF754FA20460021FBF788FF18E400BF78
S31508016D102CAE0120184B93F90030A3B1012B14D0E6
S31508016D20022B17D0032B10D0042B18D0092B0CD00B
S31508016D30082B16D0072B08D00A2B03D0062B15D003
S31508016D40052B02D0704720F0C5B90C484FF4E13144
S31508016D5020F0F2B909484FF4613120F0EDB920F07D
S31508016D6081B907484FF4E13120F0E6B903484FF4F9
S31508016D70966120F0E1B900BF442C002064B30120DC
S31508016D80A8B3012048B9074B93F86030012B05D900
S31508016D900549064A00230B7013707047044B0122FC
S31508016DA01A70F5E754180020441D00202809002010
S31508016DB0E4A9012008B5F4F76FFD012805D00328D9
S31508016DC002D0042818BF002008BD074B1B7B2BB92E
S31508016DD001460648F3F706FC032008BD03480021CF
S31508016DE0F3F700FC032008BD541800206C3E002070
S31508016DF070B5F4F751FD012801D0032070BD314E5D
S31508016E003578002D2ED03048F3F7E8FB2F4B2E4866
S31508016E101968F3F7EBFE2E48F3F7E0FB2D48F3F775
S31508016E20DDFB2948F3F7D6FB012834D02A4801218E
S31508016E30F3F7D8FB29480121F3F7D4FB28480121A8
S31508016E40F3F7D0FB274B1B78002B33D0022BD4D179
S31508016E503378002BD1D0244B1D4801211970F3F743
S31508016E60C1FBCAE7044601461748F3F7BBFB174BB4
S31508016E7015489968F3F7BAFE1B4B15481D7021464C
S31508016E80F3F7B0FB13482146F3F7ACFB0E48F3F7CB
S31508016E90A1FB0128CAD10C48F3F79CFB0128D1D1E3
S31508016EA00D48F3F79BFB0D48F3F798FB0C48F3F7EE
S31508016EB095FBC7E70C4A064813700121F3F792FBC5
S31508016EC0032070BDD91A0020842D00207C070020DC
S31508016ED0D03C0020B03600200C1E00205836002079
S31508016EE0781F0020F4090020441D0020012800D045
S31508016EF0704708B5054B064819682EF057FEBDE8D8
S31508016F000840034903225620F2F77CBA9437002039
S31508016F10D0A801201D4B1B780B3B042B04D8DFE8B6
S31508016F2003F01218212D04007047194A19491368EC
S31508016F30096805338B42136001DB01391160164B71
S31508016F4001221A7070471549134A01230B701370F1
S31508016F5070470F4A0F491368096801338B4213605A
S31508016F60EDDBEAE70A4B1A68053A002A1A60E6DAFF
S31508016F7000221A60084B01221A707047044B1A68DE
S31508016F80013A002A1A60DADAF2E700BFE4A9012019
S31508016F90FC1E002000A9012098070020F81B0020EC
S31508016FA0044B1A780B2A04D1034901202A220870B6
S31508016FB01A707047E4A901209807002030B585B0FA
S31508016FC020B10128034620D005B030BD344A354CDE
S31508016FD0536800930325D36E3349526925703348A4
S31508016FE02EF074FD324B3149C2B21A7031484FF452
S31508016FF07A7325F02BFC41F2883020F051F90121F2
S315080170002D48F2F7AFFF05B030BD2C4A2C49107850
S315080170102C4A244D137051F82000264C00230A22CD
S3150801702003A92B702FF092FC6368984203D001469E
S31508017030204620F081F8244B197811BB236933BB0C
S31508017040224B1B7893B9E3682BBB154B20499A68E9
S3150801705016482EF03BFD164B1449C2B21A70154854
S315080170604FF47A7325F0F2FB05B030BD012BECD154
S31508017070E368B3F5005FE8D00E48022120F080F8F6
S31508017080E3E70129DCD12369B3F5C06FD8D00948F4
S3150801709020F05CF8D4E70748012120F071F8D4E71D
S315080170A094030020C0330020C8EF04081CA901205E
S315080170B018A9012064B30120E8A90120C1330020E1
S315080170C098090508063400200534002007340020F5
S315080170D000EF040830B5044683B018B1012827D05B
S315080170E003B030BD1E491F481F4DF2F7D5F81F4A98
S315080170F01F4853680093D36E047052691D491E4890
S3150801710003242C702EF0E2FC1C4B1B49C2B21A70E8
S315080171101B484FF47A7325F099FB41F2883020F029
S31508017120BFF81848012103B0BDE83040F2F71ABF8D
S3150801713015480E4A0C4B0470926814490E480024EF
S315080171401C702EF0C3FC0D4B0B49C2B20C481A70C9
S315080171504FF47A7303B0BDE8304025F077BB00BF22
S31508017160D0EF0408E02E0020C0330020940300204D
S3150801717008340020C8EF04081CA9012018A9012019
S3150801718064B30120E8A901200634002000EF0408B1
S315080171902DE9F04784B0F4F77FFB012824D0C31EFC
S315080171A0DBB2012B4DD9022803D0002004B0BDE87B
S315080171B0F087264B1B782B2BF7D1254A254E264DD2
S315080171C053682649926E2648002434702C702EF096
S315080171D07DFC244B2249C2B21A7023484FF47A73B4
S315080171E025F034FB2046E1E7204B1A4E0FCB6C46BF
S315080171F084E80F00337823BB174F1B4DDFF85090F7
S31508017200DFF86C800DF1100A3B782846CBB954F8A3
S31508017210041B1FF091FFD9F80820114841462EF0AA
S3150801722055FC104B0E49C2B21A7028464FF47A73B0
S3150801723025F00CFB322020F033F833780BB9A24540
S31508017240E2D1032004B0BDE8F08700BFE4A901201C
S3150801725094030020C033002006340020F8F90408FE
S315080172601CA9012018A9012064B301205896040815
S3150801727000EF0408000000002DE9F047844D2C6852
S315080172802DED028B002C32D1824B834E1B6832685E
S31508017290013B934209D001DD013232607F4B012265
S315080172A01A70BDEC028BBDE8F0877D4C7D4F2378C3
S315080172B0002B00F098801FF0EDFF7B4B3A68821A8D
S315080172C0B3F9000008EE102AF1F75CF9774B0022B2
S315080172D0F1F7C2F9F1F7B8FCB8EE488A07EE900A59
S315080172E0B4EEE78AF1EE10FA00F3BF802C68012CA0
S315080172F0D4D1694E3368002B30D16D4FDFF8C88180
S315080173003B7883B31FF0C6FF674BD8F80020821A73
S31508017310B3F9000008EE102AF1F734F9634B00229D
S31508017320F1F79AF9F1F790FCB8EE488A07EE900A58
S31508017330B4EEE78AF1EE10FAB0DD33685D495A1CFE
S3150801734000230B7032603B702B601FF0A3FF5A4A73
S315080173505A4913880860013313809FE7C4BF03F1B4
S31508017360FF3333609AE71FF095FFDFF860A13C70A1
S31508017370C8F800001FF08EFFDAF80040DFF85091D8
S31508017380001B07EE900AF8EE677A17EE900AF1F7F6
S315080173900BF93DA3D3E90023F1F75EF9F1F734FCC4
S315080173A04749D9F800300A684EF6602C0CFB0044B0
S315080173B002EB000C434AC1F800C0034414604FF4C1
S315080173C07E700422C9F80030CAF80040F2F79CF82A
S315080173D0494604224FF47D70F2F796F83B78002B64
S315080173E03FF45CAF8EE71FF055FFDFF8E090386099
S315080173F0012323701FF04EFFD9F800A0DFF8D080D3
S31508017400A0EB0A0007EE900AF8EE677A17EE900AE3
S31508017410F1F7CAF81CA3D3E90023F1F71DF9F1F72F
S31508017420F3FB2749D8F800300A684EF6602C0CFBA6
S3150801743000AA02EB000C234AC1F800C00344C2F8B3
S3150801744000A04FF47E700422C8F80030C9F800A0E5
S31508017450F2F75AF8414604224FF47D70F2F754F8D0
S315080174602378002B3FF442AF25E733681149013BE6
S3150801747000223360012322702B600A701FF00AFF75
S315080174800E4B2C68186032E71E82BD9CEC79F13EE2
S315080174907436002024090020FC1E002098070020CD
S315080174A03F1D002044AB01203EAB0120000059409E
S315080174B0401D00203D1D002042AB0120A8370020B9
S315080174C0083800200CA8012048AB012010A801208B
S315080174D0D01A002030B583B00546F0F7A3FE421C4A
S315080174E0104601922DF02AFD044618B1019A294643
S315080174F02DF034FD2046F0F795FE98B1431E23443E
S3150801750001E001380ED01A46013B11782F29F8D12E
S31508017510012807D00023137020462BF0A5FD052866
S3150801752010D028B1204603B0BDE830402DF00EBD7D
S31508017530214609482EF056FA204603B0BDE83040E8
S315080175402DF004BD2046FFF7C5FF20462BF08CFD24
S315080175500028E7D1ECE700BFD8EF04082DE9F04F82
S31508017560DB4BDC4ADFEDDC6AD3ED007A9FEDDB7A93
S3150801757000232DED108B1360D94A67EEA67A1360A6
S31508017580D84AF0EEE76A1360F4EEC76AD64AF1EE16
S3150801759010FA8BB0136004D5D44BDFEDD57A0122EE
S315080175A01A60D44B1F6841F27E63BA1E9A4200F2F2
S315080175B06882D14B586B07EE100AB8EE477AB7EED8
S315080175C0008AC8EE07BA88EE279AF0F7CBFF02467B
S315080175D00B460020C949F1F769F90B46C849024625
S315080175E0486B07EE900AF8EE677A43EC1E2B88EE95
S315080175F027CAF0F7B7FF02460B460020BF49F1F745
S3150801760055F90B46BF490246486B07EE900AF8EE54
S31508017610677A43EC1F2BC8EE27CAF0F7A3FF024689
S315080176200B460020B549F1F741F90B46B649024622
S31508017630486B07EE900AF8EE677ACDE9022388EEE1
S3150801764027DAF0F78FFF02460B460020AB49F1F720
S315080176502DF9032FCDE9040140F31882AB4ADFED7A
S31508017660AC9A536806933B1F23F00103D2E902A69D
S315080176700333012415680892B0EE69AAF0EE69AAE7
S31508017680B0EE69BA9346079309970194DBE9049822
S31508017690A9EB0505002DB8BF6D42DBE9067407EEB7
S315080176A0905A069BF8EEE77AA8EB0303A7EB0A0ABA
S315080176B0002BB8BF5B4267EE897ABAF1000FA4EBDB
S315080176C00606B8BFCAF1000A06EE90AA002EFDEE1C
S315080176D0E77AB8BF7642F8EEE68A0DEE903AB8EE4A
S315080176E0E77A06EE906AF8EEEDDAB8EEE68A27EE64
S315080176F02B7A6DEE89DA68EE898A28EE098AB4EE64
S31508017700CB7AF1EE10FAFDEEEDDAFDEEE88ABDEE82
S31508017710C88A0BDD17EE900AF0F734FF53EC1E2BDF
S31508017720F0F79AFFF1F790FA0BEE100AF8EEED7AF8
S3150801773067EE8C7AF4EEEA7AF1EE10FA0BDD1DEEBD
S31508017740900AF0F71FFF53EC1F2BF0F785FFF1F7AF
S315080177507BFA0AEE900AF8EEE87A67EEAC7AF4EE6E
S31508017760CA7AF1EE10FA0BDD18EE900AF0F70AFF65
S31508017770DDE90223F0F770FFF1F766FA0AEE100A5F
S31508017780F8EEC87A67EE8D7AF4EEE97AF1EE10FA38
S315080177900BDD18EE100AF0F7F5FEDDE90423F0F724
S315080177A05BFFF1F751FA09EE900ADBE90853A5EBFD
S315080177B00909B9F1000FB8BFC9F10009DBE90AA641
S315080177C007EE909AA3EB0808B8F1000FF8EEE77AEE
S315080177D0AAEB0707B8BFC8F1000806EE908A002F82
S315080177E067EE897AA6EB0404B8BF7F42F8EEE6DABB
S315080177F0002C06EE907AFDEEE77AB8BF6442F8EE01
S31508017800E68AB8EEE77A06EE904A27EE2B7AB8EEC4
S31508017810E68A6DEE89DA68EE898A28EE098AB4EE77
S31508017820C7BAF1EE10FAFDEEEDDAFDEEE88ABDEE25
S31508017830C88A06930BD517EE900AF0F7A3FE53EC08
S315080178401E2BF0F709FFF1F7FFF90BEE100AF8EE18
S31508017850ED7A67EE8C7AF4EEE7AAF1EE10FA0BD51B
S315080178601DEE900AF0F78EFE53EC1F2BF0F7F4FE8F
S31508017870F1F7EAF90AEE900AF8EEE87A67EEAC7AD9
S31508017880B4EEE7AAF1EE10FA0BD518EE900AF0F766
S3150801789079FEDDE90223F0F7DFFEF1F7D5F90AEE05
S315080178A0100AF8EEC87A67EE8D7AF4EEE79AF1EEE9
S315080178B010FA2FD518EE100AF0F764FEDDE9042355
S315080178C0F0F7CAFEF1F7C0F909EE900A22E000BF07
S315080178D048080020483600200024743F0AD7233C74
S315080178E04C360020503600205436002078360020C9
S315080178F0FFFF7F7F00A90120EC2E00200000F03F4A
S31508017900302F0020201A0020641A0020F83F00209A
S3150801791000000000019B079A0233934201930BF181
S31508017920200B7FF4B3AE099F1C46089BBA46DDE9D6
S315080179300489DDE9026703EB041555F8102C2B6859
S3150801794055F80C0C69689B1A002BB8BF5B4207EE09
S31508017950903A55F8082CAB68F8EEE77A091A9A1A9C
S3150801796055F8040CEB68002967EE897AA3EB000346
S31508017970B8BF4942002AFDEEE77AB8BF5242002B4A
S31508017980B8BF5B420DEE901A08EE902AB8EEE77A78
S3150801799006EE903AF8EEEDDAF8EEE88AB8EEE68AFF
S315080179A027EE2B7A6DEE89DA68EE898A28EE098A3E
S315080179B0B4EECB7AF1EE10FA17EE900AFDEEEDDA97
S315080179C0FDEEE88ABDEEC88A04F1010405F1100549
S315080179D009DDF0F7D7FD53EC1E2BF0F73DFEF1F765
S315080179E033F90BEE100AF8EEED7A1DEE900A67EE02
S315080179F08C7AF4EEEA7AF1EE10FA09DDF0F7C2FDB7
S31508017A0053EC1F2BF0F728FEF1F71EF90AEE900A40
S31508017A10F8EEE87A18EE900A67EEAC7AF4EECA7ACE
S31508017A20F1EE10FA09DDF0F7ADFD32463B46F0F707
S31508017A3013FEF1F709F90AEE100AF8EEC87A18EEFC
S31508017A40100A67EE8D7AF4EEE97AF1EE10FA09DD9D
S31508017A50F0F798FD42464B46F0F7FEFDF1F7F4F8CC
S31508017A6009EE900AA2453FF768AF0E4B83ED00BABF
S31508017A700D4BC3ED00AA0D4B83ED00AA0C4BC3EDCC
S31508017A80009A0BB0BDEC108BBDE8F08FDFED099ABB
S31508017A90094B0893B0EE69AAF0EE69AAB0EE69BA85
S31508017AA0012442E7483600204C3600205036002093
S31508017AB05436002000000000F83F002030B5ADF52F
S31508017AC04F7D0146012242A82AF0B2FC002857D16F
S31508017AD0324B5A0758D103F5B43200200021C3E9C5
S31508017AE00001C3E9020110339342F8D12C4D02A8D3
S31508017AF042AA4FF480712BF039FC95F878305BB1C6
S31508017B00002442AA4FF4807102A82BF02FFC95F8A5
S31508017B1078300134A342F4DC42AA4FF4807102A8FA
S31508017B202BF024FC01AB1E497C2242A82AF080FED8
S31508017B3095F96130022B0CDD42AA4FF4807102A837
S31508017B402BF014FC174901AB902242A82AF070FECB
S31508017B50B0B942AA4FF4807102A82BF007FC0F496D
S31508017B6001AB4FF4B43242A82AF062FE40B942A8EA
S31508017B702BF0F8F8B0FA80F040090DF54F7D30BDCD
S31508017B8000200DF54F7D30BD03F5B431C3E9000082
S31508017B90C3E9020010338B42F8D1A7E7F83F00206A
S31508017BA054180020303300202DE9F04F99B00546CE
S31508017BB0F3F772FE0128044643D0032811D004289E
S31508017BC055D0022800F0D38000212846F3F77EFE1F
S31508017BD0924B1B780B2B6FD00324204619B0BDE8B6
S31508017BE0F08F8F492846F3F7B9F92846F3F766FE69
S31508017BF00746F2F72DFD0BAE8A498B4A034606A8BE
S31508017C002DF064FF06A930462BF03CF900283BD13C
S31508017C10864DDFF83CA2A84605F11609142406E0AC
S31508017C20AB7D53B12B7A13F0100B00F0AA804146B5
S31508017C3030462BF0E1F90028F2D0C4F11404E4B27D
S31508017C4023E07B4B1B786BBB0BAE002430462BF035
S31508017C509FF9224628467749F3F726FE284600214A
S31508017C60F3F734FE0324204619B0BDE8F08F724BB2
S31508017C701B780B2B28462ED07049F3F76FF903248E
S31508017C80204619B0BDE8F08F002430462BF080F964
S31508017C903B686B4A9B69934217D10424204619B065
S31508017CA0BDE8F08F0246674967482AF081FBC0B1F3
S31508017CB000BF00240BAEC9E72846F3F705FE0368A3
S31508017CC06249DB699847022487E7224660493846B4
S31508017CD09847042481E7F3F7FBFD0446002869D099
S31508017CE0FEE70BAE504930462BF0CCF80446002887
S31508017CF0ABD14E4FDFF83CB107F1160A8146142C79
S31508017D00A4D0394630462BF077F9804600289DD114
S31508017D10BB7D002B9AD03B7ADB06F2D55046F0F7AD
S31508017D2081FA421C0590104604922BF064FF4146E5
S31508017D30049A80462DF03AF9059B002B67D1242039
S31508017D402BF048FF04F00301012301EB41014246F0
S31508017D50194402938046CDE90099CDF80C90002389
S31508017D600134F2F74DFEE4B24BF8048BC7E7354907
S31508017D70012200202AF01CFB00283FF42EAF00BF89
S31508017D802BE74846F0F74EFA421C05901046049236
S31508017D902BF031FF5946049A83462DF007F9059BC6
S31508017DA07BBB013C14F0FF044AF804BB7FF43FAFE8
S31508017DB014246AE72846F3F781FD0646F2F748FCDC
S31508017DC0194A1849034606A82DF080FE3368214A48
S31508017DD01B69934211D12346124906AA0BA82DF015
S31508017DE075FE0BA8FFF76AFE08B972B6FEE71A49CF
S31508017DF02846F3F76BFD0524EFE630469847034618
S31508017E00EAE71A46494658462DF0A8F8C9E71A4638
S31508017E10514640462DF0A2F891E700BFE6A9012098
S31508017E204CF0040860F0040840F00408101C002017
S31508017E30D91A002030A80120E4A9012068F0040815
S31508017E40CD9D000818BA0120B4B5012054180020A8
S31508017E5080A80120C59D0008081F0020F8B5454BDC
S31508017E60454D464C1A884649464E474F28462DF0F9
S31508017E702DFE29462046454D2DF098FE44482D787D
S31508017E8000786573434DA073434A444944482D78A5
S31508017E9012780978E574D0E90750A272E173414B6B
S31508017EA0414A424936781B781278E672A061404EFB
S31508017EB02373D1E9070122743E4B3F4A36781B7872
S31508017EC066742162D2E90761A37465613B4B3C4D37
S31508017ED0E0613C4A3C48A1626662DE69296812682B
S31508017EE00568186A3B686263A363384A384BE662D9
S31508017EF02063384E384812881B882164374936680A
S31508017F000068A4F85420A4F85630354A354B098838
S31508017F10E6636564A064344E344D354812681B68BF
S31508017F20A4F85A10334936882D880088A4F8586071
S31508017F30C4E91323A4F85C50A4F85E00097884F810
S31508017F40601022672C492D4A2D4E2E4D2E48636707
S31508017F502E4B0968126836782D7800781B7884F8D4
S31508017F606160C4E9191284F8625084F8630084F8E0
S31508017F706C30F8BDF63C0020F02D00205418002086
S31508017F807CF00408AB0B0020B00B0020380300205E
S31508017F9039030020E0370020AA0B0020F43F002017
S31508017FA0EC2E002074300020442C0020302F0020B5
S31508017FB010A901201E1A0020201A0020641A002088
S31508017FC0B40B0020AC070020480800204806002012
S31508017FD0280B0020B80B00200C0900203EAB01201D
S31508017FE000A901202409002040AB01207C2D002096
S31508017FF07E2D00206C070020280300202403002082
S31508018000700B0020782D0020752D00206C32002081
S3150801801030B4384B384A9D7B384C15703848DD7B6F
S31508018020257038491D7C0570374A5D7C374C0D70C3
S31508018030DD7C15709D69364825625D69E5611C6AB6
S3150801804034490462DC69C4619C6A334A0C625C6A1D
S31508018050CC611C6B1462DC6AD461D3E90D242F4D03
S315080180602F4830492A60DA6B04600A602E482F4986
S315080180701C6C5D6C2E4A04600D602E489D6C156063
S315080180802D4CB3F8545005802C49B3F85650258029
S315080180902B4AB3F858500D802A48B3F85A50158020
S315080180A0294CB3F85C5005802849B3F85E50258001
S315080180B0274A93F860500D70264893F86150157059
S315080180C0254C93F86250057093F863502570D3E9EF
S315080180D019452249224A23480C6093F86C401560D9
S315080180E00470D3E91C032049204A086030BC136098
S315080180F0704700BF5418002039030020F43F0020C0
S31508018100442C002010A90120E0370020EC2E002085
S31508018110302F0020201A0020641A0020AC07002006
S31508018120B00B0020B80B0020B40B00204808002033
S315080181300C09002048060020280B002040AB01202E
S315080181403EAB01207C2D00207E2D00206C070020EF
S31508018150700B0020782D0020752D002028030020A3
S31508018160240300206C32002000A9012024090020E4
S3150801817030B589B00446F3F78FFB01281CD00328D4
S3150801818004D0042804D0022811D0002009B030BD3B
S315080181906D48F2F773FD012852D06B48F2F76EFD70
S315080181A020466A49F3F792FB052009B030BDFFF76F
S315080181B02FFF002009B030BD654C664B94F960204D
S315080181C005A853F82210F0F7D5FF634805A9F2F779
S315080181D04BFD05A8F1F710F8237B012B36D05F4933
S315080181E005A8F0F7C7FF5E4805A9F2F73DFD05A802
S315080181F0F1F702F800215448F2F73EFD594905A85E
S31508018200F0F7B8FF05A95848F2F732FD05A8F0F7C7
S31508018210F3FF626B554902A82DF058FC02A905A87F
S31508018220F0F7A8FF524805A9F2F71EFD05A8F0F7D1
S31508018230E3FF94F96030012B45D0DBB10320A5E7B4
S3150801824020460021F3F742FB05209FE7494905A887
S31508018250F0F790FF05A94248F2F706FD05A8F0F7E1
S31508018260CBFF454B19780129C4D13748F2F704FDEC
S315080182704249C4E7424905A8F0F77CFF05A94148E8
S31508018280F2F7F6FC05A8F0F7B7FFB4F954303E4803
S315080182903E4980FB0320DA17C2EBA00202EB8200FB
S315080182A0A3EB40031BB212B202A82DF00FFC02A9E0
S315080182B005A8F0F75FFF334805A9F2F7D5FC05A82D
S315080182C0F0F79AFFBAE7324905A8F0F753FF2D48A8
S315080182D005A9F2F7CDFC05A8F0F78EFFA36BB3F558
S315080182E0167F0EDA2848294980FB0320DA17C2EBE4
S315080182F0A00202EB8200A3EB400302A82DF0E6FBE5
S31508018300D5E7B4F95820B4F95A10224C2248134437
S315080183100B44A4FB03214FF41675A0FB030289093C
S315080183201E4805FB1131D20BA0FB010148F6A040FE
S3150801833000FB1233A4FB0303C90800919B091849E2
S3150801834002A82DF0C3FBB2E7AC3700200C3F002092
S3150801835054180020E006002008330020A8F004087D
S31508018360B832002088F00408143D0020E40105080D
S315080183709032002084F004087430002098F0040834
S31508018380C8F00408E032002067666666F0FA040859
S31508018390ACF00408B5814E1BD55204E9CDCCCCCC42
S315080183A0B8F004082DE9F047E24FDFF8F483DFF867
S315080183B0F493DFF8F4A30C4682B0054616463B460D
S315080183C0DD49DE4A20462DF081FB2046EFF72AFFDC
S315080183D033460246214628462AF062FBBB7AD84A2A
S315080183E0414620462DF072FB2046EFF71BFF334628
S315080183F00246214628462AF053FBFB7AD14A4146D2
S3150801840020462DF063FB2046EFF70CFF3346024664
S31508018410214628462AF044FB7B7BCB4A4146204627
S315080184202DF054FB2046EFF7FDFE33460246214662
S3150801843028462AF035FBBB7BC44A414620462DF027
S3150801844045FB2046EFF7EEFE33460246214628460F
S315080184502AF026FB97F90F30BD4A414620462DF0F2
S3150801846035FB2046EFF7DEFE33460246214628460F
S315080184702AF016FB97F91030B64A414620462DF0E8
S3150801848025FB2046EFF7CEFE33460246214628460F
S315080184902AF006FB7B7CB04A414620462DF016FBA6
S315080184A02046EFF7BFFE33460246214628462AF004
S315080184B0F7FA97F91230A94A414620462DF006FBEC
S315080184C02046EFF7AFFE33460246214628462AF0F4
S315080184D0E7FA97F91330A24A414620462DF0F6FAF3
S315080184E02046EFF79FFE33460246214628462AF0E4
S315080184F0D7FA7B699B4A414620462DF0E7FA204682
S31508018500EFF790FE33460246214628462AF0C8FA76
S31508018510BB69954A414620462DF0D8FA2046EFF721
S3150801852081FE33460246214628462AF0B9FAFB69F6
S315080185308E4A414620462DF0C9FA2046EFF772FECB
S3150801854033460246214628462AF0AAFA3B6A884A51
S31508018550414620462DF0BAFA2046EFF763FE334628
S315080185600246214628462AF09BFA7B6A814A4146F9
S3150801857020462DF0ABFA2046EFF754FE3346024665
S31508018580214628462AF08CFABB6A7B4A4146204690
S315080185902DF09CFA2046EFF745FE33460246214662
S315080185A028462AF07DFAFB6A744A414620462DF090
S315080185B08DFA2046EFF736FE33460246214628460F
S315080185C02AF06EFA3B6B6E4A414620462DF07EFA3A
S315080185D02046EFF727FE33460246214628462AF06B
S315080185E05FFA7B6B41464A4620462DF06FFA2046D4
S315080185F0EFF718FE33460246214628462AF050FA76
S31508018600BB6B604A414620462DF060FA2046EFF7DB
S3150801861009FE33460246214628462AF041FAFB6BF3
S315080186204146524620462DF051FA2046EFF7FAFD0B
S3150801863033460246214628462AF032FAFB6B524651
S31508018640414620462DF042FA2046EFF7EBFD334628
S315080186500246214628462AF023FA386CEFF7A4FF8A
S31508018660494ACDE90001414620462DF02FFA204618
S31508018670EFF7D8FD33460246214628462AF010FA76
S31508018680786CEFF791FF414ACDE900014146204652
S315080186902DF01CFA2046EFF7C5FD33460246214662
S315080186A028462AF0FDF97B6B4A46414620462DF0BD
S315080186B00DFA2046EFF7B6FD33460246214628460F
S315080186C02AF0EEF9BB6C324A414620462DF0FEF9F6
S315080186D02046EFF7A7FD33460246214628462AF0EB
S315080186E0DFF9FB6C2B4A414620462DF0EFF920466F
S315080186F0EFF798FD33460246214628462AF0D0F977
S315080187003B6D254A414620462DF0E0F92046EFF714
S3150801871089FD33460246214628462AF0C1F9B7F9AA
S3150801872054301E4A414620462DF0D0F92046EFF72F
S3150801873079FD3BE054180020F4F00408D4F004084D
S3150801874000F1040828F1040844F104085CF104085E
S3150801875074F1040888F104089CF10408B8F10408C6
S31508018760D4F10408E8F104080CF2040830F204080C
S3150801877058F204087CF20408A0F20408C4F20408BA
S31508018780E8F2040830F3040898F30408C0F304086F
S31508018790E4F3040808F404082CF4040850F4040863
S315080187A01CF104080CF3040864F304083346024672
S315080187B0214628462AF074F9B7F956309F4A4146A8
S315080187C020462DF083F92046EFF72CFD3346024665
S315080187D0214628462AF064F9B7F95830984A41469D
S315080187E020462DF073F92046EFF71CFD3346024665
S315080187F0214628462AF054F9B7F95A30914A414692
S3150801880020462DF063F92046EFF70CFD3346024664
S31508018810214628462AF044F9B7F95C308A4A414686
S3150801882020462DF053F92046EFF7FCFC3346024665
S31508018830214628462AF034F9B7F95E30834A41467B
S3150801884020462DF043F92046EFF7ECFC3346024665
S31508018850214628462AF024F997F960307C4A414690
S3150801886020462DF033F92046EFF7DCFC3346024665
S31508018870214628462AF014F997F96130754A414686
S3150801888020462DF023F92046EFF7CCFC3346024665
S31508018890214628462AF004F997F962306E4A41467C
S315080188A020462DF013F92046EFF7BCFC3346024665
S315080188B0214628462AF0F4F897F96330674A414673
S315080188C020462DF003F92046EFF7ACFC3346024665
S315080188D0214628462AF0E4F897F96430604A414669
S315080188E020462DF0F3F82046EFF79CFC3346024666
S315080188F0214628462AF0D4F897F96530594A41465F
S3150801890020462DF0E3F82046EFF78CFC3346024665
S31508018910214628462AF0C4F897F96630524A414654
S3150801892020462DF0D3F82046EFF77CFC3346024665
S31508018930214628462AF0B4F897F967304B4A41464A
S3150801894020462DF0C3F82046EFF76CFC3346024665
S31508018950214628462AF0A4F897F96830444A414640
S3150801896020462DF0B3F82046EFF75CFC3346024665
S31508018970214628462AF094F897F969303D4A414636
S3150801898020462DF0A3F82046EFF74CFC3346024665
S31508018990214628462AF084F897F96A30364A41462C
S315080189A020462DF093F82046EFF73CFC3346024665
S315080189B0214628462AF074F897F96B302F4A414622
S315080189C020462DF083F82046EFF72CFC3346024665
S315080189D0214628462AF064F897F86C30284A414619
